:100000000C94AC470C94CD470C94B5D10C94CD47CF
:100010000C94CD470C94CD470C94CD470C94CD4710
:100020000C94CD470C94CD470C94CD470C94E0D361
:100030000C94CD470C94CD470C94ECB50C94CD4763
:100040000C94CD470C94CD470C94CD470C94CD47E0
:100050000C94CD470C94CD470C94CD470C94CD47D0
:100060000C94CD470C94CFD10C945ED10C94CD4719
:100070000C9435CB0C94D7CA0C9413CB0C94CD476D
:100080000C9480D20C94CD470C94CD470C94CD4762
:100090000C94CD470C94CD470C94CD470C94CD4790
:1000A0000C94CD470C94CD470C94CD470C94C5BC13
:1000B0000C9469BD0C94CD470C94CD470C94DDB7DE
:1000C0000C94CD470C94CD470C94CD470C94CD4760
:1000D0000C94CD470C94CD470C94CD470C94CD4750
:1000E0000C9478A70C94CD470C94CD470C94CD4735
:1000F0000C94CD470C94CD470C94CD470C94CD4730
:100100000C949CBC0C9440BD0C9473BC0C9417BD17
:100110000C94CD470C94CD470C94CD470C94CD470F
:100120000C94CD470C94CD470C94CD470C94CD47FF
:100130000C94CD470C9441B70C94CD470C94CD470B
:100140000C94CD470C94CD470C94CD470C94CD47DF
:100150000C94CD470C94CD470C946EA70C94CD47CE
:100160000C94CD470C94CD470C94CD470C94CD47BF
:100170000C94CD470C94CD470C94CD470C94CD47AF
:100180000C94CD470C94CD470C94CD470C94CD479F
:100190000C94CD470C94CD470C94CD470C94CD478F
:1001A0000C94EEBC0C9492BD0C94CD470C94CD47AE
:1001B0000C948FB70C94CD470C94CD470C94CD473D
:1001C0000C94CD470C94CD470C94CD470C94CD475F
:1001D0000C94CD470C94CD470C94CD470C94CD474F
:1001E0000C94CD470C94CD4705720F72197223728F
:1001F0002E723478347834783478347834723478B1
:1002000034783478347834783478367240724A727C
:1002100054725E7234783478347834783478347840
:1002200068723478BE7234783478347834783478BC
:1002300034783478FD7234781976347834783478B8
:10024000347834783478347834781976347834786B
:1002500034782A732F733973437345734F735A730A
:100260003478657334783478A27334783478347899
:10027000347834783478347834783478347834781E
:100280003478347834783478AC733478347834789B
:10029000347834783478347834783478B673F373C7
:1002A0003074797483749C749C74A674B074BA743A
:1002B000C474CE74D374DD74E774327832783278D3
:1002C00032783278327832783278327832783278DE
:1002D00032783278327832783278327832783278CE
:1002E0003278A6743278327832783278327832784E
:1002F00032783278327832783278327832783278AE
:10030000327832783278F174FB7405750F75327873
:1003100032783278327832783278327832789C7427
:10032000BF777E7782778A7766776A777277767714
:100330009677AB77B377B777BB7717788E778A7571
:100340009B75AC75347834782475F6713478BD7546
:10035000CE75DF7519768D740176347835753478FD
:10036000F075467519753478347834785775687532
:1003700079750CBC14BC1CBC24BC2CBC34BC3CBC6F
:1003800044BC24BF88BE90BE98BEA0BEA8BEB0BE6E
:10039000B8BEC0BEC8BED0BED8BEE0BEE8BEF0BECD
:1003A00008BF08BF08BF08BF08BF08BF08BF08BF15
:1003B00008BF08BF08BF08BF08BF08BF08BF08BF05
:1003C00008BF08BF08BF08BF08BF08BF08BF08BFF5
:1003D00008BF08BF08BF08BF08BF08BF08BF08BFE5
:1003E00008BF08BF08BFF8BE00BF084AD73B3BCED6
:1003F000016E84BCBFFDC12F3D6C74319ABD568324
:100400003DDA3D00C77F11BED9E4BB4C3E916BAADB
:10041000AABE000000803F05A84CCDB2D44EB9382A
:1004200036A9020C50B9918688083CA6AAAA2ABE11
:10043000000000803F07634236B79BD8A71A39688F
:100440005618AEBAAB558C1D3CB7CC5763BD6DED9D
:10045000FD753EF6177231BF000000803F080000B6
:1004600000BE922449123EABAAAA2ABECDCCCC4CE7
:100470003E00000080BEABAAAAAA3E00000000BF5A
:10048000000000803F0000000000084178D3BB431B
:1004900087D1133D190E3CC3BD4282AD2B3E68ECA3
:1004A0008276BED98FE1A93E4C80EFFFBE01C4FF2A
:1004B0007F3F0000000000000C94D0AE0C94BA7492
:1004C0000C94296F0C9476BE0C94BDA80C947CBB44
:1004D0000C94AEBB0C94C3680C94C7630C94A964D1
:1004E0000C94E8790C94DECD0C9476780C94057518
:1004F0000C945A730C94C9A80C94FED00C94C47933
:100500000C940F720C9472CA0C94E25A0C9400BFB3
:100510000C9435750C94B0BE0C94CE740C94DC5BCA
:100520000C948C5E0C9424640C943AAD0C94475A51
:100530000C945C570C94665A0C94F7BA0C9414659E
:100540000C94F0750C9407BB0C94E3470C94645F17
:100550000C9413CA0C94A26E0C94D9470C946F5748
:100560000C941B4F0C948A5E0C94EE5A0C94BC575E
:100570000C94CF470C94C1A80C942F730C94D0BE4C
:100580000C944E680C94CABB0C941CBC0C94BB77A6
:100590000C942CBC0C94F0790C9476770C9465AD8B
:1005A0000C94B3CF0C94A35E0C94535D0C94CEBB0F
:1005B0000C94F1590C94D25A0C946E7A0C941864E1
:1005C0000C94DE5A0C94C85B0C9468750C9488BE2D
:1005D0000C9481570C94DD4E0C9468BA0C945FAD6A
:1005E0000C94C4740C9434720C94CE750C94AABB05
:1005F0000C940A5B0C94C45B0C94025B0C948A7799
:100600000C94BCAE0C949D570C946E4B0C94DA5A1F
:100610000C946D590C94F3730C944ACE0C94867818
:100620000C94EA5A0C94C05B0C942E580C9444BC65
:100630000C9475570C9436720C949B750C94F2C9FB
:100640000C944F5E0C9434BC0C94E1680C94F8BE8E
:100650000C94F25A0C942E720C9478CC0C940F7566
:100660000C94BD750C94735B0C944FC20C94BC5EDF
:100670000C9420640C94A6570C94065B0C9487573A
:100680000C94C1540C94CDA80C94FE5A0C9422489E
:100690000C9461AD0C9436AD0C94215A0C941975E0
:1006A0000C94D2570C94C0BE0C94E4790C9459BBB2
:1006B0000C94E36B0C94D5A80C94A9AE0C940CBCD0
:1006C0000C9479740C9423720C9430740C9464BE62
:1006D0000C948E770C944FCF0C9424BF0C94E0BEF6
:1006E0000C945B640C940E690C94B4A90C94045C97
:1006F0000C94A9810C94FD5E0C94F85B0C94236916
:100700000C94BF770C94F6570C948A750C948F64F4
:100710000C94B8C10C9443730C94F6710C94E77468
:100720000C9445730C942F7A0C946D6F0C94657334
:100730000C9424750C94F45B0C940C5A0C94C5A87E
:100740000C94B3770C947E770C94D3740C940F5C58
:100750000C94C65A0C944ACD0C9485C90C943973E8
:100760000C94F6590C94D1A80C94997A0C94CC5B07
:100770000C9490BE0C944A720C94D4930C94505BDD
:100780000C943CBC0C94ECAE0C949D5F0C941D5FDF
:100790000C948D740C9454720C9433480C94DDA812
:1007A0000C94C6BB0C9480BA0C942A730C9498BE1B
:1007B0000C9465580C94F0AE0C946CC70C94BE72FB
:1007C0000C94F0BE0C94B8BE0C9427C70C94D2BB0A
:1007D0000C94E45B0C94285E0C94114F0C94F85824
:1007E0000C94885E0C9494680C9466770C948AC17F
:1007F0000C94E05B0C94AF5D0C94CE5A0C9428647E
:100800000C9483740C943D5F0C94F4640C9414BCAD
:100810000C949CCE0C94DF750C9419720C94DD74BE
:100820000C94BD6E0C94E6C10C94D4640C94D3CE9D
:100830000C9408BF0C941BB00C94B6730C94F47910
:100840000C94135A0C941FBB0C946C790C947ABEC4
:100850000C94015E0C94E8BE0C94BF6D0C94C47AA9
:100860000C94B35D0C94C7570C941A5A0C94DD5E2B
:100870000C94B7BB0C9484CA0C9482770C940572C8
:100880000C9446750C94125B0C9475640C94AC73C8
:100890000C9438AD0C94285A0C94D9A80C94E85BAD
:1008A0000C948F580C949C740C94C25A0C94EC5B6E
:1008B0000C94B2BB0C94F1740C94B1810C945E72E4
:1008C0000C945C630C94BF790C94D65A0C94A67467
:1008D0000C94DA5D0C94F65A0C946B810C9445835D
:1008E0000C947B570C9492570C9444B00C946A77F8
:1008F0000C94D05B0C949F850C940C4F0C94C858AE
:100900000C9469570C94E1A80C94EB6B0C94E65A88
:100910000C9474BA0C94FB740C9472770C9401765A
:100920000C94AB770C94CB670C941C640C941976E4
:100930000C94D85B0C9496690C94315B0C94CA5A55
:100940000C94EF4E0C94164F0C9405590C94B777F9
:100950000C94E4AE0C94FA5A0C94B85B0C94E8AE88
:100960000C9434780C943AC10C94D45B0C94AD8103
:100970000C940E5B0C94A8BE0C947E630C94B1573F
:100980000C944F730C9418610C945EBE0C94545BE1
:100990000C94BC5B0C94EC790C94FD720C94AC75CB
:1009A0000C94F05B0C94E5570C94C8BE0C94B07496
:1009B0000C9496770C94D8BE0C94C5590C9457752A
:1009C0000C9432780C9468720C94A2730C9424BC2E
:1009D0000C9417780C94A0BE0C9440720C9479750A
:1009E0005B257325735D20257320257320706F733D
:1009F0006974696F6E2531382E336625730A005B82
:100A0000257325735D202573202573206F6666731B
:100A100065742532302E336625730A005B257325F5
:100A2000735D202573207A65726F206261636B6F3E
:100A300066662531392E336625730A005B257325DA
:100A4000735D202573206C61746368206261636B41
:100A50006F66662531382E336625730A005B257371
:100A600025735D202573206C617463682076656C46
:100A70006F636974792531332E306625732F6D6964
:100A80006E0A005B257325735D20257320736561F5
:100A90007263682076656C6F636974792531322ED4
:100AA000306625732F6D696E0A005B257325735DB3
:100AB00020257320737769746368206D6178253110
:100AC0003764205B303D6F66662C313D686F6D6921
:100AD0006E672C323D6C696D69742C333D6C696DA9
:100AE00069742B686F6D696E675D0A005B257325FD
:100AF000735D20257320737769746368206D696E58
:100B000025313764205B303D6F66662C313D686F60
:100B10006D696E672C323D6C696D69742C333D6C68
:100B2000696D69742B686F6D696E675D0A005B257E
:100B30007325735D20257320726164697573207657
:100B4000616C75652532302E346625730A005B258D
:100B50007325735D202573206A756E6374696F6EEB
:100B600020646576696174696F6E2531342E346650
:100B7000257320286C617267657220697320666135
:100B800073746572290A005B257325735D202573D4
:100B9000206A65726B20686F6D696E672531362E2D
:100BA000306625732F6D696E5E33202A2031206DEB
:100BB000696C6C696F6E0A005B257325735D202577
:100BC00073206A65726B206D6178696D756D253172
:100BD000352E306625732F6D696E5E33202A2031E5
:100BE000206D696C6C696F6E0A005B257325735DFF
:100BF0002025732074726176656C206D696E696D55
:100C0000756D2531372E336625730A005B257325F4
:100C1000735D2025732074726176656C206D617838
:100C2000696D756D2531372E336625730A005B2596
:100C30007325735D2025732076656C6F6369747905
:100C4000206D6178696D756D2531312E30662573A3
:100C50002F6D696E0A005B257325735D2025732057
:100C60006665656472617465206D6178696D756D26
:100C70002531312E306625732F6D696E0A005B2594
:100C80007325735D2025732061786973206D6F640F
:100C900065253138642025730A005B6D615D202075
:100CA0006D696E20617263207365676D656E742572
:100CB00031382E336625730A005B736C5D20207318
:100CC0006F6674206C696D697420656E61626C6515
:100CD000253132640A005B63745D202063686F72A3
:100CE00064616C20746F6C6572616E636525313769
:100CF0002E346625730A005B6A615D20206A756E7A
:100D00006374696F6E20616363656C657261746999
:100D10006F6E25382E306625730A005B6764695D47
:100D20002064656661756C742067636F6465206418
:100D3000697374616E6365206D6F6465253264202C
:100D40005B303D4739302C313D4739315D0A005B1E
:100D50006770615D2064656661756C742067636FA0
:100D60006465207061746820636F6E74726F6C25A7
:100D70003364205B303D4736312C313D4736312ED0
:100D8000312C323D4736345D0A005B67636F5D206E
:100D900064656661756C742067636F646520636F5A
:100DA0006F72642073797374656D253364205B31D1
:100DB0002D3620284735342D473539295D0A005B0B
:100DC00067756E5D2064656661756C742067636F1E
:100DD000646520756E697473206D6F646525356474
:100DE000205B303D4732302C313D4732315D0A00C7
:100DF0005B67706C5D2064656661756C7420676309
:100E00006F646520706C616E6525313064205B30E5
:100E10003D4731372C313D4731382C323D47313950
:100E20005D0A00256320776F726B206F66667365BD
:100E3000743A2531322E336625730A002563206DFE
:100E4000616368696E6520706F736E3A2531312E6B
:100E5000336625730A00256320706F736974696FA8
:100E60006E3A2531352E336625730A00546F6F6C48
:100E7000206E756D626572202020202020202020A9
:100E80002025640A00466565642072617465206DE2
:100E90006F64653A20202020202025730A004469D1
:100EA0007374616E6365206D6F64653A2020202045
:100EB00020202025730A0050617468204D6F6465FE
:100EC0003A202020202020202020202025730A00E6
:100ED000506C616E653A20202020202020202020A8
:100EE000202020202025730A004D6F74696F6E202A
:100EF0006D6F64653A20202020202020202025735B
:100F00000A00436F6F7264696E6174652073797350
:100F100074656D3A20202025730A00556E6974733C
:100F20003A202020202020202020202020202020A7
:100F300025730A00486F6D696E672073746174656C
:100F40003A202020202020202025730A00466565B5
:100F500064686F6C642073746174653A202020208B
:100F6000202025730A004D6F74696F6E20737461C1
:100F700074653A202020202020202025730A004379
:100F800079636C652073746174653A202020202099
:100F90002020202025730A00526177206D6163684C
:100FA000696E652073746174653A20202025730A88
:100FB000004D616368696E652073746174653A20E1
:100FC00020202020202025730A004C696E65206EA9
:100FD000756D6265723A2531306C750A004665653B
:100FE0006420726174653A2531362E336625732F7D
:100FF0006D696E0A0056656C6F636974793A2531C4
:10100000372E336625732F6D696E0A006310321018
:101010001210473935202D20756E6974732D706557
:10102000722D7265766F6C7574696F6E206D6F646A
:101030006500473934202D20756E6974732D7065F5
:10104000722D6D696E757465206D6F6465202869F9
:101050002E652E206665656472617465206D6F640F
:10106000652900473933202D20696E7665727365D6
:101070002074696D65206D6F6465009F107F104757
:101080003931202D20696E6372656D656E74616CF7
:101090002064697374616E6365206D6F64650047D9
:1010A0003930202D206162736F6C7574652064691E
:1010B0007374616E6365206D6F646500F010D81005
:1010C000C210473634202D20636F6E74696E756FC1
:1010D0007573206D6F6465004736312E31202D20E9
:1010E00065786163742073746F70206D6F64650040
:1010F000473631202D2065786163742070617468F3
:10110000206D6F6465002A111B110C1147313920C5
:101110002D20595A20706C616E6500473138202DA2
:1011200020585A20706C616E6500473137202D20A1
:10113000585920706C616E6500B611A4118B116A4C
:10114000114311473830202D2063616E63656C2098
:101150006D6F74696F6E206D6F646520286E6F6EA1
:1011600065206163746976652900473320202D204E
:10117000636F756E74657220636C6F636B776973F0
:101180006520617263206665656400473220202D0A
:1011900020636C6F636B776973652061726320668F
:1011A00065656400473120202D206C696E65617291
:1011B000206665656400473020202D206C696E65CF
:1011C000617220747261766572736520287365653B
:1011D0006B29007D12631249122F121512FB11E1C7
:1011E00011473539202D20636F6F7264696E617409
:1011F000652073797374656D203600473538202D6E
:1012000020636F6F7264696E6174652073797374A3
:10121000656D203500473537202D20636F6F726470
:10122000696E6174652073797374656D203400474D
:101230003536202D20636F6F7264696E617465208E
:1012400073797374656D203300473535202D206325
:101250006F6F7264696E6174652073797374656D04
:10126000203200473534202D20636F6F7264696E21
:101270006174652073797374656D2031004735336F
:10128000202D206D616368696E6520636F6F7264E5
:10129000696E6174652073797374656D00B012AA0C
:1012A00012A312486F6D696E6700486F6D65640028
:1012B0004E6F7420486F6D656400E412DF12DA121D
:1012C000D412CF12C612456E6420486F6C64004879
:1012D0006F6C6400446563656C00506C616E005314
:1012E000796E63004F666600F712F312EE12486FD4
:1012F0006C640052756E0053746F700021131713E5
:1013000011130A1306134A6F6700486F6D696E6701
:101310000050726F6265004D616368696E696E6747
:10132000004F666600571351134B13461342133C8C
:1013300013331353687574646F776E004379636C6D
:101340006500456E640053746F7000416C61726D8E
:1013500000526561647900496E697469616C697AEB
:10136000696E6700BA13B413AE13A913A513A113C2
:101370009C1396139013891385137C13536875740B
:10138000646F776E004A6F6700486F6D696E670023
:101390004379636C650050726F626500486F6C64DE
:1013A0000052756E00456E640053746F7000416C9E
:1013B00061726D00526561647900496E697469619A
:1013C0006C697A696E6700E113CB13473231202DC7
:1013D000206D696C6C696D65746572206D6F6465F4
:1013E00000473230202D20696E63686573206D6F71
:1013F0006465001B1410140414FB135B72616469B0
:1014000075735D005B696E686962697465645D002F
:101410005B7374616E646172645D005B64697361C7
:10142000626C65645D00351431142C1420646567AA
:1014300000206D6D0020696E002A2A2A204E4F542C
:10144000494345202A2A2A20526573657474696EBF
:10145000672062617564207261746520746F202555
:1014600073005B626175645D205553422062617553
:1014700064207261746525313564205B313D3936F5
:1014800030302C323D31393230302C333D3338342A
:1014900030302C343D35373630302C353D31313518
:1014A0003230302C363D3233303430305D0A005B20
:1014B00072786D5D2073657269616C205258206D81
:1014C0006F646525313564205B303D636861725F10
:1014D0006D6F64652C313D6C696E655F6D6F646521
:1014E0005D0A005B65785D2020656E61626C652039
:1014F000666C6F7720636F6E74726F6C2531306429
:10150000205B303D6F66662C313D584F4E2F584F53
:1015100046462C323D5254532F4354535D0A005BD0
:1015200065655D2020656E61626C65206563686F2E
:1015300025313864205B303D6F66662C313D6F6E1F
:101540005D0A005B65635D2020657870616E6420D4
:101550004C4620746F2043524C46206F6E205458E6
:10156000253664205B303D6F66662C313D6F6E5DC5
:101570000A00A515A0159A1594158E1587158015C6
:10158000323330343030003131353230300035379D
:1015900036303000333834303000313932303000BA
:1015A0003936303000300073797300666200000015
:1015B000001702E4794F5E885E763C5238DC437354
:1015C0007973006676000000001703E8794F5E88A3
:1015D0005E7A3CEC51783F737973006870000000CC
:1015E000000700EC79015E8C5E7E3C0000803F735A
:1015F0007973006876000000001700F0794F5EC430
:10160000797F3C0000004173797300696400000039
:10161000000400F4796C79885E723C0000000000E0
:101620000000006E00000000000000C25A015EBC15
:101630005EED3400000000000000006C696E650083
:10164000000000C25AE557BC5EED34000000000007
:1016500000000076656C0000001002285AF65788DA
:101660005E723C00000000000000006665656400DA
:10167000001002475A2E58885E723C00000000009D
:101680000000007374617400000000C65A5C578843
:101690005E723C00000000000000006D616373009A
:1016A000000000CA5A6957885E723C0000000000C2
:1016B0000000006379637300000000CE5A6F578802
:1016C0005E723C00000000000000006D6F7473004B
:1016D000000000D25A7557885E723C00000000007E
:1016E000000000686F6C6400000000D65A7B5788C9
:1016F0005E723C0000000000000000756E6974001E
:10170000000000DE5A8757885E723C00000000002F
:10171000000000636F6F7200000000E25A92578869
:101720005E723C00000000000000006D6F6D6F00F5
:10173000000000E65A9D57885E723C0000000000E1
:10174000000000706C616E00000000EA5AA6578825
:101750005E723C00000000000000007061746800D0
:10176000000000EE5AB157885E723C000000000095
:101770000000006469737400000000F25ABC5788CE
:101780005E723C000000000000000066726D6F0099
:10179000000000F65AC757885E723C000000000047
:1017A000000000746F6F6C00000000FA5AD2578876
:1017B0005E723C000000006D706F006D706F78000D
:1017C000001003045C8F58885E723C000000006DBE
:1017D000706F006D706F7900001003045C8F588883
:1017E0005E723C000000006D706F006D706F7A00DB
:1017F000001003045C8F58885E723C000000006D8E
:10180000706F006D706F6100001003045C8F58886A
:101810005E723C000000006D706F006D706F6200C2
:10182000001003045C8F58885E723C000000006D5D
:10183000706F006D706F6300001003045C8F588838
:101840005E723C00000000706F7300706F73780070
:10185000001003F85B6558885E723C000000007061
:101860006F7300706F737900001003F85B65588820
:101870005E723C00000000706F7300706F737A003E
:10188000001003F85B6558885E723C000000007031
:101890006F7300706F736100001003F85B65588808
:1018A0005E723C00000000706F7300706F73620026
:1018B000001003F85B6558885E723C000000007001
:1018C0006F7300706F736300001003F85B655888D6
:1018D0005E723C000000006F6673006F66737800F4
:1018E0000010030F5CC858885E723C000000006F57
:1018F0006673006F667379000010030F5CC8588828
:101900005E723C000000006F6673006F66737A00C1
:101910000010030F5CC858885E723C000000006F26
:101920006673006F667361000010030F5CC858880F
:101930005E723C000000006F6673006F66736200A9
:101940000010030F5CC858885E723C000000006FF6
:101950006673006F667363000010030F5CC85888DD
:101960005E723C00000000686F6D00686F6D65007E
:10197000000000DA5A8157F659723C0000000068F6
:101980006F6D00686F6D7800001000F85BB35D88C4
:101990005EC23400000000686F6D00686F6D7900F2
:1019A000001000F85BB35D885EC33400000000687F
:1019B0006F6D00686F6D7A00001000F85BB35D8892
:1019C0005EC43400000000686F6D00686F6D6100D8
:1019D000001000F85BB35D885EC53400000000684D
:1019E0006F6D00686F6D6200001000F85BB35D887A
:1019F0005EC63400000000686F6D00686F6D6300A4
:101A0000001000F85BB35D885EC734000000007012
:101A100072620070726265000000003AC1B35D88B6
:101A20005EC834000000007072620070726278005C
:101A30000010033AC14F5E885EC934000000007098
:101A400072620070726279000010033AC14F5E88C2
:101A50005ECD3400000000707262007072627A0025
:101A60000010033AC14F5E885ED134000000007060
:101A700072620070726261000010033AC14F5E88AA
:101A80005ED5340000000070726200707262620005
:101A90000010033AC14F5E885ED934000000007028
:101AA00072620070726263000010033AC14F5E8878
:101AB0005EDD34000000006A6F67006A6F677800BF
:101AC0000010003AC1AF5D0C5AE734000000006A14
:101AD0006F67006A6F6779000010003AC1AF5D134D
:101AE0005AE734000000006A6F67006A6F677A0087
:101AF0000010003AC1AF5D1A5AE734000000006AD6
:101B00006F67006A6F6761000010003AC1AF5D2126
:101B10005AE734000000007077720070777231006D
:101B2000000000D2BB07BB885E723C000000007062
:101B30007772007077723200000000D2BB07BB885A
:101B40005E723C00000000707772007077723300A4
:101B5000000000D2BB07BB885E723C000000007032
:101B60007772007077723400000000D2BB07BB8828
:101B70005E723C0000000031000000316D61000029
:101B8000000300AEBBB35D8C5EEE5A000000003176
:101B90000000003173610000001303B2BB4F5E68A8
:101BA000BAF95A6666E63F310000003174720000EF
:101BB000001B04B7BB4F5E74BAFD5A0000204231CF
:101BC000000000316D690000000300C6BBB35D80FA
:101BD000BAEF5A000000413100000031706F000080
:101BE000000300CABBB35DDD5EF35A0000803F31E5
:101BF00000000031706D0000000300CEBBB35DF744
:101C0000BAF45A0000004032000000326D6100005A
:101C1000000300AEBBB35D8C5E0D5B0000803F3205
:101C20000000003273610000001303B2BB4F5E6816
:101C3000BA185B6666E63F3200000032747200003C
:101C4000001B04B7BB4F5E74BA1C5B00002042321D
:101C5000000000326D690000000300C6BBB35D8068
:101C6000BA0E5B000000413200000032706F0000CD
:101C7000000300CABBB35DDD5E125B0000803F3233
:101C800000000032706D0000000300CEBBB35DF7B2
:101C9000BA135B0000004033000000336D610000A8
:101CA000000300AEBBB35D8C5E2C5B0000803F3355
:101CB0000000003373610000001303B2BB4F5E6885
:101CC000BA375B6666E63F3300000033747200008B
:101CD000001B04B7BB4F5E74BA3B5B00002042336D
:101CE000000000336D690000000300C6BBB35D80D7
:101CF000BA2D5B000000413300000033706F00001C
:101D0000000300CABBB35DDD5E315B000000003341
:101D100000000033706D0000000300CEBBB35DF720
:101D2000BA325B0000004034000000346D610000F6
:101D3000000300AEBBB35D8C5E4B5B000000403423
:101D40000000003473610000001303B2BB4F5E68F3
:101D5000BA565B6666E63F340000003474720000D9
:101D6000001B04B7BB4F5E74BA5A5B607607403401
:101D7000000000346D690000000300C6BBB35D8045
:101D8000BA4C5B000000413400000034706F00006A
:101D9000000300CABBB35DDD5E505B0000803F34D2
:101DA00000000034706D0000000300CEBBB35DF78F
:101DB000BA515B000000407800000078616D0000BF
:101DC000000300735BF85805597E330000803F78AC
:101DD00000000078766D0000001B00BC5B4F5EC702
:101DE00063833300007A4678000000786672000052
:101DF000001B00B85B4F5EC7637F3300007A4678F4
:101E000000000078746E0000001B03C45B4F5EC7C7
:101E1000638B33000000007800000078746D0000D0
:101E2000001B03C05B4F5EC763873300009143789C
:101E3000000000786A6D0000001B00C85B4F5E6DFB
:101E4000598F3300409C4578000000786A68000094
:101E5000001B00CC5B4F5EC559933300401C467895
:101E6000000000786A640000001B04D05B4F5EC76E
:101E7000639B330AD7233C7800000078736E000020
:101E8000000300D85BB35D64BEA2320000803F78DF
:101E90000000007873780000000300DC5BB35D6431
:101EA000BEA33200000000780000007873760000C6
:101EB000001B00E05B4F5EC763A33300803B4578A7
:101EC000000000786C760000001B00E45B4F5EC7EA
:101ED00063A7330000C84278000000786C620000FD
:101EE000001B03E85B4F5EC763AB33000020417803
:101EF000000000787A620000001B03EC5B4F5EC7B5
:101F000063AF33000000407900000079616D00008C
:101F1000000300735BF8580559B3330000803F7924
:101F200000000079766D0000001B00BC5B4F5EC7AF
:101F300063B83300007A46790000007966720000C9
:101F4000001B00B85B4F5EC763B43300007A46796C
:101F500000000079746E0000001B03C45B4F5EC775
:101F600063C033000000007900000079746D000048
:101F7000001B03C05B4F5EC763BC330000A0437906
:101F8000000000796A6D0000001B00C85B4F5E6DA9
:101F900059C43300409C4579000000796A6800000C
:101FA000001B00CC5B4F5EC559C83300401C46790E
:101FB000000000796A640000001B04D05B4F5EC71C
:101FC00063D0330AD7233C7900000079736E000098
:101FD000000300D85BB35D64BEA4320000803F798B
:101FE0000000007973780000000300DC5BB35D64DF
:101FF000BEA5320000000079000000797376000071
:10200000001B00E05B4F5EC763D83300803B45791F
:10201000000000796C760000001B00E45B4F5EC797
:1020200063DC330000C84279000000796C62000074
:10203000001B03E85B4F5EC763E03300002041797B
:10204000000000797A620000001B03EC5B4F5EC762
:1020500063E433000000407A0000007A616D000004
:10206000000300735BF8580559E8330000803F7A9D
:102070000000007A766D0000001B00BC5B4F5EC75D
:1020800063ED3300007A447A0000007A6672000043
:10209000001B00B85B4F5EC763E93300007A447AE7
:1020A0000000007A746E0000001B03C45B4F5EC723
:1020B00063F5330000F0C27A0000007A746D00000E
:1020C000001B03C05B4F5EC763F133000000007A62
:1020D0000000007A6A6D0000001B00C85B4F5E6D57
:1020E00059F933000048427A0000007A6A6800001B
:1020F000001B00CC5B4F5EC559FD3300007A447A6B
:102100000000007A6A640000001B04D05B4F5EC7C9
:102110006305340AD7233C7A0000007A736E00000E
:10212000000300D85BB35D64BEA632000000007AF5
:102130000000007A73780000000300DC5BB35D648C
:10214000BEA7320000803F7A0000007A737600005C
:10215000001B00E05B4F5EC7630D3400007A447AD9
:102160000000007A6C760000001B00E45B4F5EC745
:102170006311340000C8427A0000007A6C620000EB
:10218000001B03E85B4F5EC7631534000020417AF3
:102190000000007A7A620000001B03EC5B4F5EC710
:1021A000631934000040406100000061616D00006F
:1021B000000300735BF85805591D3400004040616E
:1021C00000000061766D0000001300BC5B4F5E6490
:1021D0005F22340080CA4661000000616672000020
:1021E000001300B85B4F5E645F1E3400804A466196
:1021F00000000061746E0000001303C45B4F5EC7F3
:10220000632A34000080BF6100000061746D00002B
:10221000001303C05B4F5E645F2634000080BF6123
:10222000000000616A6D0000001300C85B4F5E6D26
:10223000592E3400349E4861000000616A68000035
:10224000001300CC5B4F5EC559323400349E4861A8
:10225000000000616A640000001304D05B4F5E64FC
:102260005F3A34CDCCCC3D6100000061726100006A
:10227000001B03D45B4F5E645F3E34DFC3A9406143
:1022800000000061736E0000000300D85BB35D6462
:10229000BEA8320000803F6100000061737800003A
:1022A000000300DC5BB35D64BEA932000000006186
:1022B0000000006173760000001300E05B4F5E6475
:1022C0005F42340000FA4461000000616C76000057
:1022D000001300E45B4F5E645F46340000FA446123
:1022E000000000616C620000001303E85B4F5E6455
:1022F0005F4A340000A04061000000617A62000083
:10230000001303EC5B4F5E645F4E340000004062DC
:1023100000000062616D0000000300735BF8580567
:10232000595234000000006200000062766D000027
:10233000001300BC5B4F5E645F5734000061456270
:102340000000006266720000001300B85B4F5E641C
:102350005F5334000061456200000062746E00004B
:10236000001303C45B4F5EC7635F34000080BF622D
:1023700000000062746D0000001303C05B4F5E64D8
:102380005F5B34000080BF62000000626A6D000085
:10239000001300C85B4F5E6D5963340000A04162BA
:1023A000000000626A640000001300D05B4F5E64AE
:1023B0005F6F340AD7233C62000000627261000044
:1023C000001B03D45B4F5E645F73340000803F6387
:1023D00000000063616D0000000300735BF85805A6
:1023E000598734000000006300000063766D000030
:1023F000001300BC5B4F5E645F8C3400006145637A
:102400000000006366720000001300B85B4F5E645A
:102410005F8834000061456300000063746E000053
:10242000001303C45B4F5EC7639434000080BF6336
:1024300000000063746D0000001303C05B4F5E6416
:102440005F9034000080BF63000000636A6D00008D
:10245000001300C85B4F5E6D5998340000A04163C3
:10246000000000636A640000001300D05B4F5E64EC
:102470005FA4340AD7233C6300000063726100004C
:10248000001B03D45B4F5E645FA8340000803F7084
:102490003100007031667271001300BDA84F5E6498
:1024A0005FCA590000C84270310000703163736C1C
:1024B000001300C1A84F5E645FCE5900007A4470DB
:1024C0003100007031637368001300C5A84F5E646B
:1024D0005FD2590000FA4470310000703163706CB3
:1024E000001303C9A84F5E645FD6590000003E7018
:1024F0003100007031637068001303CDA84F5E6433
:102500005FDA59CDCC4C3E70310000703177736C7E
:10251000001300D1A84F5E645FDE5900007A44705A
:102520003100007031777368001300D5A84F5E64E6
:102530005FE2590000FA4470310000703177706C2E
:10254000001303D9A84F5E645FE6590000003E7097
:102550003100007031777068001303DDA84F5E64AE
:102560005FEA59CDCC4C3E703100007031706F661F
:10257000001303E1A84F5E645FEE59CDCCCC3D67FC
:102580003534006735347800001B03F05B4F5EC7BD
:1025900063EE32000000006735340067353479009F
:1025A000001B03F05B4F5EC763F232000000006760
:1025B0003534006735347A00001B03F05B4F5EC78B
:1025C00063F632000000006735340067353461007F
:1025D000001B03F05B4F5E645FFA3200000000678F
:1025E0003534006735346200001B03F05B4F5E64D6
:1025F0005FFE320000000067353400673534630049
:10260000001B03F05B4F5E645F0233000000006755
:102610003535006735357800001B03F05B4F5EC72A
:10262000630633000011436735350067353579009F
:10263000001B03F05B4F5EC7630A33000020436753
:102640003535006735357A00001B03F05B4F5EC7F8
:10265000630E3300000000673535006735356100D3
:10266000001B03F05B4F5E645F12330000000067E5
:102670003535006735356200001B03F05B4F5E6443
:102680005F1633000000006735350067353563009D
:10269000001B03F05B4F5E645F1A330000000067AD
:1026A0003536006735367800001B03F05B4F5EC798
:1026B000631E330000000067353600673536790049
:1026C000001B03F05B4F5EC763223300000000670E
:1026D0003536006735367A00001B03F05B4F5EC766
:1026E0006326330000000067353600673536610029
:1026F000001B03F05B4F5E645F2A3300000000673D
:102700003536006735366200001B03F05B4F5E64B0
:102710005F2E3300000000673536006735366300F2
:10272000001B03F05B4F5E645F3233000000006704
:102730003537006735377800001B03F05B4F5EC705
:10274000633633000000006735370067353779009E
:10275000001B03F05B4F5EC7633A33000000006765
:102760003537006735377A00001B03F05B4F5EC7D3
:10277000633E33000000006735370067353761007E
:10278000001B03F05B4F5E645F4233000000006794
:102790003537006735376200001B03F05B4F5E641E
:1027A0005F46330000000067353700673537630048
:1027B000001B03F05B4F5E645F4A3300000000675C
:1027C0003538006735387800001B03F05B4F5EC773
:1027D000634E3300000000673538006735387900F4
:1027E000001B03F05B4F5EC76352330000000067BD
:1027F0003538006735387A00001B03F05B4F5EC741
:1028000063563300000000673538006735386100D3
:10281000001B03F05B4F5E645F5A330000000067EB
:102820003538006735386200001B03F05B4F5E648B
:102830005F5E33000000006735380067353863009D
:10284000001B03F05B4F5E645F62330000000067B3
:102850003539006735397800001B03F05B4F5EC7E0
:102860006366330000000067353900673539790049
:10287000001B03F05B4F5EC7636A33000000006714
:102880003539006735397A00001B03F05B4F5EC7AE
:10289000636E330000000067353900673539610029
:1028A000001B03F05B4F5E645F7233000000006743
:1028B0003539006735396200001B03F05B4F5E64F9
:1028C0005F763300000000673539006735396300F3
:1028D000001B03F05B4F5E645F7A3300000000670B
:1028E0003932006739327800001103F05B4F5E889F
:1028F0005E5F3500000000673932006739327900C9
:10290000001103F05B4F5E885E63350000000067D6
:102910003932006739327A00001103F05B4F5E886C
:102920005E673500000000673932006739326100A8
:10293000001103F05B4F5E885E6B3500000000679E
:102940003932006739326200001103F05B4F5E8854
:102950005E6F35000000006739320067393263006E
:10296000001103F05B4F5E885E7335000000006766
:102970003238006732387800001103F45B4F5E880C
:102980005E77350000000067323800673238790022
:10299000001103F45B4F5E885E7B3500000000672A
:1029A0003238006732387A00001103F45B4F5E88DA
:1029B0005E7F350000000067323800673238610002
:1029C000001103F45B4F5E885E83350000000067F2
:1029D0003238006732386200001103F45B4F5E88C2
:1029E0005E873500000000673238006732386300C8
:1029F000001103F45B4F5E885E8B350000000067BA
:102A00003330006733307800001103F45B4F5E8889
:102A10005E8F350000000067333000673330790087
:102A2000001103F45B4F5E885E9335000000006781
:102A30003330006733307A00001103F45B4F5E8857
:102A40005E97350000000067333000673330610067
:102A5000001103F45B4F5E885E9B35000000006749
:102A60003330006733306200001103F45B4F5E883F
:102A70005E9F35000000006733300067333063002D
:102A8000001103F45B4F5E885EA335000000006A0E
:102A90006964006A696461000000003AC1285E3D13
:102AA0005F923C000000006A6964006A6964620029
:102AB0000000003AC1285E3D5F963C000000006ABD
:102AC0006964006A696463000000003AC1285E3DE1
:102AD0005F9A3C000000006A6964006A69646400EF
:102AE0000000003AC1285E3D5F9E3C00000000737C
:102AF0007973006A61000000001F00125B4F5EC71F
:102B000063BC320024F449737973006374000000DD
:102B1000001F04315B4F5EC763C0320AD7233C738A
:102B2000797300736C000000000700505BB35D8C8C
:102B30005EC43200000000737973007374000000FB
:102B400000070076BEB35D5EBE97320000803F7323
:102B50007973006D74000000001702AABB4F5E1F5E
:102B6000BBEA5A00000040000000006D6500000054
:102B70000000008AC17CBB7CBB723C0000000000EE
:102B80000000006D640000000000008AC159BB59BC
:102B9000BB723C0000000073797300656A0000009E
:102BA000000700A981B35DDD5E843C0000803F73B7
:102BB0007973006A76000000000700AD81B35D6B99
:102BC000815C3F0000A040737973006A73000000CD
:102BD000000700B181B35DDD5E5D3F0000803F73A3
:102BE00079730074760000000007004FC2B35DDD0A
:102BF0005E5D5C0000803F737973007176000000B9
:102C0000000700F0AEB35D1D5F235A0000000073A3
:102C1000797300737600000000070065ADB35DFDB9
:102C20005E305A0000803F737973007369000000C2
:102C300000070061AD015E3AAD315A00007A43737E
:102C400079730065630000000007001864B35D1429
:102C50006574320000000073797300656500000040
:102C60000007001C64B35DF464753200000000735B
:102C700079730065780000000007002064B35DD41C
:102C8000647632000000407379730072786D000042
:102C90000007002464B35DDD5E773200000000733E
:102CA00079730062617564000004002864B35D7E7E
:102CB0006372320000A04000000000737200000048
:102CC0000000005FAD36AD38AD723C000000000082
:102CD0000000007172000000000000E4AEA9AE88A0
:102CE0005E723C00000000000000007169000000FE
:102CF000000000E8AEBCAE885E723C000000000040
:102D0000000000716F000000000000ECAED0AE8843
:102D10005E723C00000000000000006572000000D0
:102D20000000003AC1B4A9885E723C0000000000B7
:102D300000000071660000000000003AC1AF5DF1C4
:102D400059723C0000000000000000727800000092
:102D5000000000B8C15C63885E723C0000000000A7
:102D60000000006D736700000000008AC1AF5D883D
:102D70005E723C0000000000000000636C65617240
:102D80000000003AC1EF4EEF4E723C000000000020
:102D9000000000616C61726D0000003AC1DD4EDD23
:102DA0004E723C0000000000000000706175736509
:102DB0000000003AC10C4F0C4F723C0000000000B4
:102DC00000000073746172740000003AC1114F1169
:102DD0004F723C0000000000000000666C757368D4
:102DE0000000003AC1164F164F723C000000000070
:102DF00000000072657365740000003AC11B4F1B30
:102E00004F723C0000000000000000747874000065
:102E10000000003AC1AF5D8A5E723C000000000015
:102E20000000007469640000000100B8C1015EBCCC
:102E30005EA23C0000000000000000746573740096
:102E40000000003AC16E7A7ABE723C0000000000B9
:102E500000000064656661000000003AC1997A5381
:102E60005D723C0000000000000000626F6F7400A3
:102E70000000003AC1C47ABF79723C000000000033
:102E800000000068656C70000000003AC12F7A886D
:102E90005E723C00000000000000006800000000BE
:102EA0000000003AC12F7A885E723C000000007377
:102EB00079730067706C0000000700FE5AB35DFD77
:102EC0005ED232000000007379730067756E0000F7
:102ED000000700025BB35DDD5ED3320000803F730C
:102EE00079730067636F0000000700065BB35D8CB9
:102EF0005ED1320000803F7379730067706100001B
:102F00000007000A5BB35DFD5ED432000000407331
:102F100079730067646900000007000E5BB35DDD34
:102F20005ED5320000000000000000676300000072
:102F30000000003AC176788678723C0000000000FC
:102F40000000006D61000000001B04545B4F5EC771
:102F500063C932CDCCCC3D756461007564613000CD
:102F6000000300B8C1285E3D5F2E3C0000000075E4
:102F70006461007564613100000300B8C1285E3DE2
:102F80005F323C00000000756461007564613200CE
:102F9000000300B8C1285E3D5F363C0000000075AC
:102FA0006461007564613300000300B8C1285E3DB0
:102FB0005F3A3C0000000075646200756462300096
:102FC000000300B8C1285E3D5F3E3C000000007574
:102FD0006462007564623100000300B8C1285E3D80
:102FE0005F423C000000007564620075646232005C
:102FF000000300B8C1285E3D5F463C00000000753C
:103000006462007564623300000300B8C1285E3D4D
:103010005F4A3C0000000075646300756463300023
:10302000000300B8C1285E3D5F4E3C000000007503
:103030006463007564633100000300B8C1285E3D1D
:103040005F523C00000000756463007564633200E9
:10305000000300B8C1285E3D5F563C0000000075CB
:103060006463007564633300000300B8C1285E3DEB
:103070005F5A3C00000000756464007564643000B1
:10308000000300B8C1285E3D5F5E3C000000007593
:103090006464007564643100000300B8C1285E3DBB
:1030A0005F623C0000000075646400756464320077
:1030B000000300B8C1285E3D5F663C00000000755B
:1030C0006464007564643300000300B8C1285E3D89
:1030D0005F6A3C000000005F7465005F7465780003
:1030E000001002E6C14F5E885E9357000000005F4B
:1030F0007465005F74657900001002E6C14F5E8858
:103100005E9757000000005F7465005F74657A0089
:10311000001002E6C14F5E885E9B57000000005F12
:103120007465005F74656100001002E6C14F5E883F
:103130005E9F57000000005F7465005F7465620069
:10314000001002E6C14F5E885EA357000000005FDA
:103150007465005F74656300001002E6C14F5E880D
:103160005EA757000000005F7472005F7472780001
:10317000001002E6C14F5E885EB858000000005F94
:103180007472005F74727900001002E6C14F5E88AD
:103190005EBC58000000005F7472005F74727A00B9
:1031A000001002E6C14F5E885EC058000000005F5C
:1031B0007472005F74726100001002E6C14F5E8895
:1031C0005EC458000000005F7472005F7472620099
:1031D000001002E6C14F5E885EC858000000005F24
:1031E0007472005F74726300001002E6C14F5E8863
:1031F0005ECC58000000005F7473005F7473310090
:10320000001002E6C14F5E885E2358000000005F98
:103210007073005F70733100001002E6C14F5E886A
:103220005E3358000000005F6373005F637331001A
:10323000001002E6C14F5E885E4358000000005F48
:103240006573005F65733100001002E6C14F5E8850
:103250005E5358000000005F7873005F78733100A0
:10326000001002E6C14F5E885E855B000000005FD3
:103270006665005F66653100001002E6C14F5E883A
:103280005E6358000000005F7473005F7473320067
:10329000001002E6C14F5E885E2758000000005F04
:1032A0007073005F70733200001002E6C14F5E88D9
:1032B0005E3758000000005F6373005F6373320085
:1032C000001002E6C14F5E885E4758000000005FB4
:1032D0006573005F65733200001002E6C14F5E88BF
:1032E0005E5758000000005F7873005F787332000B
:1032F000001002E6C14F5E885E9D5B000000005F2B
:103300006665005F66653200001002E6C14F5E88A8
:103310005E6758000000005F7473005F74733300D1
:10332000001002E6C14F5E885E2B58000000005F6F
:103330007073005F70733300001002E6C14F5E8847
:103340005E3B58000000005F6373005F63733300EF
:10335000001002E6C14F5E885E4B58000000005F1F
:103360006573005F65733300001002E6C14F5E882D
:103370005E5B58000000005F7873005F7873330075
:10338000001002E6C14F5E885EB55B000000005F82
:103390006665005F66653300001002E6C14F5E8817
:1033A0005E6B58000000005F7473005F747334003C
:1033B000001002E6C14F5E885E2F58000000005FDB
:1033C0007073005F70733400001002E6C14F5E88B6
:1033D0005E3F58000000005F6373005F637334005A
:1033E000001002E6C14F5E885E4F58000000005F8B
:1033F0006573005F65733400001002E6C14F5E889C
:103400005E5F58000000005F7873005F78733400DF
:10341000001002E6C14F5E885ECD5B000000005FD9
:103420006665005F66653400001002E6C14F5E8885
:103430005E6F5800000000000000005F64616D00D6
:103440000000003AC1665A665A723C000000000053
:1034500000000073653030000002003AC1DA5DA35D
:103460005E3C5A000000000000000073653031002F
:103470000002003AC1DA5DA35E3E5A00000000007F
:1034800000000073653032000002003AC1DA5DA32B
:103490005E405A00000000000000007365303300F9
:1034A0000002003AC1DA5DA35E425A00000000004B
:1034B00000000073653034000002003AC1DA5DA3F9
:1034C0005E445A00000000000000007365303500C3
:1034D0000002003AC1DA5DA35E465A000000000017
:1034E00000000073653036000002003AC1DA5DA3C7
:1034F0005E485A000000000000000073653037008D
:103500000002003AC1DA5DA35E4A5A0000000000E2
:1035100000000073653038000002003AC1DA5DA394
:103520005E4C5A0000000000000000736530390056
:103530000002003AC1DA5DA35E4E5A0000000000AE
:1035400000000073653130000002003AC1DA5DA36B
:103550005E505A0000000000000000736531310029
:103560000002003AC1DA5DA35E525A00000000007A
:1035700000000073653132000002003AC1DA5DA339
:103580005E545A00000000000000007365313300F3
:103590000002003AC1DA5DA35E565A000000000046
:1035A00000000073653134000002003AC1DA5DA307
:1035B0005E585A00000000000000007365313500BD
:1035C0000002003AC1DA5DA35E5A5A000000000012
:1035D00000000073653136000002003AC1DA5DA3D5
:1035E0005E5C5A0000000000000000736531370087
:1035F0000002003AC1DA5DA35E5E5A0000000000DE
:1036000000000073653138000002003AC1DA5DA3A2
:103610005E605A0000000000000000736531390050
:103620000002003AC1DA5DA35E625A0000000000A9
:1036300000000073653230000002003AC1DA5DA379
:103640005E645A0000000000000000736532310023
:103650000002003AC1DA5DA35E665A000000000075
:1036600000000073653232000002003AC1DA5DA347
:103670005E685A00000000000000007365323300ED
:103680000002003AC1DA5DA35E6A5A000000000041
:1036900000000073653234000002003AC1DA5DA315
:1036A0005E6C5A00000000000000007365323500B7
:1036B0000002003AC1DA5DA35E6E5A00000000000D
:1036C00000000073653236000002003AC1DA5DA3E3
:1036D0005E705A0000000000000000736532370081
:1036E0000002003AC1DA5DA35E725A0000000000D9
:1036F00000000073653238000002003AC1DA5DA3B1
:103700005E745A000000000000000073653239004A
:103710000002003AC1DA5DA35E765A0000000000A4
:1037200000000073797300000000003AC118619D29
:103730005F723C00000000000000007031000000DB
:103740000000003AC118619D5F723C00000000005B
:1037500000000031000000000000003AC118619D27
:103760005F723C000000000000000032000000001A
:103770000000003AC118619D5F723C00000000002B
:1037800000000033000000000000003AC118619DF5
:103790005F723C00000000000000003400000000E8
:1037A0000000003AC118619D5F723C0000000000FB
:1037B00000000078000000000000003AC118619D80
:1037C0005F723C0000000000000000790000000073
:1037D0000000003AC118619D5F723C0000000000CB
:1037E0000000007A000000000000003AC118619D4E
:1037F0005F723C000000000000000061000000005B
:103800000000003AC118619D5F723C00000000009A
:1038100000000062000000000000003AC118619D35
:103820005F723C0000000000000000630000000028
:103830000000003AC118619D5F723C00000000006A
:1038400000000067353400000000003AC118619D97
:103850005F723C000000000000000067353500008A
:103860000000003AC118619D5F723C00000000003A
:1038700000000067353600000000003AC118619D65
:103880005F723C0000000000000000673537000058
:103890000000003AC118619D5F723C00000000000A
:1038A00000000067353800000000003AC118619D33
:1038B0005F723C0000000000000000673539000026
:1038C0000000003AC118619D5F723C0000000000DA
:1038D00000000067393200000000003AC118619D05
:1038E0005F723C00000000000000006732380000FA
:1038F0000000003AC118619D5F723C0000000000AA
:1039000000000067333000000000003AC118619DDC
:103910005F723C00000000000000006D706F00004E
:103920000000003AC118619D5F723C000000000079
:10393000000000706F7300000000003AC118619D24
:103940005F723C00000000000000006F6673000022
:103950000000003AC118619D5F723C000000000049
:10396000000000686F6D00000000003AC118619D02
:103970005F723C00000000000000007072620000F6
:103980000000003AC118619D5F723C000000000019
:1039900000000070777200000000003AC118619DBD
:1039A0005F723C00000000000000006A6F670000CA
:1039B0000000003AC118619D5F723C0000000000E9
:1039C0000000006A696400000000003AC118619DAF
:1039D0005F723C00000000000000007564610000A0
:1039E0000000003AC118619D5F723C0000000000B9
:1039F00000000075646200000000003AC118619D7B
:103A00005F723C000000000000000075646300006D
:103A10000000003AC118619D5F723C000000000088
:103A200000000075646400000000003AC118619D48
:103A30005F723C00000000000000005F7465000041
:103A40000000003AC118619D5F723C000000000058
:103A50000000005F747200000000003AC118619D10
:103A60005F723C00000000000000005F7473000003
:103A70000000003AC118619D5F723C000000000028
:103A80000000005F707300000000003AC118619DE3
:103A90005F723C00000000000000005F63730000E4
:103AA0000000003AC118619D5F723C0000000000F8
:103AB0000000005F657300000000003AC118619DBE
:103AC0005F723C00000000000000005F787300009F
:103AD0000000003AC118619D5F723C0000000000C8
:103AE0000000005F666500000000003AC118619D9B
:103AF0005F723C00000000000000006D000000004C
:103B00000000003AC18F64885E723C000000000033
:103B100000000071000000000000003AC1756488D8
:103B20005E723C00000000000000006F000000001A
:103B30000000003AC15B64885E723C000000000037
:103B400000000024000000000000003AC1A96488C1
:103B50005E723C00000000486F6D696E6720657200
:103B6000726F72202D202563206178697320736540
:103B70007474696E6773206D6973636F6E666967CD
:103B8000757265640050726F62696E67206572724B
:103B90006F72202D20256320617869732063616E28
:103BA0006E6F74206D6F766520647572696E672024
:103BB00070726F62696E67005B69645D2020546992
:103BC0006E7947204944253330730A005B68765D7F
:103BD000202068617264776172652076657273690E
:103BE0006F6E2531362E32660A005B68705D2020CC
:103BF000686172647761726520706C6174666F725F
:103C00006D253132640A005B66765D20206669723C
:103C10006D776172652076657273696F6E253136D6
:103C20002E32660A005B66625D20206669726D77DF
:103C3000617265206275696C642531382E32660ABE
:103C400000456E7465722024626F6F743D3120747C
:103C50006F20656E7465722074686520626F6F7482
:103C6000206C6F616465722E0A000A0A0A232323FE
:103C70002054696E794720424F4F54204C4F4144A5
:103C800045522048656C70202323230A00456E743A
:103C900065722024646566613D3120746F20726511
:103CA000736574207468652073797374656D20740E
:103CB0006F2074686520666163746F727920646533
:103CC0006661756C742076616C7565732E0A546834
:103CD00069732077696C6C206F766572777269748E
:103CE0006520616E79206368616E67657320796F06
:103CF000752068617665206D6164652E0A000A0A88
:103D00000A2323232054696E794720524553544F88
:103D100052452044454641554C54532048656C70EB
:103D2000202323230A00496E766F6B652073656C30
:103D300066207465737420627920656E746572699B
:103D40006E672024746573743D4E207768657265D4
:103D5000204E206973206F6E65206F663A0A20201E
:103D600024746573743D312020736D6F6B6520740E
:103D70006573740A202024746573743D32202068B2
:103D80006F6D696E67207465737420202028796FC9
:103D900075206D757374207472697020686F6D6919
:103DA0006E67207377697463686573290A2020241D
:103DB000746573743D33202073717561726520746E
:103DC00065737420202028612073657269657320F3
:103DD0006F662073717561726573290A20202474DF
:103DE0006573743D342020617263207465737420A0
:103DF000202020202028736F6D65206C617267651C
:103E000020636972636C6573290A202024746573CA
:103E1000743D3520206477656C6C20746573742064
:103E2000202020286D6F7665732073706163656450
:103E30002062792031207365636F6E64206477653A
:103E40006C6C73290A202024746573743D3620201D
:103E500066656564686F6C6420746573742028659A
:103E60006E746572202120616E64207E20746F2044
:103E7000686F6C6420616E64207265737461727423
:103E80002C20726573706563746976656C79290A94
:103E9000202024746573743D3720204D20636F64A7
:103EA000657320746573742020284D20636F6465EA
:103EB0007320696E7465726D696E676C65642077D6
:103EC000697468206D6F766573290A2020247465F3
:103ED00073743D3820204A534F4E2074657374200C
:103EE00020202020286D6F74696F6E2074657374B4
:103EF0002072756E207573696E67204A534F4E208D
:103F0000636F6D6D616E6473290A2020247465737C
:103F1000743D392020696E76657273652074696D11
:103F20006520746573740A202024746573743D31B0
:103F30003020726F74617279206D6F74696F6E20BA
:103F4000746573740A202024746573743D313120C4
:103F5000736D616C6C206D6F76657320746573741E
:103F60000A202024746573743D313220736C6F779E
:103F7000206D6F76657320746573740A2020247435
:103F80006573743D313320636F6F7264696E617461
:103F9000652073797374656D206F66667365742030
:103FA0007465737420284739322C204735342D47E7
:103FB0003539290A0A546573747320617373756DFA
:103FC0006520612063656E746572656420585920B0
:103FD0006F726967696E20616E64206174206C6520
:103FE0006173742038306D6D20636C656172616E31
:103FF000636520696E20616C6C206469726563740E
:10400000696F6E730A546573747320617373756D91
:1040100065205A20686173206174206C6561737437
:104020002034306D6D20706F736969746976652016
:10403000636C656172616E63650A546573747320A5
:10404000737461727420776974682061204730202E
:104050005830205930205A30206D6F76650A486FED
:104060006D696E6720697320746865206578636583
:104070007074696F6E2E204E6F20696E697469616D
:104080006C20706F736974696F6E206F7220636C3F
:10409000656172616E636520697320617373756D0C
:1040A00065640A000A0A0A2323232054696E7947AB
:1040B0002053454C4620544553542048656C70208D
:1040C0002323230A0045616368202420636F6D6DFC
:1040D000616E642061626F766520616C736F20642D
:1040E0006973706C6179732074686520746F6B6597
:1040F0006E20666F722065616368207365747469F1
:104100006E6720696E205B205D20627261636B6563
:1041100074730A546F2076696577207365747469C7
:104120006E677320656E746572206120746F6B65B5
:104130006E3A0A0A2020243C746F6B656E3E0A0AB0
:10414000466F72206578616D706C652024796672A7
:1041500020746F20646973706C61792074686520C5
:1041600059206D6178206665656420726174650A06
:104170000A546F2075706461746520736574746986
:104180006E677320656E74657220746F6B656E2048
:10419000657175616C732076616C75653A0A0A20E9
:1041A00020243C746F6B656E3E3D3C76616C75659A
:1041B0003E0A0A466F72206578616D706C65202436
:1041C0007966723D38303020746F207365742074C6
:1041D00068652059206D617820666565642072618C
:1041E000746520746F20383030206D6D2F6D696ECE
:1041F0007574650A466F7220636F6E6669677572C3
:104200006174696F6E2064657461696C7320736595
:10421000653A2068747470733A2F2F6769746875F3
:10422000622E636F6D2F73796E746865746F732F70
:1042300054696E79472F77696B692F54696E794796
:104240002D436F6E66696775726174696F6E0A00DF
:10425000546865736520636F6D6D616E6473206172
:1042600072652061637469766520666F7220636F82
:104270006E66696775726174696F6E3A0A202024F0
:104280007379732053686F772073797374656D2029
:104290002867656E6572616C292073657474696E38
:1042A00067730A2020243120202053686F77206D07
:1042B0006F746F7220312073657474696E67732038
:1042C000286F72207768617465766572206D6F74EF
:1042D0006F7220796F752077616E7420312C322CCB
:1042E000332C34290A2020247820202053686F772B
:1042F000205820617869732073657474696E6773E0
:1043000020286F7220776861746576657220617805
:10431000697320796F752077616E7420782C792C01
:104320007A2C612C622C63290A2020246D20202005
:1043300053686F7720616C6C206D6F746F7220739F
:10434000657474696E67730A2020247120202053DD
:10435000686F7720616C6C20617869732073657475
:1043600074696E67730A2020246F20202053686FC1
:104370007720616C6C206F6666736574207365745A
:1043800074696E67730A2020242420202053686FEC
:104390007720616C6C2073657474696E67730A2092
:1043A00020246820202053686F7720746869732068
:1043B00068656C702073637265656E0A0A000A0A8C
:1043C0000A2323232054696E794720434F4E4649E0
:1043D0004755524154494F4E2048656C7020232365
:1043E000230A000A466F722064657461696C656413
:1043F0002054696E794720696E666F207365653A4F
:104400002068747470733A2F2F6769746875622E10
:10441000636F6D2F73796E746865746F732F546951
:104420006E79472F77696B692F0A466F722074681F
:1044300065206C6174657374206669726D77617252
:1044400065207365653A2068747470733A2F2F671E
:1044500069746875622E636F6D2F73796E74686509
:10446000746F732F54696E79470A506C6561736578
:10447000206C6F6720616E79206973737565732096
:10448000617420687474703A2F2F7777772E737960
:104490006E746865746F732E636F6D2F666F7275BF
:1044A0006D730A486176652066756E0A000A4E6F64
:1044B00074653A2054696E79472067656E6572614C
:1044C000746573206175746F6D61746963207374B2
:1044D00061747573207265706F72747320627920D5
:1044E00064656661756C740A546869732063616EF3
:1044F0002062652064697361626C65642062792062
:10450000656E746572696E67202473763D300A5358
:104510006565207468652077696B692062656C6FDA
:104520007720666F72206D6F7265206465746169B3
:104530006C732E0A00546865736520636F6D6D613E
:104540006E647320617265206163746976652066AC
:10455000726F6D2074686520636F6D6D616E64208D
:104560006C696E653A0A205E782020202020202089
:1045700020202020202052657365742028636F6EF0
:1045800074726F6C207829202D20736F66747761A8
:1045900072652072657365740A20203F20202020F8
:1045A0002020202020202020204D616368696E6536
:1045B00020706F736974696F6E20616E6420676329
:1045C0006F6465206D6F64656C2073746174650A37
:1045D00020202420202020202020202020202020D7
:1045E00053686F7720616E642073657420636F6E0B
:1045F00066696775726174696F6E2073657474693A
:104600006E67730A202021202020202020202020D7
:104610002020202046656564686F6C64202D20731F
:10462000746F70206D6F74696F6E20776974686F36
:104630007574206C6F73696E6720706F736974692D
:104640006F6E0A20207E2020202020202020202085
:104650002020204379636C65205374617274202D8F
:1046600020726573746172742066726F6D20666566
:104670006564686F6C640A20206820202020202058
:104680002020202020202053686F772074686973D1
:104690002068656C702073637265656E0A20202443
:1046A0006820202020202020202020202053686FF8
:1046B0007720636F6E66696775726174696F6E20CB
:1046C00068656C702073637265656E0A20202474BF
:1046D0006573742020202020202020204C697374D2
:1046E0002073656C662D74657374730A20202474BE
:1046F0006573743D4E2020202020202052756E20AE
:1047000073656C662D74657374204E0A20202468CE
:104710006F6D653D312020202020202052756E20B5
:104720006120686F6D696E67206379636C650A202C
:104730002024646566613D31202020202020205205
:104740006573746F726520616C6C20736574746935
:104750006E677320746F2022666163746F727922B2
:104760002064656661756C74730A000A0A0A232363
:10477000232054696E79472048656C7020232323D9
:104780000A0022007B2272223A7B22747874223A39
:1047900022007B723A7B7478743A22005B6A735D04
:1047A00020206A736F6E2073657269616C697A6527
:1047B000207374796C65253964205B303D72656CBB
:1047C000617865642C313D7374726963745D0A00AD
:1047D0005B6A765D20206A736F6E20766572626F09
:1047E0007369747925313564205B303D73696C657C
:1047F0006E742C313D666F6F7465722C323D6D6541
:104800007373616765732C333D636F6E666967739D
:104810002C343D6C696E656E756D2C353D76657218
:10482000626F73655D0A005B656A5D2020656E617D
:10483000626C65206A736F6E206D6F64652531331D
:1048400064205B303D746578742C313D4A534F4E83
:104850005D0A00AF59A959A2599D59945989597EA9
:1048600059725966594A593359245917590B59F7EE
:1048700058EA58D558C158BE58BB58AC58975882BA
:10488000587358635851583A581D580058E757D133
:1048900057C057AE57A1578F57755772576F576C00
:1048A0005769576657635760575D575A575757545C
:1048B0005751574E574B574857455742573F573C0C
:1048C0005739573657335730572D572A57275724BC
:1048D0005721571E571B571857155712570F570C6C
:1048E000570957065703570057FD56FA56F756F41F
:1048F00056F156EE56EB56E856E556E256DF56DCD4
:1049000056D956D656AF568B566B56515637561DFE
:1049100056F955DC55C455AE55945570555355410F
:104920005521550A55F154CF54B65498547C5464CB
:1049300054525434541F54FE53FA53F653F253EE68
:1049400053EA53E653E253DE53DA53D653D253CEEF
:1049500053CA53C653C253A8538E537B535F534D10
:1049600053365315530453E452C452AA5290527909
:104970005246521952F951D751B1518A516E514F85
:104980005135511B51F650CD50B5508A505E5028CC
:1049900050F34FE14FCF4FC04FAD4F944F724F6028
:1049A0004F4E4F3C4F2A4F184F064FF44EE24ED019
:1049B0004EBE4EAC4E9A4E884E764E724E6E4E6A3B
:1049C0004E664E624E5E4E5A4E564E524E4E4E4AB7
:1049D0004E464E424E3E4E3A4E364E324E2E4E2AA7
:1049E0004E264E124EF44DD84DAD4D884D634D5F61
:1049F0004D5B4D574D534D4F4D4B4D474D434D3FE7
:104A00004D3B4D374D334D2F4D2B4D174DFB4CDF4F
:104A10004CC34CA74C8B4C6F4C534C374C1B4CFF2E
:104A20004BE34BC74BC34BBF4BBB4BB74BB34BAF2E
:104A30004BAB4B974B6F4B484B224BF54ACF4AA29F
:104A40004A9E4A9A4A964A834A624A4D4A4A6F6740
:104A500067696E67206379636C65206661696C6560
:104A6000640050726F626520656E64706F696E7469
:104A7000206973207374617274696E6720706F6946
:104A80006E740050726F6265206379636C65206696
:104A900061696C6564003234390032343800323474
:104AA0003700486F6D696E67204572726F72202DF6
:104AB00020486F6D696E67207377697463686573EA
:104AC000206D6973636F6E6669677572656400480F
:104AD0006F6D696E67204572726F72202D204E6572
:104AE000676174697665206C6174636820626163D4
:104AF0006B6F666600486F6D696E67204572726FF6
:104B000072202D2054726176656C206D696E2026AE
:104B1000206D617820617265207468652073616D15
:104B20006500486F6D696E67204572726F72202D47
:104B3000204C617463682076656C6F6369747920BA
:104B40006973207A65726F00486F6D696E672045E2
:104B500072726F72202D20536561726368207665D2
:104B60006C6F63697479206973207A65726F00488D
:104B70006F6D696E67204572726F72202D204261E1
:104B800064206F72206E6F20617869732073706586
:104B900063696669656400486F6D696E6720637953
:104BA000636C65206661696C65640032333900327C
:104BB0003338003233370032333600323335003287
:104BC00033340032333300536F6674206C696D697F
:104BD00074206578636565646564202D2043206DCD
:104BE000617800536F6674206C696D697420657814
:104BF000636565646564202D2043206D696E0053F4
:104C00006F6674206C696D6974206578636565648E
:104C10006564202D2042206D617800536F667420FA
:104C20006C696D6974206578636565646564202DC1
:104C30002042206D696E00536F6674206C696D6947
:104C400074206578636565646564202D2041206D5E
:104C5000617800536F6674206C696D6974206578A3
:104C6000636565646564202D2041206D696E005385
:104C70006F6674206C696D6974206578636565641E
:104C80006564202D205A206D617800536F66742072
:104C90006C696D6974206578636565646564202D51
:104CA000205A206D696E00536F6674206C696D69BF
:104CB00074206578636565646564202D2059206DD6
:104CC000617800536F6674206C696D697420657833
:104CD000636565646564202D2059206D696E0053FD
:104CE0006F6674206C696D697420657863656564AE
:104CF0006564202D2058206D617800536F66742004
:104D00006C696D6974206578636565646564202DE0
:104D10002058206D696E00536F6674206C696D6950
:104D200074206578636565646564003231390032EA
:104D3000313800323137003231360032313500320D
:104D4000313400323133003231320032313100320D
:104D500031300032303900323038003230370032F2
:104D600030360054726170657A6F696420706C61CE
:104D70006E6E6572206661696C656420746F206375
:104D80006F6E7665726765004C696D697420737724
:104D90006974636820686974202D20536875746491
:104DA0006F776E206F63637572726564004D616327
:104DB00068696E6520697320616C61726D6564203D
:104DC0002D20436F6D6D616E64206E6F7420707264
:104DD0006F636573736564004D6F7665206C6573F2
:104DE00073207468616E206D696E696D756D2074D5
:104DF000696D65004D6F7665206C6573732074680E
:104E0000616E206D696E696D756D206C656E67747D
:104E1000680047656E657269632054696E79472042
:104E20006572726F720031393900313938003139A9
:104E300037003139360031393500313934003139F4
:104E400033003139320031393100313930003138F5
:104E500039003138380031383700313836003138D0
:104E600035003138340031383300313832003138D0
:104E70003100313830005420776F7264206973201C
:104E8000696E76616C6964005420776F7264206982
:104E900073206D697373696E67005220776F726457
:104EA00020697320696E76616C6964005220776FA7
:104EB0007264206973206D697373696E6700512095
:104EC000776F726420697320696E76616C69640023
:104ED0005120776F7264206973206D697373696EF6
:104EE00067004C20776F726420697320696E766169
:104EF0006C6964004C20776F7264206973206D695F
:104F00007373696E67004820776F7264206973203D
:104F1000696E76616C6964004820776F72642069FD
:104F200073206D697373696E67004520776F7264D3
:104F300020697320696E76616C6964004520776F23
:104F40007264206973206D697373696E6700442011
:104F5000776F726420697320696E76616C69640092
:104F60004420776F7264206973206D697373696E72
:104F700067005020776F7264206973206E6F742011
:104F8000612076616C696420746F6F6C206E756D42
:104F9000626572005020776F7264206973206E6FB3
:104FA0007420616E20696E746567657200502077A9
:104FB0006F7264206973206E65676174697665003D
:104FC0005020776F7264206973207A65726F005089
:104FD00020776F726420697320696E76616C6964F2
:104FE000005020776F7264206973206D6973736954
:104FF0006E670041726320737065636966696361FF
:1050000074696F6E206572726F72202D20656E64F8
:10501000706F696E74206973207374617274696E45
:105020006720706F696E74004172632073706563EE
:10503000696669636174696F6E206572726F722050
:105040002D2072616469757320617263206F7574BD
:10505000206F6620746F6C6572616E6365004172CB
:10506000632073706563696669636174696F6E203C
:105070006572726F72202D206D697373696E67207F
:105080006F666673657428732900417263207370BC
:105090006563696669636174696F6E206572726FBA
:1050A00072202D206D697373696E67206178697352
:1050B00028657329004172632073706563696669AE
:1050C000636174696F6E206572726F7200537069EC
:1050D0006E646C65206D75737420626520747572E2
:1050E0006E696E6720666F72207468697320636FE3
:1050F0006D6D616E64005370696E646C65206D75D2
:105100007374206265206F666620666F7220746813
:10511000697320636F6D6D616E64005370696E64B6
:105120006C65205320776F726420697320696E76F6
:10513000616C6964005370696E646C6520532077FC
:105140006F7264206973206D697373696E670053B1
:1051500070696E646C652073706565642065786342
:105160006565646564206D6178696D756D00537067
:10517000696E646C652073706565642062656C6F30
:1051800077206D696E696D756D0050726F67726121
:105190006D6D656420706F696E742073616D65203C
:1051A00061732063757272656E7420706F696E74BE
:1051B0000043757474657220636F6D70656E736102
:1051C00074696F6E2063616E6E6F74206265206516
:1051D0006E61626C656400526571756573746564B7
:1051E0002076656C6F6369747920657863656564A2
:1051F00073206C696D697473004730206F722047AB
:1052000031206D7573742062652061637469766501
:1052100020666F722047353300526F7461727920B7
:10522000617865732063616E6E6F742062652075AE
:105230007365642077697468207468697320636F8C
:105240006D6D616E6400496E766572736520746978
:105250006D65206D6F64652063616E6E6F74206292
:105260006520757365642077697468207468697354
:1052700020636F6D6D616E64004665656472617474
:1052800065206E6F7420737065636966696564007C
:1052900053656C656374656420706C616E6520692C
:1052A0007320696E76616C69640053656C65637424
:1052B000656420706C616E65206973206D6973731D
:1052C000696E670041786973207461726765742044
:1052D000706F736974696F6E20697320696E76618F
:1052E0006C69640041786973207461726765742029
:1052F000706F736974696F6E206973206D69737361
:10530000696E67004178697320697320646973610D
:10531000626C6564004178697320697320696E76F8
:10532000616C696420666F72207468697320636FB2
:105330006D6D616E6400417869732063616E6E6F9C
:10534000742062652070726573656E7400417869BF
:105350007320776F7264206D697373696E6700479D
:10536000636F6465206D6F64616C2067726F757028
:105370002076696F6C6174696F6E004D20636F6495
:105380006520756E737570706F7274656400476325
:105390006F646520636F6D6D616E6420756E7375EB
:1053A00070706F727465640047656E657269632022
:1053B00047636F646520696E707574206572726FE3
:1053C0007200313239003132380031323700313237
:1053D000360031323500313234003132330031326F
:1053E0003200313231003132300031313900313167
:1053F00038003131370031313600313135004A5310
:105400004F4E20747874206669656C647320636104
:105410006E6E6F74206265206E6573746564004AF9
:10542000534F4E20737472696E6720746F6F206CD7
:105430006F6E67004A534F4E20696E707574206816
:10544000617320746F6F206D616E79207061697275
:1054500073004A534F4E2073796E746178206572E1
:10546000726F7200496E7075742076616C7565207C
:1054700072616E6765206572726F7200496E707539
:10548000742065786365656473206D6178696D75F6
:105490006D2076616C756500496E707574206C6561
:1054A0007373207468616E206D696E696D756D200F
:1054B00076616C756500496E7075742065786365FA
:1054C000656473206D6178206C656E677468004355
:1054D0006F6D6D616E64206E6F74206163636570C3
:1054E00074656420617420746869732074696D65E3
:1054F00000506172616D657465722063616E6E6FDC
:1055000074206265207265616400506172616D652E
:1055100074657220697320726561642D6F6E6C7999
:1055200000556E737570706F72746564206E756D62
:10553000626572206F72204A534F4E2074797065F5
:1055400000426164206E756D62657220666F726DD7
:10555000617400496E76616C6964206F72206D61C0
:105560006C666F726D656420636F6D6D616E640053
:10557000556E7265636F676E697A656420636F6DDF
:105580006D616E64206F7220636F6E666967206E56
:10559000616D650047656E6572696320617373654F
:1055A0007274696F6E206661696C757265004D6515
:1055B0006D6F7279206661756C74206465746563C3
:1055C00074656400537461636B206F766572666CFA
:1055D0006F7720646574656374656400436F6E74EF
:1055E000726F6C6C657220617373657274696F6E33
:1055F000206661696C7572650043616E6F6E6963E8
:10560000616C206D616368696E652061737365729A
:1056100074696F6E206661696C75726500506C61AB
:105620006E6E657220617373657274696F6E206649
:1056300061696C7572650053746570706572206184
:105640007373657274696F6E206661696C757265DB
:1056500000456E636F64657220617373657274696F
:105660006F6E206661696C75726500494F207375B5
:10567000622D73797374656D2061737365727469DB
:105680006F6E206661696C75726500436F6E666946
:1056900067207375622D73797374656D2061737300
:1056A000657274696F6E206661696C757265004918
:1056B0004F206D656D6F727920616C6C6F636174E2
:1056C000696F6E20617373657274696F6E206661B5
:1056D000696C757265003838003837003836003824
:1056E0003500383400383300383200383100383073
:1056F0000037390037380037370037360037350084
:105700003734003733003732003731003730003656
:105710003900363800363700363600363500363434
:10572000003633003632003631003630003539006D
:10573000353800353700353600353500353400351D
:10574000330035320035310035300034390034381B
:10575000003437003436003435003434003433003C
:105760003432003431003430003339003338003300
:10577000370033360042616420737461747573209E
:105780007265706F72742073657474696E6700500F
:10579000657273697374656E6365206572726F728A
:1057A00000466C6F6174206973204E414E00466C58
:1057B0006F617420697320696E66696E6974650033
:1057C0004D6F76652074696D65206973204E414E7A
:1057D000004D6F76652074696D6520697320696E70
:1057E00066696E6974650047656E657269632065F8
:1057F0007863657074696F6E207265706F72740083
:105800004661696C656420746F2067657420706CF4
:10581000616E6E657220627566666572005379739B
:1058200074656D20616C61726D202D2073687574D4
:1058300074696E6720646F776E00496E6974696180
:105840006C697A6174696F6E206661696C757265E6
:1058500000526561642D6F6E6C79206164647265BD
:10586000737300496E76616C69642041646472658B
:10587000737300446976696465206279207A657281
:105880006F00466C6F6174696E6720706F696E742B
:10589000206572726F7200496E7465726E616C2061
:1058A00072616E6765206572726F7200496E746511
:1058B000726E616C206572726F720031390031381E
:1058C0000046756E6374696F6E206973207374751A
:1058D0006262656400456E746572696E6720626F0E
:1058E0006F74206C6F6164657200496E69746961E0
:1058F0006C697A696E6700427566666572206675C6
:105900006C6C202D20666174616C00427566666562
:10591000722066756C6C0042756666657220656DF6
:10592000707479004E6F20737563682064657669C2
:105930006365004D61782066696C652073697A65DE
:105940002065786365656465640043616E6E6F749D
:1059500020777269746520746F2064657374696E52
:105960006174696F6E00456E64206F662066696CB5
:105970006500456E64206F66206C696E6500486145
:105980007264207265736574005465726D696E612E
:1059900074656400436F6D706C657465004E6F6F65
:1059A000700045616761696E004572726F72004FE9
:1059B0004B005B7031706F665D2070776D20706892
:1059C000617365206F66662020202531352E336691
:1059D000205B302E2E315D0A005B70317770685D80
:1059E0002070776D2063637720706861736520682D
:1059F000692531352E3366205B302E2E315D0A004D
:105A00005B703177706C5D2070776D2063637720F9
:105A10007068617365206C6F2531352E3366205BAD
:105A2000302E2E315D0A005B70317773685D207017
:105A3000776D2063637720737065656420686925DE
:105A400031352E30662052504D0A005B703177732D
:105A50006C5D2070776D206363772073706565647B
:105A6000206C6F2531352E30662052504D0A005B78
:105A700070316370685D2070776D20637720706887
:105A8000617365206869202531352E3366205B30CF
:105A90002E2E315D0A005B703163706C5D20707773
:105AA0006D206377207068617365206C6F202531ED
:105AB000352E3366205B302E2E315D0A005B70314F
:105AC0006373685D2070776D206377207370656500
:105AD00064206869202531352E30662052504D0AE9
:105AE000005B703163736C5D2070776D206377208D
:105AF0007370656564206C6F202531352E3066200B
:105B000052504D0A005B70316672715D2070776D86
:105B1000206672657175656E6379202020253135A8
:105B20002E306620487A0A0053595354454D20526E
:105B300045414459004C6F6164696E6720636F6E24
:105B4000666967732066726F6D20454550524F4DF0
:105B500000496E697469616C697A696E6720636F68
:105B60006E6669677320746F2053686170656F6B30
:105B70006F32203530306D6D2070726F66696C65E4
:105B8000007B226572223A7B226662223A25302E01
:105B900032662C227374223A25642C226D7367229C
:105BA0003A222573227D7D0A007B65723A7B66620C
:105BB0003A25302E32662C73743A25642C6D736747
:105BC0003A222573227D7D0A005B71765D2020716B
:105BD00075657565207265706F7274207665726286
:105BE0006F73697479253764205B303D6F66662C6E
:105BF000313D73696E676C652C323D747269706CEF
:105C0000655D0A00716F3A25640A0071693A25647E
:105C10000A0071723A25640A005B73765D20207376
:105C20007461747573207265706F7274207665721A
:105C3000626F73697479253664205B303D6F6666E8
:105C40002C313D66696C74657265642C323D7665F5
:105C500072626F73655D0A005B73695D2020737407
:105C60006174757320696E74657276616C25313468
:105C70006C75206D730A004D6F746F722025632060
:105C8000706F77657220656E61626C6564207374F5
:105C90006174653A25322E30660A005B25732573E0
:105CA0005D206D257320706F776572206D616E6168
:105CB00067656D656E7425313064205B303D6469C5
:105CC0007361626C65642C313D616C77617973201E
:105CD0006F6E2C323D696E206379636C652C333DA9
:105CE0007768656E206D6F76696E675D0A005B256B
:105CF0007325735D206D257320706F6C61726974FC
:105D00007925313864205B303D6E6F726D616C2C8B
:105D1000313D726576657273655D0A005B2573259A
:105D2000735D206D2573206D6963726F7374657088
:105D30007325313664205B312C322C342C385D0ACB
:105D4000005B257325735D206D2573207472617669
:105D5000656C20706572207265766F6C7574696F02
:105D60006E2531302E346625730A005B257325734A
:105D70005D206D2573207374657020616E676C659E
:105D80002532302E336625730A005B257325735D3B
:105D9000206D2573206D617020746F2061786973A8
:105DA00025313564205B303D582C313D592C323D36
:105DB0005A2E2E2E5D0A005B6D745D20206D6F746F
:105DC0006F722069646C652074696D656F757425E8
:105DD00031342E3266205365630A00EA5DE65DE1E8
:105DE0005D2064656700206D6D0020696E005B7347
:105DF000745D2020737769746368207479706525F9
:105E0000313864205B303D4E4F2C313D4E435D0AAE
:105E1000005465737420232564206E6F7420666FB0
:105E2000756E640A004E312054314D360A4E3220D0
:105E30004731370A4E33204732310A4E3820463137
:105E40003830300A4E392047310A4E313030204741
:105E5000393220582D32352E313737592D33342EE3
:105E6000303732205A2D312E303030202854454DD5
:105E7000502C2052454D4F5645204C4154455229F7
:105E80000A4E33343320582D32352E353935592DBD
:105E900033342E3334390A4E33343420582D3235CE
:105EA0002E373031592D33342E3433360A4E3334B5
:105EB0003520582D32352E373931592D33342E3582
:105EC00032300A4E33343620582D32352E3836349F
:105ED000592D33342E3630310A4E33343720582D75
:105EE00032352E393230592D33342E3637390A4E69
:105EF00033343820582D32352E393630592D33343D
:105F00002E3735340A4E33343920582D32352E3958
:105F10003832592D33342E3832360A4E333530204C
:105F2000582D32352E393837592D33342E383935EE
:105F30000A4E33353120582D32352E393736592D0A
:105F400033342E3936310A4E33353220582D32351E
:105F50002E393438592D33352E3032330A4E3335FD
:105F60003320582D32352E393033592D33352E30DC
:105F700038320A4E33353420582D32352E383431EC
:105F8000592D33352E3133380A4E33353520582DBF
:105F900032352E373633592D33352E3139300A4EBE
:105FA00033353620582D32352E363639592D333586
:105FB0002E3233390A4E33353720582D32352E35AF
:105FC0003539592D33352E3238340A4E3335382091
:105FD000582D32352E343333592D33352E33323557
:105FE0000A4E33353920582D32352E323931592D5C
:105FF00033352E3336330A4E33363020582D323572
:106000002E313334592D33352E3339370A4E33364A
:106010003120582D32342E393633592D33352E3424
:1060200032380A4E33363220582D32342E37373735
:10603000592D33352E3435350A4E33363320582D0D
:1060400032342E353737592D33352E3437370A4E03
:1060500033363420582D32342E333637592D3335DC
:106060002E3439360A4E33363520582D32342E31FF
:106070003434592D33352E3531310A4E33363620EE
:10608000582D32332E393039592D33352E353232A1
:106090000A4E33363720582D32332E363631592DAD
:1060A00033352E3532390A4E33363820582D3233B7
:1060B0002E343033592D33352E3533320A4E3336A4
:1060C0003920582D32332E313333592D33352E3577
:1060D00033320A4E33373020582D32322E38353392
:1060E000592D33352E3532370A2F4E32353138207F
:1060F000473058302E333237592D33332E35323125
:106100005A2D312E3030300A4E32353139204D3350
:1061100030004E31204732300A4E3520473430208F
:106120004731370A4E3130205431204D30360A285D
:106130004E313520473930204730205830205930F3
:10614000205A30290A4E3230205335303030204D1D
:106150003033200A4E32352058302E303634205914
:10616000302E333236205A300A4E34302047303108
:10617000204631362E300A4E35302058302E3036FB
:10618000342059302E3332360A4E35352058302ED1
:106190003036302059302E3239330A4E36302058BE
:1061A000302E3037372059302E3236370A4E3635BA
:1061B0002058302E3131312059302E3235370A4EA9
:1061C00037302058302E3134392059302E32353284
:1061D0000A4E37352058302E3138382059302E327B
:1061E00035350A4E38302058302E3232372059306B
:1061F0002E3236380A4E38352058302E3235372078
:1062000059302E3237310A4E39302058302E333340
:10621000352059302E3236350A4E39352058302E39
:106220003431322059302E3237310A4E313030205D
:1062300058302E3437342059302E3238370A4E3108
:1062400030352058302E3439312059302E323839FB
:106250000A4E3131302058302E3531372059302E0A
:106260003237330A4E3131352058302E3534342010
:1062700059302E3236330A4E3132302058302E35D6
:1062800038302059302E3236310A4E3132352058CE
:10629000302E3539352059302E3236330A4E3133CF
:1062A000302058302E3632312059302E3237340AD1
:1062B0004E3133352058302E3635392059302E3373
:1062C00030360A4E3134302058302E36373320598C
:1062D000302E3333350A4E3134352058302E363790
:1062E000392059302E3336310A4E3135302058306E
:1062F0002E3637382059302E3338390A4E3135355D
:106300002058302E3637302059302E3432300A4E55
:106310003136302058302E3637302059302E343434
:10632000360A4E3136352058302E36383020593026
:106330002E3437340A4E3137302058302E3730342F
:106340002059302E3439370A4E3137352058302E07
:106350003733322059302E3531350A4E313830201E
:1063600058302E3739342059302E3533350A4E31D6
:1063700038352058302E3837322059302E353637C0
:106380000A4E3139302058302E3935302059302ED0
:106390003630340A4E3139352058312E30333120E1
:1063A00059302E3634370A4E3230302058312E31A3
:1063B00034392059302E3732320A4E323035205897
:1063C000312E3330382059302E3835340A4E3231A0
:1063D000302058312E3433302059302E3938340A99
:1063E0004E3231352058312E3434372059302E3941
:1063F00038360A4E3232302058312E363238205953
:10640000302E3832320A4E3232352058312E373360
:10641000322059302E3731340A4E32333020583240
:106420002E3030392059302E3338310A4E32333540
:106430002058322E3131362059302E3236360A4E1F
:106440003234302058322E3232382059302E313505
:10645000370A4E3234352058322E323830205930F7
:106460002E3132330A4E3235302058322E33333209
:106470002059302E3039340A4E3235352058322EDC
:106480003432332059302E3037300A4E32363020F5
:1064900058322E3438392059302E3036350A4E32A3
:1064A00036352058322E3535372059302E30363695
:1064B0000A4E3237302058322E3632372059302E9D
:1064C0003038340A4E3237352058322E36393320A0
:1064D00059302E3130390A4E3238302058322E376A
:1064E00033302059302E3133330A4E32383520586C
:1064F000322E3830352059302E3139300A4E32396B
:10650000302058322E3832392059302E3231360A66
:106510004E3239352058322E3838302059302E320C
:1065200039310A4E3330302058322E383834205921
:10653000302E3330300A4E3330352058322E383931
:10654000382059302E3333320A4E3331302058320E
:106550002E3930352059302E3336370A4E33313507
:106560002058322E3931302059302E3430370A4EEF
:106570003332302058322E3930382059302E3434CE
:10658000360A4E3332352058322E393031205930C8
:106590002E3439350A4E3333302058322E383937BD
:1065A0002059302E3439350A4E3333352058322EA7
:1065B0003839302059302E3532340A4E33343020B9
:1065C00058322E3834322059302E3630340A4E3379
:1065D00034352058322E3831342059302E36363565
:1065E0000A4E3335302058322E3739342059302E68
:1065F0003735300A4E3335352058322E3739312071
:1066000059302E3833380A4E3336302058322E382F
:1066100031392059302E3937360A4E333635205825
:10662000322E3833372059312E3034340A4E333736
:10663000302058322E3836322059312E3131320A3C
:106640004E3337352058322E3837372059312E31D6
:1066500034350A4E3338302058322E3931322059F1
:10666000312E3231370A4E3338352058322E3931F7
:10667000372059312E3232360A4E333930205832D3
:106680002E3935312059312E3238310A4E333935D1
:106690002058322E3937302059312E3239350A4EB2
:1066A0003430302058322E3939362059312E323993
:1066B000350A4E3430352058332E3031332059319D
:1066C0002E3237350A4E3431302058332E303234A2
:1066D0002059312E3235340A4E3431352058332E7C
:1066E0003037302059312E3135310A4E3432302096
:1066F00058332E3037372059312E3133340A4E3447
:1067000032352058332E3132352059312E3033393D
:106710000A4E3433302058332E3133382059312E3D
:106720003031390A4E3433352058332E323035204B
:1067300059302E3930380A4E3434302058332E3206
:1067400038322059302E3739370A4E3434352058F4
:10675000332E3336312059302E3639310A4E343506
:10676000302058332E3432362059302E3539320A03
:106770004E3435352058332E3435362059302E35A9
:1067800034330A4E3436302058332E3437392059BA
:10679000302E3439330A4E3436352058332E3439BE
:1067A000342059302E3437320A4E343730205833A3
:1067B0002E3530352059302E3434360A4E343735A4
:1067C0002058332E3531382059302E3431370A4E87
:1067D0003438302058332E3533302059302E333969
:1067E000310A4E3438352058332E3536342059305E
:1067F0002E3330300A4E3439302058332E35373767
:106800002059302E3235330A4E3439352058332E44
:106810003536382059302E3231320A4E353030205C
:1068200058332E3534342059302E3137360A4E3510
:1068300030352058332E3534312059302E3134360E
:106840000A4E3531302058332E3535332059302E0D
:106850003131390A4E3531352058332E353736200F
:1068600059302E3130360A4E3532302058332E35DD
:1068700039372059302E3130320A4E3532352058D2
:10688000332E3631382059302E3130390A4E3533D7
:10689000302058332E3633392059302E3132390AD0
:1068A0004E3533352058332E3635302059302E3181
:1068B00035390A4E3534302058332E363633205988
:1068C000302E3137380A4E3534352058332E36378E
:1068D000382059302E3139320A4E35353020583370
:1068E0002E3639392059302E3139370A4E35353563
:1068F0002058332E3732332059302E3139360A4E54
:106900003536302058332E3736342059302E313733
:10691000390A4E3536352058332E38303520593027
:106920002E3136350A4E3537302058332E3838342C
:106930002059302E3135390A4E3537352058332E0F
:106940003934392059302E3136350A4E3538302019
:1069500058332E3936362059302E3137350A4E35D8
:1069600038352058332E3937382059302E313934C4
:106970000A4E3539302058332E3937382059302EC9
:106980003232330A4E3539352058332E39363020DD
:1069900059302E3234350A4E3630302058332E38A6
:1069A00033342059302E3331310A4E3630352058A9
:1069B000332E3736322059302E3334350A4E3631A5
:1069C000302058332E3732362059302E3338390A9A
:1069D0004E3631352058332E3730332059302E344F
:1069E00035380A4E3632302058332E363832205958
:1069F000302E3533300A4E3632352058332E363766
:106A0000392059302E3533340A4E3633302058333E
:106A10002E3632362059302E3638310A4E3633353E
:106A20002058332E3536382059302E3832380A4E19
:106A30003634302058332E3434342059312E303807
:106A4000300A4E3634352058332E34303520593103
:106A50002E3136370A4E3635302058332E34303406
:106A60002059312E3136370A4E3635352058332EDF
:106A70003338372059312E3230380A4E36363020EE
:106A800058332E3338342059312E3230380A4E36AE
:106A900036352058332E3336352059312E3236359F
:106AA0000A4E3637302058332E3335352059312EA3
:106AB0003238350A4E3637352058332E33343820A5
:106AC00059312E3330380A4E3638302058332E3371
:106AD00033332059312E3335300A4E36383520586D
:106AE000332E3332312059312E3339310A4E363973
:106AF000302058332E3331312059312E3432380A78
:106B00004E3639352058332E3333392059312E340F
:106B100032330A4E3730302058332E343430205937
:106B2000312E3430360A4E3730352058332E353139
:106B3000302059312E3430380A4E37313020583316
:106B40002E3538352059312E3432310A4E37313511
:106B50002058332E3631312059312E3433390A4EF4
:106B60003732302058332E3631312059312E3434DB
:106B7000310A4E3732352058332E363135205931CF
:106B80002E3434310A4E3733302058332E363336D4
:106B90002059312E3438380A4E3733352058332EA9
:106BA0003633342059312E3531370A4E37343020C0
:106BB00058332E3632322059312E3534330A4E377F
:106BC00034352058332E3630352059312E35363372
:106BD0000A4E3735302058332E3537362059312E6E
:106BE0003537350A4E3735352058332E3534342075
:106BF00059312E3538310A4E3736302058332E343D
:106C000037392059312E3539320A4E37363520582A
:106C1000332E3435312059312E3539380A4E373735
:106C2000302058332E3338372059312E3632360A39
:106C30004E3737352058332E3339302059312E36E0
:106C400033360A4E3738302058332E3533322059F8
:106C5000312E3630320A4E3738352058332E363002
:106C6000312059312E3539370A4E373930205833D3
:106C70002E3636382059312E3539380A4E373935C7
:106C80002058332E3738322059312E3631320A4EC1
:106C90003830302058332E3739342059312E3631A0
:106CA000380A4E3830352058332E3836382059318E
:106CB0002E3633360A4E3831302058332E3931389B
:106CC0002059312E3635350A4E3831352058332E7D
:106CD0003934352059312E3636370A4E3832302085
:106CE00058332E3936342059312E3638350A4E383D
:106CF00032352058332E3936372059312E36383533
:106D00000A4E3833302058332E3937342059312E3B
:106D10003639390A4E3833352058332E3938342035
:106D200059312E3732350A4E3834302058332E3907
:106D300038342059312E3735380A4E3834352058FA
:106D4000332E3937302059312E3739300A4E383505
:106D5000302058332E3934352059312E3831370A06
:106D60004E3835352058332E3931382059312E38A8
:106D700032360A4E3836302058332E3839312059C1
:106D8000312E3832370A4E3836352058332E3834C3
:106D9000322059312E3830390A4E383730205833A6
:106DA0002E3739382059312E3738340A4E38373596
:106DB0002058332E3734362059312E3737320A4E89
:106DC0003838302058332E3639382059312E37365E
:106DD000340A4E3838352058332E36333520593161
:106DE0002E3736360A4E3839302058332E35353363
:106DF0002059312E3738350A4E3839352058332E40
:106E00003437382059312E3832300A4E393030205C
:106E100058332E3430392059312E3836340A4E3911
:106E200030352058332E3334352059312E3931380E
:106E30000A4E3931302058332E3236342059322E12
:106E40003032330A4E3931352058332E323438201F
:106E500059322E3035310A4E3932302058332E32E5
:106E600034302059322E3038310A4E3932352058DC
:106E7000332E3331362059322E3038360A4E3933DC
:106E8000302058332E3339302059322E3130340AE5
:106E90004E3933352058332E3431342059322E3187
:106EA00032310A4E3934302058332E3433312059A0
:106EB000322E3135330A4E3934352058332E34339F
:106EC000332059322E3138300A4E3935302058337C
:106ED0002E3432372059322E3230350A4E3935357C
:106EE0002058332E3431332059322E3232340A4E68
:106EF0003936302058332E3339322059322E32343D
:106F0000320A4E3936352058332E33333520593234
:106F10002E3234340A4E3937302058332E32373837
:106F20002059322E3233360A4E3937352058332E17
:106F30003235362059322E3234320A4E393830202A
:106F400058332E3233392059322E3235310A4E39E8
:106F500038352058332E3231312059322E323830E4
:106F60000A4E3939302058332E3137342059322ED9
:106F70003335360A4E3939352058332E31353920DC
:106F800059322E3339370A4E313030302058332EB3
:106F90003135302059322E3433380A4E31303035C5
:106FA0002058332E3134302059322E3438310A4EA5
:106FB000313031302058332E3133322059322E3592
:106FC00031300A4E313031352058332E31313820AE
:106FD00059322E3534330A4E313032302058332E68
:106FE0003039392059322E3537360A4E3130323564
:106FF0002058332E3035312059322E3633310A4E57
:10700000313033302058332E3030332059322E3641
:1070100036360A4E313033352058322E3935372046
:1070200059322E3638350A4E313034302058322E0F
:107030003930372059322E3639390A4E313034350D
:107040002058322E3836302059322E3731310A4E00
:10705000313035302058322E3831392059322E37E0
:1070600032370A4E313035352058322E37363820F7
:1070700059322E3734350A4E313036302058322EC0
:107080003731362059322E3735370A4E31303635C2
:107090002058322E3637352059322E3735370A4EA2
:1070A000313037302058322E3537392059322E378B
:1070B00033310A4E313037352058322E35373020B3
:1070C00059322E3732330A4E313038302058322E72
:1070D0003535392059322E3732300A4E3130383575
:1070E0002058322E3533302059322E3730310A4E67
:1070F000313039302058322E3530312059322E3649
:1071000039330A4E313039352058322E3437312058
:1071100059322E3638330A4E313130302058322E23
:107120003434332059322E3636380A4E3131303528
:107130002058322E3339362059322E3633340A4E07
:10714000313131302058322E3335342059322E35FA
:1071500039310A4E313131352058322E3335322013
:1071600059322E3539310A4E313132302058322ED3
:107170003332352059322E3534330A4E31313235DF
:107180002058322E3331352059322E3532310A4EC5
:10719000313133302058322E3330372059322E34AB
:1071A00039380A4E313133352058322E32393620B3
:1071B00059322E3436340A4E313134302058322E82
:1071C0003239332059322E3432370A4E3131343588
:1071D0002058322E3239352059322E3336360A4E67
:1071E000313135302058322E3332312059322E335E
:1071F00030330A4E313135352058322E3335382070
:1072000059322E3234370A4E313136302058322E30
:107210003431392059322E3230330A4E313136353D
:107220002058322E3431392059322E3137390A4E16
:10723000313137302058322E3430352059322E310A
:1072400035380A4E313137352058322E3336322018
:1072500059322E3132330A4E313138302058322EE5
:107260003335342059322E3130340A4E31313835ED
:107270002058322E3335342059322E3039310A4ECF
:10728000313139302058322E3338302059322E30B7
:1072900036350A4E313139352058322E34313020CE
:1072A00059322E3035310A4E313230302058322E9C
:1072B0003431302059322E3034370A4E31323035A5
:1072C0002058322E3430352059322E3032380A4E82
:1072D000313231302058322E3430382059322E306D
:1072E00031300A4E313231352058322E3431362089
:1072F00059312E3939350A4E313232302058322E3A
:107300003433332059312E3938320A4E3132323546
:107310002058322E3433382059312E3936330A4E24
:10732000313233302058322E3434372059312E390F
:1073300034380A4E313233352058322E343631202B
:1073400059312E3933380A4E313234302058322EEA
:107350003438302059312E3933310A4E31323435F8
:107360002058322E3437382059312E3839390A4EC8
:10737000313235302058322E3438372059312E38BA
:1073800037350A4E313235352058322E35303420DB
:1073900059312E3835340A4E313236302058322E9B
:1073A0003532372059312E3834380A4E313236359D
:1073B0002058322E3534392059312E3834390A4E7E
:1073C000313237302058322E3537372059312E3868
:1073D00036310A4E313237352058322E363034208D
:1073E00059312E3836360A4E313238302058322E46
:1073F0003633312059312E3835340A4E3132383552
:107400002058322E3634302059312E3832370A4E39
:10741000313239302058322E3634302059312E371F
:1074200039320A4E313239352058322E363239202F
:1074300059312E3735390A4E313330302058322EFB
:107440003631322059312E3732370A4E313330350A
:107450002058322E3537362059312E3639340A4EDF
:10746000313331302058322E3533362059312E36D3
:1074700036320A4E313331352058322E34373020EF
:1074800059312E3631360A4E313332302058322EB1
:107490003334352059312E3535310A4E31333235BA
:1074A0002058322E3330372059312E3532310A4EA2
:1074B000313333302058322E3236302059312E3489
:1074C00038320A4E313333352058322E323433209D
:1074D00059312E3437370A4E313334302058322E5A
:1074E0003232382059312E3436390A4E3133343560
:1074F0002058322E3232322059312E3434380A4E4E
:10750000313335302058322E3232382059312E3432
:1075100032350A4E313335352058322E323534204B
:1075200059312E3430350A4E313336302058322E10
:107530003236382059312E3337330A4E313336350F
:107540002058322E3237392059312E3334320A4EF8
:10755000313337302058322E3330382059312E32E3
:1075600038370A4E313337352058322E33343020F5
:1075700059312E3235340A4E313338302058322EBC
:107580003430372059312E3230310A4E31333835CC
:107590002058322E3434312059312E3135360A4EAE
:1075A000313339302058322E3435342059312E3190
:1075B00033310A4E313339352058322E34363020AB
:1075C00059312E3130360A4E313430302058322E77
:1075D0003436342059312E3130320A4E3134303580
:1075E0002058322E3437312059312E3033360A4E5E
:1075F000313431302058322E3436362059302E393D
:1076000037310A4E313431352058322E343531205D
:1076100059302E3839370A4E313432302058322E14
:107620003431352059302E3739310A4E3134323524
:107630002058322E3430332059302E3736370A4E08
:10764000313433302058322E3338382059302E37E9
:1076500036350A4E313433352058322E3330362009
:1076600059302E3834310A4E313434302058322ECD
:107670003232322059302E3931310A4E31343435DC
:107680002058322E3131342059302E3939350A4EB6
:10769000313435302058322E3030322059312E30AE
:1076A00037360A4E313435352058312E39303520B1
:1076B00059312E3133390A4E313436302058312E7B
:1076C0003735342059312E3232330A4E3134363583
:1076D0002058312E3633372059312E3237380A4E62
:1076E000313437302058312E3538322059312E334D
:1076F00030310A4E313437352058312E3535382067
:1077000059312E3331350A4E313438302058312E2C
:107710003436302059312E3335320A4E3134383533
:107720002058312E3339392059312E3336300A4E14
:10773000313439302058312E3333382059312E33FB
:1077400035340A4E313439352058312E323837200D
:1077500059312E3332390A4E313530302058312EDE
:107760003234382059312E3239340A4E31353035E1
:107770002058312E3231372059312E3235340A4ECD
:10778000313531302058312E3231342059312E32BA
:1077900035320A4E313531352058312E31373220CD
:1077A00059312E3139350A4E313532302058312E8B
:1077B0003132382059312E3133390A4E3135323594
:1077C0002058312E3131302059312E3131370A4E87
:1077D000313533302058302E3935382059302E3954
:1077E00034310A4E313533352058302E3839312076
:1077F00059302E3837330A4E313534302058302E38
:107800003832352059302E3830380A4E313534353B
:107810002058302E3735352059302E3734370A4E20
:10782000313535302058302E3631392059302E360A
:1078300033330A4E313535352058302E3437372022
:1078400059302E3532360A4E313536302058302EEA
:107850003437372059302E3532340A4E31353635EB
:107860002058302E3431312059302E3437360A4EDC
:10787000313537302058302E3333312059302E34C3
:1078800035340A4E313537352058302E32373820CE
:1078900059302E3432370A4E313538302058302E98
:1078A0003233312059302E3339370A4E313538359D
:1078B0002058302E3138332059302E3337390A4E84
:1078C000313539302058302E3133352059302E3370
:1078D00036350A4E313539352058302E303736207E
:1078E00059302E3334310A4E31363035204730305E
:1078F000204633302E300A4E31363130204D30356F
:10790000200A4E3136313520473930205830205941
:1079100030205A300A4E31363135204D33300A2866
:10792000456E64206F6620434E432050726F67722D
:10793000616D2900284D53472A2A2A2A204D696360
:10794000726F737465702054657374205B76315D5B
:10795000202A2A2A2A290A4730302047313720474F
:1079600032312047343020473439204738302047DF
:1079700039300A6730783079307A300A7B22316DBD
:1079800069223A317D0A7B22326D69223A317D0AC1
:107990007B22336D69223A317D0A7B22346D692264
:1079A0003A317D0A6730207831300A7B22316D69A7
:1079B000223A327D0A78300A7B22316D69223A34CC
:1079C0007D0A7831300A7B22316D69223A387D0A8E
:1079D00078300A6730207931300A7B22326D692293
:1079E0003A327D0A79300A7B22326D69223A347D3F
:1079F0000A7931300A7B22326D69223A387D0A7960
:107A0000300A6730207A31300A7B22336D69223A9E
:107A1000327D0A7A300A7B22336D69223A347D0A3C
:107A20007A31300A7B22336D69223A387D0A7A3006
:107A30000A6730206131300A7B22346D69223A3284
:107A40007D0A61300A7B22346D69223A347D0A61F5
:107A500031300A7B22346D69223A387D0A61300A5E
:107A60006D3200284D53472A2A2A2A20436F6F720D
:107A700064696E617465206F6666736574732074E3
:107A8000657374205B76315D202A2A2A2A290A67C9
:107A900030306731376732316734306734396738AF
:107AA000306739300A6735340A67393278307930CF
:107AB0007A300A663630300A284D53472A2A2A2A55
:107AC000207465737420473932206F66667365745D
:107AD000732A2A2A2A290A286D736753746570202D
:107AE000313A204D6F76652066726F6D20302C30F4
:107AF00020746F2033302C30206D6D20696E207023
:107B00006F7369746976652058206469726563745F
:107B1000696F6E290A286D73675374657020323A55
:107B2000205265736574206F726967696E20746F87
:107B300020302E30207573696E6720473932290A4C
:107B4000286D73675374657020333A204D6F7665E6
:107B500020746F2032302C302E2053686F756C6487
:107B6000206D6F7665203230206D6D20696E20703B
:107B70006F736974697665205820646972656374EF
:107B8000696F6E20616E6420737461747573207206
:107B900065706F72742073686F756C6420737461A4
:107BA00072742066726F6D20302C30290A286D7334
:107BB000675374657020343A204D6F766520746F7A
:107BC00020302E3020202053686F756C64206D6F3C
:107BD0007665203230206D6D20696E206E6567619C
:107BE00074697665205820646972656374696F6E84
:107BF00020616E6420737461747573207265706F98
:107C000072742073686F756C642073746172742071
:107C100066726F6D2032302C30290A67317833302C
:107C20000A67393278300A67317832300A6731783A
:107C30003079300A2473720A67393278300A67342F
:107C400070302E350A284D53472A2A2A2A20746577
:107C5000737420473535206F6666736574732A2AFE
:107C60002A2A290A286D73675374657020313A20D7
:107C700053657420436F6F7264696E61746520731D
:107C8000797374656D2032205B6735355D20746FC4
:107C9000206F6666736574206F662035302C353032
:107CA000290A286D73675374657020323A20536532
:107CB0006C6563742047353520636F6F7264696E3D
:107CC0006174652073797374656D290A286D736713
:107CD0005374657020333A204D6F766520746F20A1
:107CE000302C302E20486561642073686F756C6499
:107CF000206D6F766520646961676F6E616C6C7969
:107D000020696E202B5820616E64202B5920616EF3
:107D10006420737461747573207265706F7274205F
:107D200073686F756C642073746172742066726F0F
:107D30006D20302C30290A6731304C327032783562
:107D4000307935300A6735350A6730783079300A4E
:107D5000673470302E350A284D53472A2A2A2A20A4
:107D60007465737420473533206162736F6C75746A
:107D700065206F7665727269646573202A2A2A2AE3
:107D8000290A286D73675374657020313A20527543
:107D90006E20612073717561726520696E204735B0
:107DA000352073797374656D290A286D7367537470
:107DB000657020323A2052756E20612073717561B2
:107DC000726520772F473533206F7665727269644C
:107DD00065290A6730783079300A6730783230792F
:107DE000300A67307832307932300A67307830794B
:107DF00032300A6730783079300A673470302E3587
:107E00000A6735336730783079300A673533673041
:107E100078323079300A67353367307832307932EA
:107E2000300A673533673078307932300A67353356
:107E30006730783079300A6730783079300A6734C3
:107E400070302E350A284D53472A2A2A2A20746575
:107E500073742052657475726E20746F20686F6D34
:107E600065202A2A2A2A290A286D736753746570A7
:107E700020313A2052657475726E20746F20686FDD
:107E80006D65207573696E6720473238290A286D41
:107E900073675374657020323A205265736574209D
:107EA000746F2047353420636F6F72642073797369
:107EB00074656D290A6732380A6735340A6D3330C4
:107EC00000284D53472A2A2A2A20546573742061BA
:107ED00063637572616379206F6620736C6F7720BE
:107EE0006D6F766573205B76315D202A2A2A2A29F8
:107EF0000A6735350A6730783079300A6734703070
:107F00002E350A673470302E350A67317831306685
:107F100032320A6735340A6730783079300A6D3387
:107F20003000284D53472A2A2A2A2054657374208A
:107F3000766572792073686F7274206D6F766573E1
:107F4000205B76315D202A2A2A2A290A6730783078
:107F500079300A673470302E350A673178302E3127
:107F600066313030300A78300A78302E310A783075
:107F70000A78302E310A78300A78302E310A78307B
:107F80000A78302E310A78300A78302E310A78306B
:107F90000A78302E310A78300A78302E310A78305B
:107FA0000A78302E310A78300A78302E310A78304B
:107FB0000A78302E310A78300A78302E310A78303B
:107FC0000A78302E310A78300A78302E310A78302B
:107FD0000A78302E310A673470302E350A78300A2C
:107FE00078302E30310A78300A78302E30310A78E5
:107FF000300A78302E30310A78300A78302E30311D
:108000000A78300A78302E30310A78300A78302EEB
:1080100030310A78300A78302E30310A78300A78D8
:10802000302E30310A78300A78302E30310A7830EC
:108030000A78302E30310A78300A78302E30310A02
:1080400078300A78302E30310A78300A78302E3085
:10805000310A78300A78302E30310A67307830793A
:10806000300A6D3200284D53472A2A2A2A20526F9F
:10807000746172792041786973204D6F74696F6EF5
:108080002054657374205B76315D202A2A2A2A29C0
:108090000A673030673137673231673430673439D7
:1080A0006738306739300A6730783079307A306134
:1080B00030623063300A6735350A6730783079309E
:1080C0000A6633363030300A6730613336300A6240
:1080D0003336300A633336300A61300A62300A635D
:1080E000300A673161313434300A62313434300A55
:1080F00063313434300A61300A62300A63300A670F
:1081000031613134343062373230633336300A789B
:108110003079307A306130623063300A67317836D6
:1081200030613134343062373230633336300A787C
:108130003079307A306130623063300A67317836B6
:108140003079353061313434306237323063333630
:10815000300A783079307A306130623063300A67C3
:1081600031783630793530783235613134343062B7
:10817000373230633336300A783079307A306130D4
:10818000623063300A6735340A6730783079300AF4
:108190006D333000284D53472A2A2A2A20496E760B
:1081A000657273652054696D65204D6F74696F6EDB
:1081B0002054657374205B76315D202A2A2A2A298F
:1081C0000A673030673137673231673430673439A6
:1081D0006738306739300A6735350A673078307963
:1081E000300A6739330A66302E30310A6731783108
:1081F000300A7931300A7A31300A6131300A783008
:108200000A79300A7A300A61300A67317831307978
:1082100031307A2D31306131300A67307830793041
:108220007A3061300A66302E310A6732783130791F
:108230002D31307A2D32306931300A67307830791B
:10824000307A300A6733783130792D31307A2D32F7
:10825000306931300A6730783079307A300A6732E5
:1082600078323079307A2D32306931300A6730789F
:108270003079307A300A673378323079306931308A
:108280000A6730783079307A300A6732783079305E
:108290007A2D33306931300A6733783079307A306B
:1082A0006931300A6730783079307A300A6732784D
:1082B00030793069323020284357203336302064FB
:1082C000656772656573290A67337830793069327A
:1082D0003020284343572033363020646567726569
:1082E0006573290A6739340A6735340A673078308C
:1082F00079300A6D3330007B226763223A2267307F
:108300003067313767323167343067343967383036
:10831000673930227D0A7B226763223A226735352E
:10832000227D0A7B226763223A22673078307930D7
:10833000227D0A7B226763223A2266353030227D15
:108340000A7B226763223A22284D53477371756175
:1083500072657329227D0A7B226763223A22673085
:10836000783230227D0A7B226763223A22793230CA
:10837000227D0A7B226763223A227830227D0A7BA3
:10838000226763223A227930227D0A7B22676322A8
:108390003A226731783130227D0A7B226763223AA4
:1083A00022793130227D0A7B226763223A2278309B
:1083B000227D0A7B226763223A227930227D0A7B62
:1083C000226763223A22284D5347636972636C65C2
:1083D0007329227D0A7B226763223A226732783131
:1083E00030792D3130693130227D0A7B226763225A
:1083F0003A22673078307930227D0A7B2267632207
:108400003A226733783130792D3130693130227D2D
:108410000A7B226763223A22673078307930227DE6
:108420000A7B226763223A226732783230793069D8
:108430003130227D0A7B226763223A22673078300E
:108440007930227D0A7B226763223A2267337832B1
:10845000307930693130227D0A7B226763223A22EB
:10846000673078307930227D0A7B226763223A2296
:10847000673278307930693130227D0A7B22676338
:10848000223A22673378307930693130227D0A7B95
:10849000226763223A22673534227D0A7B22676392
:1084A000223A22673078307930227D0A7B22676356
:1084B000223A226D3330227D00284D53472A2A2A42
:1084C0002A204D636F6465732074657374205B7636
:1084D000315D202A2A2A2A290A6735350A67307829
:1084E0003079300A6D330A673470310A6D350A67A6
:1084F0003470310A6D340A673470310A6D350A6799
:108500003470310A6D370A673470310A6D390A6781
:108510003470310A6D380A673470310A6D390A6671
:108520003530300A67307832300A7932300A6D33AC
:108530000A78300A6D340A79300A6D350A67317865
:1085400031300A6D370A7931300A6D380A78300ACD
:108550006D390A79300A6732783130792D313069D6
:1085600031300A6D330A6730783079300A6D340A59
:108570006733783130792D31306931300A6D350A01
:108580006730783079300A6D370A6732783230795F
:10859000306931300A6D380A6730783079300A6DC9
:1085A000390A673378323079306931300A67307888
:1085B0003079300A6732783079306931300A673380
:1085C000783079306931300A6735340A673078306D
:1085D00079300A6D333000284D53472A2A2A2A2041
:1085E00046656564686F6C642054657374205B76BF
:1085F000315D202A2A2A2A290A284D53472A2A2A65
:108600002A204D616E75616C6C7920656E7465729F
:10861000202120616E64207E20647572696E67205F
:108620006D6F76656D656E7420746F2074657374FC
:10863000202A2A2A2A290A6735350A6730783079AC
:10864000300A673470330A67303067313767323148
:108650006734306734396738306739300A66363006
:10866000300A6730783130307637362E3736350A73
:10867000783079300A6735340A6730783079300AD3
:108680006D333000284D53472A2A2A2A2044776523
:108690006C6C2054657374205B76315D202A2A2A25
:1086A0002A290A6730306731376732316739300A33
:1086B0006735350A6730783079300A663530300AE8
:1086C00067307831300A673470310A673078323079
:1086D0000A673470310A67307831300A6734703194
:1086E0000A67307830300A673470310A79350A67A2
:1086F00035340A6730783079300A6D330A67347060
:10870000310A67307831307931300A6D350A673493
:1087100070310A67307832307932300A6D340A6746
:108720003470310A67307833307933300A6D380A63
:10873000673470310A67307834307934300A6D39F3
:108740000A673470310A67307835307935300A6716
:1087500030783079300A6D3330004E312067303058
:10876000673137673231673430673439673830679B
:1087700039300A4E3130206730783079300A4E3245
:108780003020663530300A4E333020673278313051
:10879000792D31306931302028435720323730204D
:1087A00064656772656573290A4E343020673078D6
:1087B0003079300A4E3530206733783130792D31B9
:1087C00030693130202843435720393020646567B1
:1087D00072656573290A4E363020673078307930FB
:1087E0000A4E3830206732783230793069313020A3
:1087F00028435720313830206465677265657329D6
:108800000A4E3730206730783079300A4E383020C1
:10881000673378323079306931302028434357202C
:108820003138302064656772656573290A4E3930C6
:10883000206730783079300A4E393920463132306D
:10884000300A4E313030206732783079306932303A
:10885000202843572033363020646567726565737E
:10886000290A4E3131302067327830793069323020
:10887000202843572033363020616761696E290A0A
:108880004E313230206637303020284368616E67C1
:108890006520666565642072617465207768696C1F
:1088A0006520696E204732206D6F74696F6E206D90
:1088B0006F6465290A4E3133302067327830793061
:1088C00069323020284357203336302033726420F9
:1088D00074696D65290A4E313430206732783079F9
:1088E00030693230202843572033363020347468C2
:1088F0002074696D65290A4E313530206635303077
:108900000A4E313630206733783079307A34306926
:108910003230202843435720333630206465677255
:108920006565732077697468206C696E6561722073
:1089300074726176656C290A4E313730206733785E
:108940003079307A3069323020284343572033362B
:108950003020616761696E290A4E313830206637F0
:10896000303020286D73672A2A2A2A4368616E678F
:108970006520666565642072617465207768696C3E
:108980006520696E204733206D6F74696F6E206DAE
:108990006F64652A2A2A2A290A4E31393020673322
:1089A00078307930693230202843435720333630CD
:1089B000203372642074696D65290A4E323030208C
:1089C0006733783079306932302028434357203379
:1089D0003630203474682074696D65290A4E32314E
:1089E0003020286D73672A2A2A2A47313820457695
:1089F000616C20746573742A2A2A2A290A4E32323D
:108A000030204731205833302E373037205A353018
:108A10002E37323720463530300A4E323330204739
:108A2000313820473032205836372E373338205AE5
:108A300032332E3631372052323520463235300A25
:108A40004E323430206738300A4E323530206730AD
:108A5000783079307A300A4E323630206D3330003B
:108A6000284D53472A2A2A2A20537175617265734B
:108A7000204D6F74696F6E2054657374205B76317E
:108A80005D202A2A2A2A290A67303067313767325F
:108A9000316734306734396738306739300A6730C6
:108AA000783079300A6730783230202874726176F5
:108AB0006572736520612032306D6D207371756150
:108AC000726520696E205820616E642059290A79E8
:108AD00032300A78300A79300A67317831306635B9
:108AE000303020286472617720612031306D6D2034
:108AF00073717561726520696E205820616E642003
:108B0000592061742046353030290A7931300A788D
:108B1000300A79300A67307A3230202874726176F0
:108B20006572736520612032306D6D2073717561DF
:108B3000726520696E205820616E64205A290A7877
:108B400032300A7A300A78300A6731783230793236
:108B5000307A3230663530302028666565642061B1
:108B60002032306D6D20646961676F6E616C2069C1
:108B70006E20582C205920616E64205A290A7830C2
:108B800079307A300A7834307934307A34302028A9
:108B9000747261766572736520612034306D6D206A
:108BA0006375626520696E20582C205920616E64BF
:108BB000205A290A78343079307A300A783079347A
:108BC000307A34300A7834307934307A300A783078
:108BD00079307A34300A78307934307A300A78341F
:108BE0003079307A34300A783079307A300A673820
:108BF000300A6730783079300A673078310A673068
:108C000078300A6D333000284D53472A2A2A2A200B
:108C1000486F6D696E672054657374205B76315DB3
:108C2000202A2A2A2A290A6732382E3278307930C7
:108C30007A300A6D333000284D53472A2A2A2A20D9
:108C4000536D6F6B652054657374205B76315D20C6
:108C50002A2A2A2A290A473030204731372047322A
:108C600031204734302047343920473830204739C5
:108C7000300A6D33673470310A6D35673470310AEC
:108C80006D34673470310A6D33673470310A6D3575
:108C9000673470310A6D37673470310A6D39673463
:108CA00070310A6D38673470310A6D390A6730786F
:108CB0003079307A300A673030207832300A7830B4
:108CC0000A7932300A79300A7A32300A7A300A6107
:108CD00032300A61300A4730302078323020793221
:108CE00030207A3230206132300A473030207830FC
:108CF000207930207A302061300A473031206633C5
:108D000030207832207932207A322061320A78306D
:108D1000207930207A302061300A673078310A6754
:108D20003078300A6D32005B74765D20207465788F
:108D30007420766572626F736974792531356420A9
:108D40005B303D73696C656E742C313D7665726283
:108D50006F73655D0A0025660A00256C750A00259B
:108D6000730A0074696E7967205B25735D206572F4
:108D7000723A2025733A202573200074696E796752
:108D8000205B25735D206F6B3E2000456E64206F75
:108D90006620636F6D6D616E642066696C650A00A4
:108DA00085C927C7F2C913CA72CA6CC74ACD27C77B
:108DB000DECD4ACE78CC6CC700004006400610409D
:108DC000B800B84ACD27C7DECD4ACE78CC6CC700F4
:108DD00000400620060840B800B8B3CF27C7D3CE5E
:108DE0004FCFFED09CCEA00840060506090108B36F
:108DF000CF27C7D3CE4FCF84CA6CC7B00840060573
:108E000040B030800000000000F0E0D0C010010051
:108E1000CF673322211F1B1301016E616E00696E43
:108E200066004E414E494E495459494E46CDCCCC30
:108E30003D0AD7233C17B7D13877CC2B329595E62E
:108E4000241FB14F0A000020410000C84200401C0E
:108E50004620BCBE4CCA1B0E5AAEC59D7400407A5B
:108E600010F35A00A0724E18090010A5D4E80000B3
:108E7000E87648170000E40B54020000CA9A3B0051
:108E80000000E1F505000080969800000040420FC8
:108E9000000000A08601000000102700000000E88C
:108EA00003000000006400000000000A0000000051
:108EB000000100000000002C76D888DC674F0823F2
:108EC000DFC1DFAE59E1B1B796E5E3E453C63AE658
:108ED00051997696E8E6C28426EB898C9B62ED4038
:108EE0007C6FFCEFBC9C9F40F2BAA56FA5F4900587
:108EF0005A2AF75C936B6CF9676DC11BFCE0E40DBB
:108F000047FEF520E6B500D0ED902E0300943577AE
:108F1000050080841E080000204E0A000000C80CD6
:108F2000333333330F986E12831141EF8D2114893F
:108F30003BE65516CFFEE6DB18D1844B381BF77C99
:108F40001D901DA4BBE424203284725E228100C9DE
:108F5000F124ECA1E53D270011241FBECFEFCDBFCA
:108F6000DFE5DEBF00E00CBF13E2A0E0B0E2E0E42A
:108F7000F9EC01E00BBF02C007900D92AA38B107CF
:108F8000D9F72CE5AAE8B3E201C01D92A037B207D9
:108F9000E1F70E9453820C949EE40C940000FC01C3
:108FA00060817181828193810E944CD660933F35AC
:108FB0000895FC0160817181828193810E944CD669
:108FC00060933E350895AF92BF92CF92DF92EF92B9
:108FD000FF920F931F93CF93DF937B018C0182EC61
:108FE000C82E84E3D82EE601AA24A394BC2EBC1874
:108FF000F70161917191819191917F012CEA35EC9A
:1090000047E257E30E94DBD718164CF4F801408181
:109010005181628173818B2D0E948283A8820C5FB3
:109020001F4F2196F4E3C83CDF0701F7DF91CF9192
:109030001F910F91FF90EF90DF90CF90BF90AF9076
:109040000C948D83FC0160817181828193810E94E7
:109050004CD660934035613019F481E00E948B78E2
:1090600081E00C94AC78CF93DF93CDB7DEB76897EF
:10907000CDBFDEBFFC0160817181828193810E943E
:109080004CD66093413581E0613019F40E948B78B1
:109090000CC00E94AC78CE01019628E1FC0111922F
:1090A0002A95E9F7BC010E9422486896CDBFDEBF31
:1090B000DF91CF9108950F931F93CF93DF93CDB797
:1090C000DEB72D97CDBFDEBF27E0E8EDF0E28E01E1
:1090D0000F5F1F4FD80101900D922A95E1F7BC0157
:1090E000660F771F680F791F660F771F660F771F50
:1090F000660F771F65557A4E45E050E0CE01089621
:109100000E9412E2688570E0C8010E9440E2009768
:1091100039F46B8570E0C8010E9440E2009711F0BD
:10912000801B01C08FEF2D96CDBFDEBFDF91CF91A9
:109130001F910F9108950F931F93CF93DF93CDB796
:10914000DEB7C058D109CDBFDEBFFC010D96248526
:109150002F9323852F9322852F9321852F939F93E0
:109160008F937196FF93EF939F938F937F936F935A
:109170008E010F5F1F4F1F930F930E94C9E3C80119
:109180000E943BC1CDBFDEBFC058DF4FCDBFDEBFA9
:10919000DF91CF911F910F910895EF92FF920F935E
:1091A0001F93CF93DF93CDB7DEB7C058D109CDBFA2
:1091B000DEBF8C01F62EE72EFC01848195810E9492
:1091C0005B4883309CF58F3F09F03BC02FC098016E
:1091D000235F3F4F9F938F93F80184858F938385FF
:1091E0008F9382858F9381858F933F932F930F5E0B
:1091F0001F4F1F930F933F932F93EF92FF928E0178
:109200000F5F1F4F1F930F930E94C9E3C8010E9475
:109210003BC1CDBFDEBFC058DF4FCDBFDEBFDF914A
:10922000CF911F910F91FF90EF900895EAE2F4E142
:10923000659174914FE450E084E69FE30E9412E24E
:10924000C6CFE0913835F0E0EE0FFF1FEA5DFB4E30
:10925000659174914FE450E084E69FE30E9412E22E
:10926000B6CFEF92FF920F931F93CF93DF93CDB7BB
:10927000DEB7C058D109CDBFDEBF8C01F62EE72E78
:10928000FC01848195810E945B488330B4F58F3F57
:1092900009F03EC032C0A8014F5E5F4F9801235FC6
:1092A0003F4F9F938F93F80184858F9383858F938E
:1092B00082858F9381858F935F934F933F932F93F5
:1092C0005F934F933F932F93EF92FF928E010F5F27
:1092D0001F4F1F930F930E94C9E3C8010E943BC117
:1092E000CDBFDEBFC058DF4FCDBFDEBFDF91CF9116
:1092F0001F910F91FF90EF900895EAE2F4E16591DC
:1093000074914FE450E084E69FE30E9412E2C3CFE1
:10931000E0913835F0E0EE0FFF1FEA5DFB4E6591FE
:1093200074914FE450E084E69FE30E9412E2B3CFD1
:10933000DF92EF92FF920F931F93CF93DF93CDB7FE
:10934000DEB7C858D109CDBFDEBF8B01E42ED52EC4
:1093500037E0EFEDF0E2DE01AF57BF4F01900D9225
:109360003A95E1F7C857DF4F2883C858D0400E948C
:109370005B48F82EC857DF4F2881C858D04082E09C
:109380008F1518F0E22FF0E002C0E2E0F0E0EE0FFF
:10939000FF1FEA5DFB4E659174914FE450E084E657
:1093A0009FE30E9412E29F938F93F80183818F9332
:1093B00082818F9381818F9380818F93E1E8F0E0A8
:1093C000EC0FFD1FEF0DF11D80811F928F93DF9237
:1093D000EF928E010F5F1F4F1F930F930E94C9E3FF
:1093E000C8010E943BC1CDBFDEBFC857DF4FCDBF14
:1093F000DEBFDF91CF911F910F91FF90EF90DF9033
:1094000008954F925F926F927F92AF92BF92CF92E8
:10941000DF92EF92FF920F931F93CF93DF93C2ECF3
:10942000D4E307E813E35C018991813009F042C07D
:10943000F801C480D580E680F7804080518062804A
:109440007380A3019201C701B6010E942FD49F77B8
:109450002CEA35EC47E257E30E94D8D587FD2AC0B5
:1094600020E034E244E759ECC701B6010E94DBD7A3
:1094700018165CF4F5012081318142815381C701C6
:10948000B6010E94DBD7181604F120E034E244E76D
:1094900059ECC301B2010E94DBD718165CF4F50148
:1094A0002081318142815381C301B2010E94D8D50C
:1094B00087FD0BC00B5C1F4FF4E0AF0EB11C84E3C3
:1094C000C83CD80709F0B0CF02C08CED01C080E0E5
:1094D000DF91CF911F910F91FF90EF90DF90CF9090
:1094E000BF90AF907F906F905F904F900895809164
:1094F000BE34811105C08091BD348093BC3429C035
:10950000823031F487E08093BC348091BD3421C037
:10951000833031F489E08093BC348091BD3419C02C
:10952000843031F48AE08093BC348091BD3411C022
:109530008091BF34813031F485E08093BC348091D8
:10954000BD3407C0823019F486E08093BC3480912A
:10955000BD34863019F08091BC3408958BE080933F
:10956000BC3408958091BD3408958093BF34813018
:1095700059F018F0823041F008958DEE94E3809315
:10958000EB349093EC34089583EB98E58093EB34BF
:109590009093EC340895FC0184810895845B9F4F7F
:1095A000FC0180810895855B9F4FFC0180810895B7
:1095B000825B9F4FFC0180810895815B9F4FFC017E
:1095C00080810895875B9F4FFC01808108950C94F2
:1095D0008398CD96FC016081718182819381089589
:1095E000FC01648308958B5A9F4FFC0160830895AA
:1095F0008F5B9F4FFC014083518362837383089587
:109600006093ED347093EE348093EF349093F034A4
:1096100088EE91E20C94F062BF92CF92DF92EF92CB
:10962000FF920F931F93CF93DF93D0903A357C0135
:109630000FE515E38091393590E0EC01CC0FDD1F8B
:10964000C80FD91FCC0FDD1FCC0FDD1FCC0FDD1FC6
:10965000CA52DD4C81E0D816A9F0B881A981CA8030
:10966000BB804091B235413091F4F80120813181C5
:10967000428153816B2F7A2F8C2D9B2D0E9430D4E9
:109680009B0109C020E030E080E090E004C02B2F77
:109690003A2F8C2D9B2DA901BC01F701458F568FC8
:1096A000678F70A3F4E0EF0EF11C0C5F1F4F249640
:1096B00085E30737180771F6DF91CF911F910F915E
:1096C000FF90EF90DF90CF90BF900895835B9F4F06
:1096D000FC0160838DEE94E30C940C4B4F925F92EF
:1096E0006F927F928F929F92AF92BF92CF92DF92B2
:1096F000EF92FF920F931F93CF93DF93CDB7DEB717
:109700006897CDBFDEBF8C016091B23570E080E01C
:1097100090E00E947AD62B013C01F80160817181B2
:10972000828193810E944CD670E05B01AA0CBB1C25
:10973000A60EB71EAA0CBB1CAA0CBB1CAA0CBB1CF9
:10974000C5018A529D4C5C010FE515E3FE0131967F
:109750004F01F501C190D190E190F1905F01F801C6
:1097600061917191819191918F01A30192010E9468
:109770007DD89B01AC01C701B6010E9430D4F40131
:1097800061937193819391934F01F5E307371F071D
:1097900001F7CE0101960E9466988DEE94E30E9437
:1097A0000C4B6896CDBFDEBFDF91CF911F910F911B
:1097B000FF90EF90DF90CF90BF90AF909F908F90F1
:1097C0007F906F905F904F9008958D5E944369F401
:1097D000E62FF0E0EE0FFF1FEE0FFF1FE95BFA4CE4
:1097E00060817181828193810895862F0C945B98AA
:1097F000CF92DF92EF92FF920F931F93CF93DF935D
:10980000EC0184E3CD3ED80709F04AC070E0FB01CB
:10981000EE0FFF1FEE0FFF1FE95BFA4CC080D180F7
:10982000E280F38080913A35813059F18091393569
:1098300090E0FC01EE0FFF1FE80FF91FEE0FFF1F76
:10984000E60FF71FEE0FFF1FEE0FFF1FEA52FD4C52
:1098500000811181B281A3812091B2352130B1F410
:10986000FB01EE0FFF1FEE0FFF1FE15AFA4C2081A4
:10987000318142815381B8018B2F9A2F0E9430D4BD
:1098800008C060E070E080E090E003C0B8018B2F7A
:109890009A2F9B01AC01C701B6010E942FD403C0CF
:1098A000862F0E946F98C55BDF4F2881211106C06B
:1098B00023E333E34BEC51E40E94DFD5DF91CF91FA
:1098C0001F910F91FF90EF90DF90CF90089588E166
:1098D000E2EFF4E3A7E4B5E301900D928A95E1F796
:1098E0008091363581110CC08091F134813041F482
:1098F00010922A3510922B3510922C3510922D355E
:1099000008954F925F926F927F928F929F92AF9243
:10991000BF92CF92DF92EF92FF920F931F93CF935C
:10992000DF93CDB7DEB76997CDBFDEBF8091BE3480
:10993000811155C08091E334813009F050C00E94FC
:10994000C6C681114CC01092E3349EEE692E92E39C
:10995000792E26E3822E912C8E010E5E1F4F36EE5D
:10996000A32E30E2B32E33C0F70181917F011F9205
:109970008F935F924F92BF92AF921F930F930E946B
:10998000A0E3B80187E493E20E94E65F8D839E83A3
:10999000F60181919191A191B1916F018A879B8785
:1099A000AC87BD87CE0101960E94AE5CCDBFDEBF05
:1099B0009EEDE91690E2F906B9F6E8E16E0E711C2B
:1099C000FFEF8F1A9F0A8CE38816910441F024015F
:1099D00089EDE82E80E2F82E630188E7C8CF80E0A9
:1099E0006996CDBFDEBFDF91CF911F910F91FF90A0
:1099F000EF90DF90CF90BF90AF909F908F907F902F
:109A00006F905F904F9008952F923F924F925F9288
:109A10006F927F928F929F92AF92BF92CF92DF927E
:109A2000EF92FF920F931F93CF93DF93CDB7DEB7E3
:109A30002997CDBFDEBF4C015B0140903C35509073
:109A40003A35209039356090B235709038356B01D9
:109A500082EF94E3888799875EE7E52E53E3F52E3E
:109A600098E1299E100111248401D6016D917D9108
:109A70008D919D916D012CEA35EC47E257E30E94F0
:109A8000D8D587FD80C0F70180818150823008F0F1
:109A90007AC041104CC0F1E05F1609F1E885F98504
:109AA000E20DF31DEC51F2408081898391819D8309
:109AB000B281A381E1E06E1217C0E885F985E35910
:109AC000FF4F2081318142815381BC018B2F9A2F1E
:109AD0000E9430D469837D838E839F8307C019825F
:109AE0001D821E821F8202C0BE83AF8371100CC014
:109AF00023E333E34BEC51E4D8016D917D918D91DB
:109B00009C910E947DD805C0F8016081718182819D
:109B1000938129813D814E815F810E9430D4A88547
:109B2000B9856D937D938D939C9313972CC0A885D5
:109B3000B9858D919D910D90BC91A02D89839A83BB
:109B4000AB83BC8371100EC023E333E34BEC51E4D1
:109B5000F80160817181828193810E947DD89B018F
:109B6000AC0105C0D8012D913D914D915C91698169
:109B70007A818B819C810E9430D4E885F98560834D
:109B800071838283938388859985049688879987D2
:109B900095E3E90EF11C0C5F1F4FA885B985AE5FF8
:109BA000B44309F062CF6090383570903C35F09145
:109BB0003A35F983C09039352091B2352D838CE048
:109BC000A80EB11CADE1B4E3A887B9874EEFE42E2F
:109BD00044E3F42EB8E1CB9E600111248401F50129
:109BE00061917191819191915F012CEA35EC47E28D
:109BF00057E30E94D8D587FD8CC0A885B9858C9184
:109C0000882309F486C08150823030F4F80124841E
:109C10003584468457843BC0611016C023E333E388
:109C20004BEC51E4D8011C966D917D918D919C91E6
:109C30001F970E947DD820E030E044EB53E40E945F
:109C40007DD81B012C010DC020E030E044EB53E433
:109C5000F80164857585868597850E947DD81B01EE
:109C60002C012BED3FE049EC50E4A885B985919695
:109C70006D917D918D919C9194970E947DD89B01CF
:109C8000AC01C201B1010E94DFD51B012C01711092
:109C900031C0B981B130E1F0F701EC0DFD1DEC519F
:109CA000F240A081B18192808380ED81E130A1F406
:109CB000F701E359FF4F2081318142815381BD017A
:109CC000892D982D0E9430D4DB01982E892E04C056
:109CD000A0E0B0E0912C812CA2019101BD01892D61
:109CE000982D0E9430D4D7016D937D938D939C93D2
:109CF00013970FC0A2019101F701608171818281E8
:109D000093810E9430D4D7016D937D938D939C9362
:109D10001397E885F985F596E887F987F4E0EF0E63
:109D2000F11C0C5F1F4F888599858C5B944309F06B
:109D300056CF2996CDBFDEBFDF91CF911F910F91F6
:109D4000FF90EF90DF90CF90BF90AF909F908F905B
:109D50007F906F905F904F903F902F9008958091EB
:109D6000BA329091BB328F3E924111F08FE5089547
:109D700080917136909172368F3E9241B9F7809101
:109D80004335909144358F3E924181F78091B935AA
:109D90009091BA358F3E924149F780910B5990913D
:109DA0000C598F3E924111F78091C8599091C95931
:109DB0008F3E9241D9F680E008958BE10E9474A90C
:109DC00082E08093BD3480E00895CF93C82F0E9435
:109DD00074A982E08093BD348C2FCF910895809137
:109DE000BE34811104C083E08093BD3403C085E09C
:109DF0008093BD3480E00895CF93C82F0E94C1B4F2
:109E000080E00E9456B08C2F0E9474A986E0809357
:109E1000BD348C2FCF91089581E08093E43480E0AD
:109E2000089581E08093E63480E0089581E0809396
:109E3000E53480E008950E94457980E0089580939C
:109E4000373580E008958093383580E00895809319
:109E50003C3580E008954F925F926F927F929F927F
:109E6000AF92BF92CF92DF92EF92FF920F931F9328
:109E7000CF93DF93C82FB62E8A01F22ED32F8FEF08
:109E80008C0F863008F082C06091453670E080E02B
:109E900090E00E947AD62CEA35EC47E257E30E9424
:109EA000D8D587FD75C082E0B81619F0E4E1BE127E
:109EB00071C090903835CF2CDD2E8C2F90E0EC01C6
:109EC000CC0FDD1FC80FD91FCC0FDD1FCC0FDD1F3E
:109ED000CC0FDD1FCA52DD4C780107E415E3AA243C
:109EE000A394F60161917191819191916F012CEA96
:109EF00035EC47E257E30E94DBD71816DCF5F2E0B9
:109F0000BF1214C091100CC023E333E34BEC51E4B7
:109F1000F70160817181828193810E947DD824C084
:109F2000F70160817181828193811EC0F8014080B8
:109F300051806280738091100EC023E333E34BECB9
:109F400051E4F70160817181828193810E947DD803
:109F50009B01AC0105C0F701208131814281538111
:109F6000C301B2010E942FD4688379838A839B83C3
:109F7000A092E3342496F4E0EF0EF11C0C5F1F4F27
:109F800085E30F35180709F0ACCF06C081EA05C09C
:109F90008CEA03C08DEA01C080E0DF91CF911F9170
:109FA0000F91FF90EF90DF90CF90BF90AF909F9078
:109FB0007F906F905F904F900895CF93DF93CDB7D0
:109FC000DEB76897CDBFDEBF80933935682F70E06C
:109FD00080E090E00E9478D669837A838B839C83AB
:109FE0001D821E821F82188619861A861B861C8671
:109FF0001D861E861F86188A198A1A8A1B8A1C8A41
:10A000001D8A1E8A1F8A188EAE014F5F5F4FBA01EC
:10A010008EE69BE40E94C48480E06896CDBFDEBFDC
:10A02000DF91CF910895CF93DF93EDEEF4E386E5D2
:10A03000DF011D928A95E9F78BE5ABEBB5E3ED0106
:10A04000982F19929A95E9F7A6E1B6E3ED011992D6
:10A050008A95E9F78FEE92E18093BA329093BB3202
:10A060008093713690937236809343359093443544
:10A070008093B9359093BA3580930B5990930C59CE
:10A080008093C8599093C959E093EB34F093EC3422
:10A090008091D332809338358091D1320E94DD4F48
:10A0A0008091D232809337358091D43280933B3582
:10A0B0008091D53280933C3581E080933635809312
:10A0C000B33594E09093F1341092E4341092E53477
:10A0D0001092E6348093BD348093BC340E94F4AE79
:10A0E000DF91CF910C940686CF92DF92EF92FF9290
:10A0F000CF93C82F6A017B01E82FF0E0DF01AA0FA0
:10A10000BB1FAA0FBB1FA95BBA4C4D935D936D9308
:10A110007C931397EE0FFF1FEE0FFF1FEE50FB4CCB
:10A1200040835183628373838C2F0E947783B701AE
:10A13000A6018C2F0E948283CF91FF90EF90DF9039
:10A14000CF900C948D839F92AF92BF92CF92DF926B
:10A15000EF92FF920F931F93CF93DF93CDB7DEB7AC
:10A160006897CDBFDEBF962EA72EC62ED72E7C01B8
:10A1700000E010E0B12CF601619171918191919113
:10A180006F012CEA35EC47E257E30E94DBD7181643
:10A19000A4F58091383581110EC023E333E34BECF5
:10A1A00051E4F70160817181828193810E947DD8A1
:10A1B000AB01BC0105C0F70140815181628173810F
:10A1C000E1E0F0E0EC0FFD1FE00FF11F4083518351
:10A1D00062837383C80186549D4CFC01E357FD4F95
:10A1E0004083518362837383E555F1094083518332
:10A1F000628373838B2D0E947783B3940C5F1F4F10
:10A20000F4E0EF0EF11C0831110509F0B4CF492D2F
:10A210005A2DBE016F5F7F4F83EE97E40E94C48486
:10A2200080E06896CDBFDEBFDF91CF911F910F9187
:10A23000FF90EF90DF90CF90BF90AF909F900895E8
:10A240004F925F926F927F928F929F92AF92BF9246
:10A25000CF92DF92EF92FF920F931F93CF93DF93F2
:10A26000CDB7DEB76897CDBFDEBF21E02093B23512
:10A2700080903935909038355B016C0107E415E327
:10A28000882D90E07C01EE0CFF1CE80EF91EEE0C10
:10A29000FF1CEE0CFF1CEE0CFF1CC7018A529D4CEC
:10A2A0007C01F50161917191819191915F012CEA9D
:10A2B00035EC47E257E30E94DBD7181664F5F70147
:10A2C0002081318142815381F801608171818281D5
:10A2D00093810E942FD42B013C0191100EC023E3E7
:10A2E00033E34BEC51E4F60160817181828193810B
:10A2F0000E947DD89B01AC0105C0F601208131810F
:10A3000042815381C301B2010E942FD4F801608FB2
:10A31000718F828F938FF4E0CF0ED11C0C5F1F4F93
:10A3200084E0E80EF11C95E30F35190709F0B9CF69
:10A33000682D70E080E090E00E9478D669837A838F
:10A340008B839C831D821E821F82188619861A8623
:10A350001B861C861D861E861F86188A198A1A8AE5
:10A360001B8A1C8A1D8A1E8A1F8A188EAE014F5FA7
:10A370005F4FBA018EE69BE40E94C48480E0689639
:10A38000CDBFDEBFDF91CF911F910F91FF90EF9076
:10A39000DF90CF90BF90AF909F908F907F906F9005
:10A3A0005F904F900895CF93DF93CDB7DEB7689756
:10A3B000CDBFDEBF1092B23510925F35109260357E
:10A3C00010926135109262351092633510926435A7
:10A3D0001092653510926635109267351092683587
:10A3E0001092693510926A3510926B3510926C3567
:10A3F00010926D3510926E3510926F351092703547
:10A400001092713510927235109273351092743526
:10A4100010927535109276356091393570E080E094
:10A4200090E00E9478D669837A838B839C831D8217
:10A430001E821F82188619861A861B861C861D8618
:10A440001E861F86188A198A1A8A1B8A1C8A1D8AE8
:10A450001E8A1F8A188EAE014F5F5F4FBA018EE6CB
:10A460009BE40E94C48480E06896CDBFDEBFDF918C
:10A47000CF910895CF93DF93CDB7DEB76897CDBF67
:10A48000DEBF1092B2356091393570E080E090E027
:10A490000E9478D669837A838B839C831D821E8277
:10A4A0001F82188619861A861B861C861D861E86A4
:10A4B0001F86188A198A1A8A1B8A1C8A1D8A1E8A74
:10A4C0001F8A188EAE014F5F5F4FBA018EE69BE484
:10A4D0000E94C48480E06896CDBFDEBFDF91CF913B
:10A4E0000895CF93DF93CDB7DEB76897CDBFDEBFBA
:10A4F00081E08093B2356091393570E080E090E082
:10A500000E9478D669837A838B839C831D821E8206
:10A510001F82188619861A861B861C861D861E8633
:10A520001F86188A198A1A8A1B8A1C8A1D8A1E8A03
:10A530001F8A188EAE014F5F5F4FBA018EE69BE413
:10A540000E94C48480E06896CDBFDEBFDF91CF91CA
:10A550000895CF931092F1340E94044D8091C4323B
:10A56000813069F482EF94E30E94014AC82F882366
:10A5700031F00E9474A982E08093BD3417C08DEE43
:10A5800094E30E940C4B85E08093BD348091BE34EF
:10A59000811105C081E08093BE340E9469AD8DEECB
:10A5A00094E30E9490980E94674CC0E08C2FCF915A
:10A5B000089588E1E7E4F5E3A7E7B5E301900D929C
:10A5C0008A95E1F780E008950F931F93CF93DF936F
:10A5D000CDB7DEB76A97CDBFDEBF8C0181E0809337
:10A5E0003A358DEE94E3698F7A8F0E940C4B698D1A
:10A5F0007A8DC8010E94A9520E94FE838823E1F34C
:10A6000088E1E0E0F0E2DE01119601900D928A957A
:10A61000E1F7BE016F5F7F4F87E795E30E94A95284
:10A620006A96CDBFDEBFDF91CF911F910F91089544
:10A6300088E1E7E4F5E3AFE8B5E301900D928A9590
:10A64000E1F780E008950F931F93CF93DF93CDB789
:10A65000DEB76A97CDBFDEBF8C0181E080933A35CB
:10A660008DEE94E3698F7A8F0E940C4B698D7A8D01
:10A67000C8010E94A9520E94FE838823E1F388E169
:10A68000E0E0F0E2DE01119601900D928A95E1F78B
:10A69000BE016F5F7F4F8FE895E30E94A9526A96D3
:10A6A000CDBFDEBFDF91CF911F910F910895FB01C8
:10A6B000DC0180913635811111C09B01AD0160E054
:10A6C00070E080E89FE30E94DFD560932A357093A5
:10A6D0002B3580932C3590932D3518C080913835CB
:10A6E000811109C023E333E34BEC51E4CD010E9417
:10A6F0007DD8FB0101C0CD01AF01BC0140932A35DB
:10A7000050932B3560932C3570932D3580E0089550
:10A710008093363580E0089580933B3580E008953E
:10A72000609332357093333580933435909335355B
:10A730000E941C8580E008950F931F93CF93DF93B1
:10A74000EC018B0180913635882399F080912A3570
:10A7500090912B35A0912C35B0912D35BC01CD01B8
:10A760009F772CEA35EC47E257E30E94D8D587FD66
:10A7700030C081E08093F134B801CE010E94044DD5
:10A780008091C432813069F482EF94E30E94014ADF
:10A79000C82F882331F00E9474A982E08093BD34D1
:10A7A00019C08DEE94E30E940C4B85E08093BD347C
:10A7B0008091BE34811105C081E08093BE340E9437
:10A7C00069AD8DEE94E30E949098C82F0E94674C6B
:10A7D00001C0CEE88C2FDF91CF911F910F9108958A
:10A7E000CF93DF93CDB7DEB76897CDBFDEBF682FBD
:10A7F00070E080E090E00E9478D669837A838B8352
:10A800009C831D821E821F82188619861A861B86CB
:10A810001C861D861E861F86188A198A1A8A1B8A1C
:10A820001C8A1D8A1E8A1F8A188EAE014F5F5F4FD9
:10A83000BA018FEC97E40E94C48480E06896CDBF93
:10A84000DEBFDF91CF910895CF93DF93CDB7DEB711
:10A850006897CDBFDEBF60913F3570E080E090E04B
:10A860000E9478D669837A838B839C831D821E82A3
:10A870001F82188619861A861B861C861D861E86D0
:10A880001F86188A198A1A8A1B8A1C8A1D8A1E8AA0
:10A890001F8A188EAE014F5F5F4FBA0189ED97E4B2
:10A8A0000E94C48480E06896CDBFDEBFDF91CF9167
:10A8B0000895CF93DF93CDB7DEB76897CDBFDEBFE6
:10A8C000682F70E080E090E00E9478D669837A83F8
:10A8D0008B839C831D821E821F82188619861A868E
:10A8E0001B861C861D861E861F86188A198A1A8A50
:10A8F0001B8A1C8A1D8A1E8A1F8A188EAE014F5F12
:10A900005F4FBA0182E298E40E94C48480E06896B6
:10A91000CDBFDEBFDF91CF910895CF93DF93CDB749
:10A92000DEB76897CDBFDEBF682F70E080E090E0B3
:10A930000E9478D669837A838B839C831D821E82D2
:10A940001F82188619861A861B861C861D861E86FF
:10A950001F86188A198A1A8A1B8A1C8A1D8A1E8ACF
:10A960001F8A188EAE014F5F5F4FBA0183E398E4F0
:10A970000E94C48480E06896CDBFDEBFDF91CF9196
:10A980000895CF93FC0160817181828193810E943F
:10A990004CD66093BD341092BF348DEE94E3809317
:10A9A000EB349093EC348091BE34813011F41092EA
:10A9B000BE341092C0341092E6340E944998C0917F
:10A9C000BD34C430C9F40E94D3518091D1320E9469
:10A9D000DD4F8091D232809337358091D53280938C
:10A9E0003C3580E00E9456B080E00E948D5481E0AA
:10A9F00080933635C093F13481E0CF910C944CAC08
:10AA00008093AF358093B0358093B83580E008955A
:10AA10002CEA35EC47E257E360915D3670915E3683
:10AA200080915F36909160360E94DBD71816B4F49F
:10AA30008091023690910336A0910436B09105368C
:10AA4000BC01CD019F772CEA35EC47E257E30E9429
:10AA5000D8D587FF03C01092AF3503C081E0809343
:10AA6000AF3580E008958093AF35809102369091A4
:10AA70000336A0910436B09105368093A7359093A4
:10AA8000A835A093A935B093AA3580E008952CEAA3
:10AA900035EC47E257E360915D3670915E36809108
:10AAA0005F36909160360E94DBD71816B4F480911F
:10AAB000023690910336A0910436B0910536BC0160
:10AAC000CD019F772CEA35EC47E257E30E94D8D5B9
:10AAD00087FF03C01092B03503C081E08093B0358A
:10AAE00080E008958093B0358091023690910336CE
:10AAF000A0910436B09105368093AB359093AC3578
:10AB0000A093AD35B093AE3580E008952CEA35ECD6
:10AB100047E257E360915D3670915E3680915F3613
:10AB2000909160360E94DBD71816B4F480910236FB
:10AB300090910336A0910436B0910536BC01CD0149
:10AB40009F772CEA35EC47E257E30E94D8D587FF80
:10AB500003C01092B83503C081E08093B83580E01F
:10AB600008958093B8358091023690910336A09174
:10AB70000436B09105368093B4359093B535A093E3
:10AB8000B635B093B73580E00895BC018DEE90E204
:10AB90000C94136381E08093E434089581E0809302
:10ABA000E534089581E08093E63408951F93CF93B0
:10ABB000DF93CDB7DEB76897CDBFDEBF0E94839825
:10ABC0008130C9F10E9476D20E947AC90E948184A4
:10ABD00080E00E947EAD10E0812F0E945B98AB0167
:10ABE000BC01812F0E9474501F5F1630A9F780E0CE
:10ABF00090E0A0E4B0E489839A83AB83BC831D8298
:10AC00001E821F82188619861A861B861C861D8640
:10AC10001E861F86188A198A1A8A1B8A1C8A1D8A10
:10AC20001E8A1F8A188EBE016F5F7F4FCB010E9464
:10AC3000C15480E001C08AE66896CDBFDEBFDF91D7
:10AC4000CF911F9108958091E4348130A9F420912F
:10AC5000BF34213079F48091C03481110BC082E07F
:10AC60008093BF3483EB98E58093EB349093EC347E
:10AC70002093C0341092E4348091E534813091F413
:10AC80008091BF34882331F0823061F49091C034D8
:10AC9000943051F40E948398811104C01092E534DD
:10ACA0000E94D6559091C0348091E6348130C1F431
:10ACB0002091E534211114C09150933088F0109206
:10ACC000E63495E09093C0349093BD349091BE34B7
:10ACD000911104C08093BE340E9469AD0E94F5A01A
:10ACE00080E0089585E08093BD348091BE34811169
:10ACF00005C081E08093BE340C9469AD0895CF9374
:10AD0000DF93CDB7DEB76897CDBFDEBF8091BE348D
:10AD1000882311F180E090E0A0E4B0E489839A8375
:10AD2000AB83BC831D821E821F82188619861A86F9
:10AD30001B861C861D861E861F86188A198A1A8AFB
:10AD40001B8A1C8A1D8A1E8A1F8A188EBE016F5F8D
:10AD50007F4FCB010E94C1546896CDBFDEBFDF910B
:10AD6000CF910895CF93DF93CDB7DEB76897CDBF6E
:10AD7000DEBF80E090E0A0E4B0E489839A83AB83F7
:10AD8000BC831D821E821F82188619861A861B8626
:10AD90001C861D861E861F86188A198A1A8A1B8A97
:10ADA0001C8A1D8A1E8A1F8A188EAE014F5F5F4F54
:10ADB000BA0181EC94E50E94C4846896CDBFDEBFE1
:10ADC000DF91CF910895CF93DF93CDB7DEB768972A
:10ADD000CDBFDEBF80E090E0A0E8B0E489839A8335
:10ADE000AB83BC831D821E821F82188619861A8639
:10ADF0001B861C861D861E861F86188A198A1A8A3B
:10AE00001B8A1C8A1D8A1E8A1F8A188EAE014F5FFC
:10AE10005F4FBA0181EC94E50E94C4846896CDBF6F
:10AE2000DEBFDF91CF910895CF93DF93CDB7DEB72B
:10AE30002797CDBFDEBF97E0EFEDF0E2DE01119680
:10AE400001900D929A95E1F7873050F4E1E0F0E03F
:10AE5000EC0FFD1FE80FF11D87FDFA95808101C001
:10AE600080E22796CDBFDEBFDF91CF9108950F938B
:10AE70001F93CF93DF93EC01042F10E020E030E02C
:10AE800009871A872B873C8782E08F8350E0440F25
:10AE9000551F640F751FFB01659174914FE450E0DD
:10AEA00084E69FE30E9412E2BC01CE01DF91CF91C4
:10AEB0001F910F910C94B562CF93DF93EC010E9428
:10AEC000774A482F64E673E1CE01DF91CF910C946D
:10AED00037574091BD3465E273E10C943757409188
:10AEE000BE346CEF72E10C9437574091BF3468EE7A
:10AEF00072E10C9437574091C0346AEB72E10C94C4
:10AF000037574091C1346DE972E10C943757E091A5
:10AF1000EB34F091EC34E55BFF4F408167EC73E17B
:10AF20000C943757E091EB34F091EC34E45BFF4F35
:10AF3000408163ED71E10C943757E091EB34F0916F
:10AF4000EC34448169E371E10C943757E091EB34C0
:10AF5000F091EC34E65BFF4F408166E071E10C94C8
:10AF60003757E091EB34F091EC34E25BFF4F4081D6
:10AF70006CEB70E10C943757E091EB34F091EC34CA
:10AF8000E15BFF4F40816BE770E10C943757E09134
:10AF9000EB34F091EC34E75BFF4F40816CE070E103
:10AFA0000C943757E091EB34F091EC34EF5AFF4FAB
:10AFB000408150E060E070E0FC0141875287638788
:10AFC000748722E0278380E00895E091EB34F091CC
:10AFD000EC344081518162817381FC014187528749
:10AFE0006387748722E0278380E00895CF93DF93FF
:10AFF000EC018091BF34811105C019861A861B8629
:10B000001C8614C00E94529869877A878B879C8718
:10B010002091FE5821110AC025E832E441E25DE3A7
:10B020000E947DD869877A878B879C878C819D81D8
:10B03000FC01EE0FFF1FE80FF91FEE0FFF1FEE0FD1
:10B04000FF1FEE0FFF1FEE54FA4E859194918887F3
:10B0500084E08F8380E0DF91CF910895CF93DF93D9
:10B06000EC012091EB343091EC34F901FD966081D4
:10B0700071818281938169877A878B879C873E96CD
:10B08000208121110AC025E832E441E25DE30E94FB
:10B090007DD869877A878B879C878C819D81FC010D
:10B0A000EE0FFF1FE80FF91FEE0FFF1FEE0FFF1F40
:10B0B000EE0FFF1FEE54FA4E85919491888784E03D
:10B0C0008F8380E0DF91CF910895CF93DF93EC01E0
:10B0D0008C819D810E945B48682F8091EB34909118
:10B0E000EC340E94F84B69877A878B879C878C8128
:10B0F0009D81FC01EE0FFF1FE80FF91FEE0FFF1FF0
:10B10000EE0FFF1FEE0FFF1FEE54FA4E8591949144
:10B11000888784E08F8380E0DF91CF910895CF937B
:10B12000DF93EC018C819D810E945B482091EB3480
:10B130003091EC342D5E344369F4E82FF0E0EE0FEB
:10B14000FF1FEE0FFF1FE95BFA4C60817181828166
:10B15000938102C00E945B9869877A878B879C875E
:10B160008C819D81FC01EE0FFF1FE80FF91FEE0F90
:10B17000FF1FEE0FFF1FEE0FFF1FEE54FA4E8591DB
:10B180009491888784E08F8380E0DF91CF91089548
:10B19000CF93DF93EC018C819D810E945B48E0910D
:10B1A000EB34F091EC3494E0899FE00DF11D112413
:10B1B000458D568D678D70A149875A876B877C872F
:10B1C0008C819D81FC01EE0FFF1FE80FF91FEE0F30
:10B1D000FF1FEE0FFF1FEE0FFF1FEE54FA4E85917B
:10B1E0009491888784E08F8380E0DF91CF910895E8
:10B1F000CF93DF93EC010E94B35D498563EF73E168
:10B20000CE01DF91CF910C943757CF93DF93EC01B0
:10B210008C819D810E945B48833054F48F3F91F470
:10B2200007C0CE010E948C5E80E016C08DE614C07F
:10B2300049855A856B857C854430510561057105CA
:10B24000A8F7EFCF49855A856B857C85433051053A
:10B250006105710558F7E5CFDF91CF91089595E32A
:10B26000899FF0011124E157FC4C6081718182813A
:10B2700093810895CF92DF92EF92FF92CF93DF9365
:10B280006A017B0125E3829FC001112486549D4CF5
:10B29000FC01EB52FF4F4083518362837383EC01C7
:10B2A000C352DF4F20E034E244E759E4C701B6015E
:10B2B0000E947DD89B01AC0160E070E080E89FE3D4
:10B2C0000E94DFD5688379838A839B83DF91CF9146
:10B2D000FF90EF90DF90CF900895CF92DF92EF92A2
:10B2E000FF92CF93DF93EC01C984DA84EB84FC8472
:10B2F00020E034E244E759E4C701B6010E94DBD7FD
:10B30000181664F420E034E244E759E4C701B601BA
:10B310000E94DFD569877A878B879C87CE010E9440
:10B32000C763C984DA84EB84FC848C819D810E948C
:10B330005B4825E3829FC001112486549D4CFC018B
:10B34000EB52FF4FC082D182E282F382EC01C35202
:10B35000DF4F20E034E244E759E4C701B6010E9420
:10B360007DD89B01AC0160E070E080E89FE30E9423
:10B37000DFD5688379838A839B8380E0DF91CF91D7
:10B38000FF90EF90DF90CF900895CF92DF92EF92F1
:10B39000FF92CF93DF93EC01C984DA84EB84FC84C1
:10B3A00020E034E244E759E4C701B6010E94DBD74C
:10B3B000181664F420E034E244E759E4C701B6010A
:10B3C0000E94DFD569877A878B879C87CE010E9490
:10B3D000C76380E0DF91CF91FF90EF90DF90CF9037
:10B3E000089581E08093E53480E00895FC01818533
:10B3F0009285A385B4850197A105B10511F40E943A
:10B40000816B80E008956091E7347091E834809119
:10B41000E9349091EA3408950E94645F80E00E94CC
:10B42000046E80E008950E94645F81E00E94046ED3
:10B4300080E008950E94645F82E00E94046E80E0D4
:10B4400008950E94645F83E00E94046E80E0089586
:10B45000CF93DF93EC01E091EB34F091EC34E55BBA
:10B46000FF4FE081F0E0EE0FFF1FEA5DFB4E6591BC
:10B4700074914FE450E084E69FE30E9412E2AC0135
:10B4800065EF7FE0CE01DF91CF910C94EAC1CF93BD
:10B49000DF93EC01E091EB34F091EC34E55BFF4F8E
:10B4A000E081F0E0EE0FFF1FEA5DFB4E65917491C5
:10B4B0004FE450E084E69FE30E9412E2AC016DEDA0
:10B4C0007FE0CE01DF91CF910C94EAC1CF93DF935F
:10B4D000EC0181EF90E20E9473E3CE010E94285AB2
:10B4E000CE010E94475A6AEC7FE0CE010E9416C24C
:10B4F00061EB7FE0CE010E9460C168E97FE0CE0190
:10B500000E9460C16FE77FE0CE010E9460C166E6E5
:10B510007FE0CE010E9460C16DE47FE0CE010E9419
:10B5200060C164E37FE0CE010E9460C16BE17FE017
:10B53000CE010E9460C162E07FE0CE010E9460C146
:10B5400069EE7EE0CE010E9460C160ED7EE0CE013A
:10B550000E9460C167EB7EE0CE010E9460C16EE98F
:10B560007EE0CE010E9460C165E87EE0CE010E94CF
:10B5700060C16CE67EE0CE010E948EC180E0DF916A
:10B58000CF9108956AEC7FE00C9416C261EB7FE0E6
:10B590000C9460C168E97FE00C9460C16FE77FE0C4
:10B5A0000C9460C166E67FE00C9460C16DE47FE0BE
:10B5B0000C9460C164E37FE00C9460C16BE17FE0B8
:10B5C0000C9460C162E07FE00C9460C169EE7EE0A3
:10B5D0000C9460C160ED7EE00C9460C167EB7EE08E
:10B5E0000C9460C16EE97EE00C9460C165E87EE079
:10B5F0000C9460C16CE67EE00C948EC160EF7DE03F
:10B600000C948EC16FEB7DE00C948EC16AE87DE0F6
:10B610000C948EC16FE47DE00C948EC16BE17DE0F3
:10B620000C948EC1CF93DF93EC01E091EB34F09159
:10B63000EC34E55BFF4FE081F0E0EE0FFF1FEA5DC9
:10B64000FB4E659174914FE450E084E69FE30E94C5
:10B6500012E2AC0167EF7CE0CE01DF91CF910C9458
:10B66000EAC1CF93DF93EC01E091EB34F091EC343D
:10B67000E55BFF4FE081F0E0EE0FFF1FEA5DFB4E60
:10B68000659174914FE450E084E69FE30E9412E2DA
:10B69000AC0166ED7CE0CE01DF91CF910C94EAC164
:10B6A00069EB7CE00C9416C2CF93DF93EC01E09140
:10B6B000EB34F091EC34E55BFF4FE081F0E0EE0F0E
:10B6C000FF1FEA5DFB4E659174914FE450E084E604
:10B6D0009FE30E9412E2AC016AE97CE0CE01DF91B7
:10B6E000CF910C94EAC10F931F93CF93DF93CDB703
:10B6F000DEB7C058D109CDBFDEBF8C01DC01199681
:10B70000EC91F0E0EE0FFF1FED50FC4E659174914F
:10B710004FE450E084E69FE30E9412E29801235F29
:10B720003F4F9F938F93F80181851F928F933F9393
:10B730002F930F5E1F4F1F930F933F932F938EE70F
:10B740009CE09F938F938E010F5F1F4F1F930F936A
:10B750000E94C9E3C8010E943BC1CDBFDEBFC058F3
:10B76000DF4FCDBFDEBFDF91CF911F910F910895C5
:10B7700066E57CE00C94CD486EE27CE00C94CD480C
:10B780006CE07CE00C94CD486AEE7BE00C94CD48F4
:10B7900068EB7BE00C94CD4867E87BE00C94CD48E7
:10B7A0006EE47BE00C94CD486EE27BE00C94CD48D7
:10B7B0006CEE7AE00C949B486AEA7AE00C949B4821
:10B7C00063E87AE00C94CD486DE57AE00C94CD48BE
:10B7D0006CE37AE00C94CD486CE17AE00C94CD48AF
:10B7E0006FEF79E00C94314960EE79E00C943149C7
:10B7F000BC01675F7F4F2091383546E55EE0FC0174
:10B80000848195810C949849BC01675F7F4F21E04A
:10B810004CE35EE0FC01848195810C949849BC0165
:10B82000675F7F4F21E043E25EE0FC018481958108
:10B830000C949849CF93DF93EC014F8345E050E09F
:10B8400041960E946BE2E881F9818781883021F47A
:10B8500086818F5F8E8302C086818E83DF91CF9138
:10B8600008950F931F93CF93DF93EC010C811D81FB
:10B870000E94346508171907C4F48C819D81FC016E
:10B88000EE0FFF1FE80FF91FEE0FFF1FEE0FFF1F58
:10B89000EE0FFF1FE954FA4E25913491CE01F901C4
:10B8A000DF91CF911F910F91199485E1DF91CF9195
:10B8B0001F910F9108950F931F93CF93DF93EC0186
:10B8C0000C811D810E94346508171907C4F48C810E
:10B8D0009D81FC01EE0FFF1FE80FF91FEE0FFF1F08
:10B8E000EE0FFF1FEE0FFF1FEB54FA4E2591349120
:10B8F000CE01F901DF91CF911F910F91199485E14C
:10B90000DF91CF911F910F9108950F931F93CF93C4
:10B91000DF93EC010C811D810E9434650817190723
:10B92000C4F48C819D81FC01EE0FFF1FE80FF91F0D
:10B93000EE0FFF1FEE0FFF1FEE0FFF1FED54FA4E2D
:10B9400025913491CE01F901DF91CF911F910F9193
:10B950001994DF91CF911F910F910895CF93DF93A9
:10B96000EC018C819D810E9447658823C9F08C8100
:10B970009D81FC01EE0FFF1FE80FF91FEE0FFF1F67
:10B98000EE0FFF1FEE0FFF1FEF54FA4EE491E1FFA1
:10B9900005C0CE01DF91CF910C94DC8280E001C024
:10B9A00085E1DF91CF910895AF92BF92CF92DF9260
:10B9B000EF92FF920F931F93CF93DF93EC0181E0FF
:10B9C0000E94234F1C821D8280E090E07E0121E1D5
:10B9D000E20EF11C54E0A52E62E0B62E51C00C819F
:10B9E0001D816801CC0CDD1C9601200F311F220F38
:10B9F000331F220F331F220F331F2F543A4EF901EA
:10BA0000849180FF38C0F601E00FF11FEE0FFF1F99
:10BA1000EE0FFF1FEE0FFF1FE554FA4E6591759173
:10BA20008591949169877A878B879C87F901249106
:10BA300024FD08C00E944CD669877A878B879C8733
:10BA4000BF8201C0AF82B601600F711F660F771F02
:10BA5000660F771F660F771F65557A4E45E050E0F9
:10BA6000C7010E9412E2CE010E94315CCE010E9409
:10BA7000AE5C0C811D810F5F1F4F0C831D83C801BD
:10BA80000E9437658111ABCF81E00E94FBA9DF9155
:10BA9000CF911F910F91FF90EF90DF90CF90BF90CB
:10BAA000AF900C94E0A9CF92DF92EF92FF92CF93E8
:10BAB000DF93EC01C984DA84EB84FC8481E0C8164E
:10BAC000D104E104F10449F0CE01DF91CF91FF9060
:10BAD000EF90DF90CF900C94997ACE010E94D45CC5
:10BAE00082E08F83C986DA86EB86FC8680E0DF9170
:10BAF000CF91FF90EF90DF90CF90089580912C3CF4
:10BB000090912D3C8F3E924111F08AE508958091ED
:10BB10006E3C90916F3C8F3E9241B9F78091FE361A
:10BB20009091FF368F3E924181F78091243A909117
:10BB3000253A8F3E924149F78091263A9091273AD3
:10BB40008F3E924111F780912A3C90912B3C8F3E81
:10BB50009241D9F68091B33F8111D7CF0895FC016E
:10BB6000178289E60895CF93DF93DC0114968D91B7
:10BB70009C911597FC01EE0FFF1FE80FF91FEE0FC8
:10BB8000FF1FEE0FFF1FEE0FFF1FE754FA4EC59188
:10BB9000D491488150E060E070E019964D935D9338
:10BBA0006D937C931C9782E017968C9380E0DF91D5
:10BBB000CF910895CF93DF93DC0114968D919C91E2
:10BBC0001597FC01EE0FFF1FE80FF91FEE0FFF1F87
:10BBD000EE0FFF1FEE0FFF1FE754FA4EC591D491F1
:10BBE0004881598160E070E019964D935D936D93A3
:10BBF0007C931C9782E017968C9380E0DF91CF9125
:10BC00000895CF93DF93DC0114968D919C91159745
:10BC1000FC01EE0FFF1FE80FF91FEE0FFF1FEE0FE5
:10BC2000FF1FEE0FFF1FE754FA4EC591D4914881D4
:10BC300059816A817B8119964D935D936D937C93B5
:10BC40001C9782E017968C9380E0DF91CF91089546
:10BC5000CF93DF93DC0114968D919C911597FC0195
:10BC6000EE0FFF1FE80FF91FEE0FFF1FEE0FFF1F74
:10BC7000EE0FFF1FE754FA4EC591D49148815981C8
:10BC80006A817B8119964D935D936D937C931C978C
:10BC900083E017968C9380E0DF91CF910895CF9346
:10BCA000DF93DC0114968D919C911597FC01EE0FAA
:10BCB000FF1FE80FF91FEE0FFF1FEE0FFF1FEE0F24
:10BCC000FF1FE754FA4EC591D491488159816A818A
:10BCD0007B8119964D935D936D937C931C97FC012A
:10BCE000EE0FFF1FE80FF91FEE0FFF1FEE0FFF1FF4
:10BCF000EE0FFF1FEE54FA4E8591949118968C9397
:10BD0000189784E017968C9380E0DF91CF91089587
:10BD100088E6089580E00895FC0124813581F901C9
:10BD2000EE0FFF1FE20FF31FEE0FFF1FEE0FFF1FBF
:10BD3000EE0FFF1FE754FA4EA591B491FC018185E7
:10BD40008C9380E00895FC0124813581F901EE0F88
:10BD5000FF1FE20FF31FEE0FFF1FEE0FFF1FEE0F8F
:10BD6000FF1FE754FA4EA591B491FC01818592859D
:10BD70008D939C9380E00895CF93DF93FC01248101
:10BD80003581F901EE0FFF1FE20FF31FEE0FFF1FCA
:10BD9000EE0FFF1FEE0FFF1FE754FA4EC591D4912F
:10BDA000FC0181859285A385B48588839983AA83C4
:10BDB000BB8380E0DF91CF910895FC0141855285DE
:10BDC000638574854230510561057105A0F4848155
:10BDD0009581FC01EE0FFF1FE80FF91FEE0FFF1F0B
:10BDE000EE0FFF1FEE0FFF1FE754FA4EA591B4911F
:10BDF0004C9380E008958EE60895FC0141855285BC
:10BE0000638574854330510561057105A0F4848113
:10BE10009581FC01EE0FFF1FE80FF91FEE0FFF1FCA
:10BE2000EE0FFF1FEE0FFF1FE754FA4EA591B491DE
:10BE30004C9380E008958EE60895FC01418552857B
:10BE4000638574854430510561057105A0F48481D2
:10BE50009581FC01EE0FFF1FE80FF91FEE0FFF1F8A
:10BE6000EE0FFF1FEE0FFF1FE754FA4EA591B4919E
:10BE70004C9380E008958EE60895CF93DF93DC0124
:10BE800014968D919C911597FC01EE0FFF1FE80F02
:10BE9000F91FEE0FFF1FEE0FFF1FEE0FFF1FE754FE
:10BEA000FA4EC591D49119964D915D916D917C9109
:10BEB0001C97488359836A837B8383E017968C930E
:10BEC00080E0DF91CF910895CF93DF93DC0114964A
:10BED0008D919C911597FC01EE0FFF1FE80FF91F44
:10BEE000EE0FFF1FEE0FFF1FEE0FFF1FE754FA4E7E
:10BEF000C591D49119964D915D916D917C911C974E
:10BF0000488359836A837B83FC01EE0FFF1FE80F90
:10BF1000F91FEE0FFF1FEE0FFF1FEE0FFF1FEE5476
:10BF2000FA4E8591949118968C93189784E0179601
:10BF30008C9380E0DF91CF9108951F93CF93DF938F
:10BF4000EC018091843C8823D1F01DE10A80DB81E3
:10BF5000C02D209711F480E013C08F818F3FD9F35B
:10BF6000811104C0CE010E945B5C06C0CE010E941C
:10BF7000315CCE010E94AE5C115041F7ECCF85E6FA
:10BF8000DF91CF911F910895CF93DF93EC01BC0116
:10BF90008FEF90E20E944BE2892B41F0BE0182E0DC
:10BFA00091E20E944BE221E0892B09F420E0822FEC
:10BFB000DF91CF91089541E0209100373091013712
:10BFC0002817390709F040E0842F08950F931F9335
:10BFD000CF93DF93CDB7DEB72997CDBFDEBF8B01FF
:10BFE00044E050E0BC01CE0101960E946BE246E0C5
:10BFF00050E0B801CE0101960E945BE20E943465D8
:10C00000181619060CF03FC07981AA81BB811C81EA
:10C010000D812BEA35E140E050E0F90164916713AE
:10C0200027C03196E491E11103C0A11121C029C0BC
:10C03000EA131EC0F9013296E491E11103C0B11177
:10C0400017C01FC0EB1314C0F9013396E491E1113E
:10C0500003C011110DC015C0E1130AC0F9013496D7
:10C06000E491E11103C0011103C00BC0E01749F0D6
:10C070004F5F5F4F285E3F4F4817590709F0CDCFFC
:10C0800002C0CA0102C08FEF9FEF2996CDBFDEBF6D
:10C09000DF91CF911F910F910895CF93DF93FC0112
:10C0A0002189222371F1EC016196BE0186E091E2C3
:10C0B0000E944BE2892B39F1BE018FEF90E20E9482
:10C0C0004BE2892B11F1BE0189E091E20E944BE223
:10C0D000892BD9F0BE018DEE90E20E944BE2892BB4
:10C0E000B1F0BE018CE091E20E944BE2892B79F025
:10C0F000BE0188EE91E20E944BE2892B51F485E06B
:10C1000009C080E007C082E005C083E003C084E08E
:10C1100001C081E0DF91CF910895EF92FF920F93DC
:10C120001F93CF93DF93EC010C811D810E94346536
:10C13000081719070CF075C02C813D818FEF8F8394
:10C1400019861A861B861C861886198A1D861F8AE0
:10C15000188E8E010F5E1F4FB901660F771F620F99
:10C16000731F660F771F660F771F660F771F655562
:10C170007A4EC8010E94F3E17E018DE0E80EF11CC9
:10C180002C813D81B901660F771F620F731F660F07
:10C19000771F660F771F660F771F69557A4EC701A5
:10C1A0000E94F3E18D85882311F18C819D81FC0132
:10C1B000EE0FFF1FE80FF91FEE0FFF1FEE0FFF1F1F
:10C1C000EE0FFF1FEF54FA4EE491E2FF02C01D860E
:10C1D00010C0F70101900020E9F7BF016E197F0937
:10C1E000605F7F4F6C0F7D1FC8010E9454E28C81FD
:10C1F0009D81FC01EE0FFF1FE80FF91FEE0FFF1FDF
:10C20000EE0FFF1FEE0FFF1FEB54FA4E25913491F6
:10C21000CE01F901DF91CF911F910F91FF90EF9027
:10C220001994DF91CF911F910F91FF90EF90089596
:10C230008F929F92AF92BF92CF92DF92EF92FF9236
:10C240000F931F93CF93DF9300D01F92CDB7DEB72C
:10C250006C015C0181E1A80EB11C88E0F6018783C6
:10C2600067EAE62E65E1F62E00E010E01DC0B7019A
:10C27000CE0101960E94F3E1BE016F5F7F4FC501C1
:10C280000E944BE2892B59F44601F9E18F0E911C73
:10C29000F601058F168FC4010E948D6064010F5F47
:10C2A0001F4FF8E1EF0EF11CC8010E9437658111A4
:10C2B000DECF2496CDBFDEBFDF91CF911F910F91CE
:10C2C000FF90EF90DF90CF90BF90AF909F908F90B6
:10C2D0000895FC018FEF87831482158211861286E0
:10C2E000138614861086118A1586178A108ECF0140
:10C2F0000895CF93DF931092283A1092293AFC01C7
:10C300002081222311F032E001C031E0ABEEB6E330
:10C31000E4E0F7E32FEFA083B18379965B96ED938A
:10C32000FC935C975D961D921C925E97EF0163975C
:10C33000388322961882219728832A961882599644
:10C340004AE3E432F40739F710920D3A10920E3AAC
:10C35000109204371092053710920A37FC012081A1
:10C36000222359F021E02093233728E0209324371B
:10C37000BC018EE297E30E9454E28DE197E3DF91E6
:10C38000CF910895EF92FF920F931F93CF93DF9376
:10C3900080E090E00E947961EC018FEE92E1809361
:10C3A0002C3C90932D3C80936E3C90936F3C8093FB
:10C3B000FE369093FF368093243A9093253A8093EB
:10C3C000263A9093273A80932A3C90932B3C81E025
:10C3D0000E94234F1C821D82CE010E94B3822091B5
:10C3E000763C3091773C4091783C5091793C69851E
:10C3F0007A858B859C850E942FD49F772CEA35EC1B
:10C4000047E257E30E94DBD7181624F4CE010E94BE
:10C41000D45C58C00E94E5A91C821D8280E090E097
:10C420008E010F5E1F4F42E0E42E54E0F52E44C013
:10C430006C817D81CB01880F991FFC01E60FF71FEE
:10C44000EE0FFF1FEE0FFF1FEE0FFF1FEF54FA4E10
:10C45000E491E0FF2CC0680F791F660F771F660F0D
:10C46000771F660F771F65557A4E45E050E0C8018B
:10C470000E9412E2CE010E94B3828C819D81FC0158
:10C48000EE0FFF1FE80FF91FEE0FFF1FEE0FFF1F4C
:10C49000EE0FFF1FEF54FA4EE491E4FF02C0FF825B
:10C4A00001C0EF82CE010E94315C6C817D816F5FA3
:10C4B0007F4F6C837D83CB010E9437658111B8CF9C
:10C4C0000E94FBA960E171E287E493E20E94E65FCB
:10C4D000809300379093013764E171E287E493E23F
:10C4E0000E94E65F8093023790930337DF91CF91EC
:10C4F0001F910F91FF90EF900895CF93DF9340E04D
:10C50000E4E0F7E3878187FF26C00280F381E02D16
:10C510004F5F4032B9F71CC0ED01CE1BDF0BC20FDD
:10C52000D31F5F81599657FD07C0EC01AA83BB83D7
:10C530008D939C931197CD014F5F403269F7108224
:10C540001182DC0112961D921C921397CF010AC032
:10C5500080E090E007C0DF01582FCF019F01275EE8
:10C560003F4FE1CFDF91CF910895EF92FF920F936C
:10C570001F93CF93DF938C012091283A3091293A71
:10C58000EB0109900020E9F72197C61BD70BAE01FC
:10C59000420F531F41305240D8F4F901E65DF54C8B
:10C5A0007F01AE014F5F5F4FCF010E942CE24091AF
:10C5B000283A5091293A4F5F5F4F4C0F5D1F4093CF
:10C5C000283A5093293AF801E78AF08E80E001C0BA
:10C5D0008DE0DF91CF911F910F91FF90EF90089523
:10C5E000CF93DF932EE1CDE1D7E33F813F3F59F079
:10C5F0000A80DB81C02D209719F480E090E010C004
:10C60000215099F7FACFBC0187E493E20E94E65FDC
:10C610008C839D83019689F3CE010E948D60CE01AB
:10C62000DF91CF9108950F931F93CF93DF938B01E9
:10C630002EE1CDE1D7E33F813F3F59F00A80DB8116
:10C64000C02D209719F480E090E018C0215099F790
:10C65000FACF45E0BC01CE010E941A5CB801CE01C0
:10C660000E94B5628111EFCFBE016F5E7F4F87E4FC
:10C6700093E20E94E65F8C839D83CE01DF91CF9190
:10C680001F910F9108952091843C213021F4209135
:10C69000603F213029F4BC018DEE90E20C941363CD
:10C6A00080E090E008959091843C913019F4642FDB
:10C6B0000C9460810C9433C1CF93DF93EC01809193
:10C6C000773281110BC00E946ED2482F50E060E09B
:10C6D00070E049875A876B877C870AC00E947CC9B3
:10C6E000482F50E060E070E049875A876B877C876D
:10C6F00082E08F8380E0DF91CF9108950F931F93A5
:10C70000CF93DF93CDB7DEB7C058D109CDBFDEBF21
:10C71000DC011996EC918FEF8E0F863030F088E4B3
:10C7200091E20E9443638EE629C0E093723281E079
:10C7300080937332F0E0EE0FFF1FEE58FA4E6591D2
:10C7400074914FE450E084E69FE30E9412E29F93CD
:10C750008F9389E394E19F938F938E010F5F1F4F17
:10C760001F930F930E94C9E3C8010E9443630F9077
:10C770000F900F900F900F900F9080E0C058DF4FF8
:10C78000CDBFDEBFDF91CF911F910F9108950F9321
:10C790001F93CF93DF93EC018DEE94E30E94D34A75
:10C7A000882329F009851A858B859C8511C023E390
:10C7B00033E34BEC51E469857A858B859C850E9437
:10C7C0007DD88B01AB01BC0149875A876B877C8779
:10C7D0002C813D81F901EE0FFF1FE20FF31FEE0FD9
:10C7E000FF1FEE0FFF1FEE0FFF1FE754FA4EA5913C
:10C7F000B491A801BC014D935D936D937C93139705
:10C80000F901EE0FFF1FE20FF31FEE0FFF1FEE0FF8
:10C81000FF1FEE0FFF1FEE54FA4E8591949188870B
:10C8200084E08F8380E0DF91CF911F910F91089575
:10C8300063E475E10C9416C26FE175E10C9416C2C5
:10C8400063EE74E10C9416C26FEA74E10C9416C2A4
:10C8500062E674E10C9416C21F93CF93DF93EC0150
:10C8600010E08881882311F180E090E00E947961D6
:10C8700045E050E0BE018EE297E30E946BE26EE27B
:10C8800077E387E493E20E94E65F809321379093F9
:10C8900022378DE197E30E948D6042E063E080E003
:10C8A0000E9453631F5F26961D31D9F684E0DF9105
:10C8B000CF911F910895CF93DF93CDB7DEB7EC975B
:10C8C000CDBFDEBF8CE3E8E1F0E2DE01119601901E
:10C8D0000D928A95E1F7CE0101960E942C64EC96A8
:10C8E000CDBFDEBFDF91CF910895CF93DF93CDB75A
:10C8F000DEB7AA97CDBFDEBF8AE2E4E5F0E2DE0153
:10C90000119601900D928A95E1F7CE0101960E9451
:10C910002C64AA96CDBFDEBFDF91CF910895CF934F
:10C92000DF93CDB7DEB76E97CDBFDEBF8EE1EEE70A
:10C93000F0E2DE01119601900D928A95E1F7CE01A9
:10C9400001960E942C646E96CDBFDEBFDF91CF9121
:10C950000895CF93DF93EC0143E759E763E770E075
:10C96000498B5A8B6B8B7C8B0E94186142E063E091
:10C9700080E00E945363CE010E948F64CE010E942A
:10C98000756420E731E340E0298B3A8B4B8BCE0175
:10C990000E94186142E063E080E00E945363CE0190
:10C9A000DF91CF910C945B64FC0181859285A38516
:10C9B000B48583309105A105B105A0F4809376324A
:10C9C000892B8A2B8B2B39F064E070E080E00E9489
:10C9D00055C780E0089568E070E080E00E9455C788
:10C9E00080E008958EE60895FC0181859285A385F7
:10C9F000B48582309105A105B105A0F4809375320C
:10CA0000892B8A2B8B2B39F060E170E080E00E944B
:10CA100055C780E0089560E270E080E00E9455C74D
:10CA200080E008958EE60895FC0181859285A385B6
:10CA3000B48582309105A105B105A0F480937432CC
:10CA4000892B8A2B8B2B39F060E470E080E00E9408
:10CA500055C780E0089560E870E080E00E9455C707
:10CA600080E008958EE6089582E991E0089521E03E
:10CA70008934914008F020E0822F08959C012556CA
:10CA8000314081E02932310508F080E0089521E04D
:10CA90008636914008F020E0822F0895CF92DF92F1
:10CAA000EF92FF92CF93DF93EC01C984DA84EB8499
:10CAB000FC84A7019601C701B6010E949ED981118D
:10CAC0003CC0E894F7F82FEF3FEF4FE75FE7C7016F
:10CAD000B6010E949ED981110AC02FEF3FEF4FE7A8
:10CAE0005FE7C701B6010E94D8D5181634F18C81D2
:10CAF0009D81FC01EE0FFF1FE80FF91FEE0FFF1FD6
:10CB0000EE0FFF1FEE0FFF1FEF54FA4EE491E3FF0D
:10CB100014C08DEE94E30E94D34A81110EC025E823
:10CB200032E441E25DE369857A858B859C850E94CC
:10CB30007DD869877A878B879C87DF91CF91FF901B
:10CB4000EF90DF90CF90089580917332882349F061
:10CB5000109273326091723280E00E945DC780E073
:10CB6000089583E00895CF93DF93E091A63CF09180
:10CB7000A73C04C0E093A63CF093A73CEF01819151
:10CB8000982F9D7F9032B1F38930A1F34FE750E0A9
:10CB9000BE018AEA9EE30E946BE21092A23C1092D0
:10CBA000A33C1092A43C1092A53C6881611105C081
:10CBB0008091843C81116FC039C0613221F4DF91D2
:10CBC000CF910C94CA55653221F4DF91CF910C942A
:10CBD000CE556E3721F4DF91CF910C94D2556F333F
:10CBE00079F4FE0101900020E9F73197EC1BFD0B71
:10CBF000329780F02196C093A63CD093A73C4BC0BF
:10CC00006B3741F481E08093843CCE01DF91CF917A
:10CC10000C94797E70E088E791E20E9440E2892BD3
:10CC200059F01092843CCE010E9427BF6AEA7EE34D
:10CC3000DF91CF910C948DC08091843C811109C00B
:10CC4000CE010E94D0706AEA7EE3DF91CF910C940E
:10CC50008DC080E090E00E947961EC0127E633E628
:10CC600040E0298B3A8B4B8B6091A63C7091A73C9E
:10CC70000E94B56285E08F838091A63C9091A73C8D
:10CC80000E94D07042E060E00E94536380E0DF9138
:10CC9000CF910C944CACDF91CF910895FF920F93FC
:10CCA0001F93CF93DF931F921F92CDB7DEB7F82E5D
:10CCB000E0E7FCE32CEB32E0DF01C9011D920197B4
:10CCC000E9F72FEE32E12083318320932A3F30931E
:10CCD0002B3F02E518E32CED33E40093763C1093F0
:10CCE000773C2093783C3093793C0CEE11E528E7B3
:10CCF0003FE300937A3C10937B3C20937C3C309341
:10CD00007D3C81E080937E3C83E08093853C8F2D49
:10CD10004A8369830E946DC76981862F0E9478C704
:10CD20004A81842F0E9483C7F0927132F0926F3251
:10CD30000F900F90DF91CF911F910F91FF90089569
:10CD4000CF93DF931F921F92CDB7DEB780E6F82E08
:10CD500001E010E00E9457798230E1F30E945E7991
:10CD60008230C1F30E94B24A863009F0D9C00E94D5
:10CD700050C580908B3C90908C3CA0908D3CB090A6
:10CD80008E3C86169706A806B90620F70E9450C565
:10CD90006C597F4F8F4F9F4F60938B3C70938C3CAF
:10CDA00080938D3C90938E3C0E94CD78D3CF0E948F
:10CDB0000DBE882329F08CEC0E94FC4E823051F28B
:10CDC0000E942356823031F20E944F9F823011F22E
:10CDD0000E947E5D8093B43F81112EC08091703C93
:10CDE0009091713C8F3E924109F0AAC080912A3FF8
:10CDF00090912B3F8F3E924109F0A2C097C00E94B4
:10CE000049838093B43F811117C00E947CB4809302
:10CE1000B43F811111C00E949B708093B43F811177
:10CE20000BC00E947CC68093B43F811105C00E9454
:10CE300074B5823031F48ECF0E94FC4E8230B9F747
:10CE400089CF0E947EAC823009F484CF0E94CBADA2
:10CE5000823009F47FCF0E9487AE823009F47ACF06
:10CE600009831A8368EA7CE3CE0101960E9492C787
:10CE70008093A63C9093A73C8F3F2FEF920739F405
:10CE800083E10E94E54E823009F464CF04C0892B0F
:10CE900011F00E94B3650E94AE8D823009F45ACF22
:10CEA0000E94D06B823009F455CF0E948F6E823081
:10CEB00009F450CF0E947670823009F449CF0E9465
:10CEC000814C823009F444CF0E94FE838430F0F517
:10CED0003FCF8091853C843038F484E08093853C5A
:10CEE0000E94CE550E94EDA983E090E089839A8349
:10CEF00068EA7CE3CE0101960E9492C78093A63C2B
:10CF00009093A73C8F3F2FEF920721F482E10E947C
:10CF1000E54E1ECF892B09F41BCF0E94B36518CFB5
:10CF20000E94B24A823009F44BCF41CF1092B43FF5
:10CF30000E94AF4E8093B43F882309F460CF7CCF2A
:10CF4000F092B43F80E60E94FC4E78CF8091E429B5
:10CF50009091E5290E94E2D0682F70E080E090E097
:10CF60000E947AD620E030E048E451E40E94DBD70A
:10CF700087FFEECE0E94A465823009F0AACFE8CEEA
:10CF80008091713280936F32089580936F3208954B
:10CF9000809370320895CF93C82F80919323882374
:10CFA00079F040E050E0BA018C2F0E947450EC2FD1
:10CFB000FF27E7FDF095EE53FB4C81E080830AC02C
:10CFC0006C2F83EB98E50E94F84BAB01BC018C2FD2
:10CFD0000E9474504091BA235091BB236091BC23AE
:10CFE0007091BD238C2F0E943A5986E999E680936F
:10CFF00094239093952382E0CF910895CF92DF926E
:10D00000EF92FF920F931F93CF93DF93CDB7DEB7CD
:10D01000E097CDBFDEBF98E17E01A9E1EA0EF11CE9
:10D02000F701A92F1192AA95E9F7FE0131966F0138
:10D0300011929A95E9F7F60194E08902E00DF11D4D
:10D040001124408F518F628F738F80E090E0A0E8B1
:10D05000BFE380839183A283B38300932A35109327
:10D060002B3520932C3530932D350E9481840E94DE
:10D07000D255B601C7010E949C538093B43F8111E1
:10D0800001C082E0E096CDBFDEBFDF91CF911F915E
:10D090000F91FF90EF90DF90CF9008950F931F9323
:10D0A000E0918D23FF27E7FDF095E956FD4C938134
:10D0B000913099F400919E2310919F232091A023F9
:10D0C0003091A1234091A6235091A7236091A823DA
:10D0D0007091A9230E94FE671DC0E0918E23FF2757
:10D0E000E7FDF095E956FD4C9381913099F400915C
:10D0F0009E2310919F232091A0233091A123409142
:10D10000A6235091A7236091A8237091A92370585A
:10D110000E94FE6784E998E6809394239093952378
:10D1200082E01F910F9108950F931F93CF93C82F03
:10D1300085E3C802F0011124ED56FC4C4081518179
:10D14000628173818C2F0E943A5900919E23109125
:10D150009F232091A0233091A12340919A235091A5
:10D160009B2360919C2370919D238C2F0E94FE67CE
:10D1700083E299E6809394239093952382E0CF9164
:10D180001F910F9108950F931F9300919E2310916B
:10D190009F232091A0233091A1234091AA23509155
:10D1A000AB236091AC237091AD230E94FE678BECA2
:10D1B00097E6809394239093952382E01F910F919B
:10D1C00008950E9481848091B3230E94DD4F809155
:10D1D000B2230E94234F8091B4230E94274F809155
:10D1E000B5230E9488538091B6239091B723A091D4
:10D1F000B823B091B92380932A3590932B35A0930F
:10D200002C35B0932D3564E08DEE94E30E94F04A06
:10D210000E947F561092BE3480E00895CF93C82FAD
:10D220004091BA235091BB236091BC237091BD23E0
:10D230000E943A598C2F0E94E16880E00E944CAC19
:10D2400080EFCF9108950F931F93E0918D23FF27D7
:10D25000E7FDF095E956FD4C9381913039F08EE071
:10D2600099E6809394239093952318C00091A2236C
:10D270001091A3232091A4233091A5234091A623AC
:10D280005091A7236091A8237091A9230E94FE6763
:10D2900083EC98E6809394239093952382E01F91EA
:10D2A0000F910895FF920F931F93CF93DF93CDB704
:10D2B000DEB7C058D109CDBFDEBFF82E87E493E2B8
:10D2C0000E9479618EEFF81205C08DE791E20E940D
:10D2D000436319C08F2D0E9414571F928F9327E527
:10D2E0003BE33F932F938E010F5F1F4F1F930F93CD
:10D2F0000E94C9E3C8010E9443630F900F900F90F2
:10D300000F900F900F9042E062E080EF0E94536315
:10D310008F2D0E94E16880EFC058DF4FCDBFDEBF88
:10D32000DF91CF911F910F91FF9008954F925F92DF
:10D330006F927F929F92AF92BF92CF92DF92EF92C5
:10D34000FF920F931F93CF93DF938F3F09F045C058
:10D350002CEA35EC47E257E360912536709126368A
:10D3600080912736909128360E94DBD718160CF44E
:10D3700069C12CEA35EC47E257E360911D367091A4
:10D380001E3680911F36909120360E94DBD71816EA
:10D390000CF45DC12CEA35EC47E257E3609121368D
:10D3A0007091223680912336909124360E94DBD7EB
:10D3B00018160CF455C12CEA35EC47E257E360919E
:10D3C000293670912A3680912B3690912C360E9406
:10D3D000DBD718160CF43FC171C18230A1F52CEADD
:10D3E00035EC47E257E360911D3670911E3680910F
:10D3F0001F36909120360E94DBD718160CF427C1F7
:10D400002CEA35EC47E257E36091213670912236E1
:10D4100080912336909124360E94DBD718160CF4A5
:10D420001FC12CEA35EC47E257E360912936709131
:10D430002A3680912B3690912C360E94DBD7181615
:10D440000CF409C131C18823D9F2813051F32CC1C8
:10D450007E018DEEE80EF11CF70180819181A281A1
:10D46000B381BC01CD019F772CEA35EC47E257E34D
:10D470000E94D8D587FD46C06E01F1EFCF0ED11CBA
:10D48000F601408051806280738020E030E0A90185
:10D49000C301B2010E94D8D587FD34C0FE01EF520E
:10D4A000FF4F2081318142815381349760817181A6
:10D4B000828193810E942FD49B01AC015F77C301CD
:10D4C000B2010E9430D42B013C019F772CEA35EC4D
:10D4D00047E257E30E94D8D587FD14C0AB2CAA0CB5
:10D4E0008A2D0E9407BE80938B23992493949A0CD3
:10D4F000892D0E9407BE80938C2320918B23822745
:10D5000080FD02C08B2DDBC0B0928A23F8018081A0
:10D510009181A281B381BF7780939E2390939F23B3
:10D52000A093A023B093A123F70140815181628190
:10D5300073817F774093A2235093A3236093A42306
:10D540007093A52320FF2DC0A0928D2390928E234F
:10D5500077FA709477F8709440929A2350929B23B4
:10D5600060929C2370929D23F60180819181A2811B
:10D57000B3818093A6239093A723A093A823B0936D
:10D58000A923CB50DF4F88819981AA81BB818093E9
:10D59000AA239093AB23A093AC23B093AD238A2D01
:10D5A0002AC090928D23A0928E2340929A2350926B
:10D5B0009B2360929C2370929D23F6018081918130
:10D5C000A281B381B0588093A6239093A723A09300
:10D5D000A823B093A923CB50DF4F88819981AA81DA
:10D5E000BB81B0588093AA239093AB23A093AC2324
:10D5F000B093AD23892D0E9407BE8D7F813039F015
:10D6000086E999E6809394239093952369C080914D
:10D610008E230E9407BE811103C08FEF80938E235B
:10D620008B2D0E942F596093BA237093BB23809354
:10D63000BC239093BD238EE498E68093942390932B
:10D6400095234EC082E090E032E0B32E0DC080E022
:10D6500090E0B12C09C083E090E023E0B22E04C03A
:10D6600081E090E0BB24B394FC01EE53FB4C1082AC
:10D6700025E3289FE001299FD00D1124C654DD4CDD
:10D680008E0107511F4FF80180819181A281B381E2
:10D69000BC01CD019F772CEA35EC47E257E30E94AD
:10D6A000D8D587FFD5CE2ECF81E08093C13481EECF
:10D6B00098E6809394239093952312C08EEFDF9188
:10D6C000CF911F910F91FF90EF90DF90CF90BF907F
:10D6D000AF909F907F906F905F904F900C945269A5
:10D6E00082E0DF91CF911F910F91FF90EF90DF903B
:10D6F000CF90BF90AF909F907F906F905F904F9032
:10D700000895CF93DF93CBEED4E3888199810E9473
:10D71000D34A8093B223888199810E94CE4A809314
:10D72000B323888199810E94DD4A8093B423888144
:10D7300099810E94E24A8093B523888199810E9451
:10D74000E94A6093B6237093B7238093B8239093EC
:10D75000B92381E00E94234F81E00E94274F80E09F
:10D760000E94DD4F81E00E94885381E080939323E3
:10D770008FEF80938A2386E999E680939423909390
:10D78000952383E08093BE341092C13480E0DF9112
:10D79000CF9108950E94816B1092932380E00895A9
:10D7A0008091BE34833059F40E94E74A813049F0B9
:10D7B000E0919423F091952380918A23199483E03A
:10D7C000089582E008958BEE9BE68093CF2390939B
:10D7D000D02382E008952F923F924F925F926F92F2
:10D7E0007F928F929F92AF92BF92CF92DF92EF92F1
:10D7F000FF920F931F93CF93DF93CDB7DEB7CA5439
:10D80000D109CDBFDEBF98E19E01275E3F4F29AB16
:10D810003AABD901E92F1D92EA95E9F72851310970
:10D820001901D9011D929A95E9F724E08202F001CD
:10D8300011242B96EEAFFFAF2B97E20DF31D80E086
:10D8400090E0A0E8BFE380839183A283B383C0907C
:10D85000C723D090C823E090C923F090CA234090FA
:10D86000C3235090C4236090C5237090C62380903A
:10D87000BF239090C023A090C123B090C223A501E4
:10D880009401C301B2010E94D8D518165CF080E063
:10D8900090E0A0E8BFE329968CAF9DAFAEAFBFAFDD
:10D8A00029970AC080E090E0A0E8BFEB29968CAFF2
:10D8B0009DAFAEAFBFAF2997A3019201C501B401DF
:10D8C0000E942FD40E9447D69B0177FF04C02227D5
:10D8D0003327261B370BB901882777FD8095982FB2
:10D8E0000E947AD625966CAF7DAF8EAF9FAF2597FD
:10D8F000C0922A35D0922B35E0922C35F0922D35FE
:10D900000E9481840E94D25520E030E040E050E443
:10D9100025966CAD7DAD8EAD9FAD25970E94DBD772
:10D9200018166CF08091CB239091CC23A091CD233D
:10D93000B091CE238BAF9CAFADAFBEAFDBC02AE0C2
:10D9400037ED43E25CE325966CAD7DAD8EAD9FADCA
:10D9500025970E94DBD718162CF709E110E08AE022
:10D96000882E87ED982E83E2A82E8CE3B82E412CCA
:10D97000512C32012B96AEADBFAD2B97A20DB31D2E
:10D9800058962196AEAFBFAF21974BAA5CAA6DAA5D
:10D990007EAA8FAA98AEA9AEBAAE29962CAD3DAD9F
:10D9A0004EAD5FAD29976FA978AD89AD9AAD0E9454
:10D9B0007DD89B01AC016091C3237091C4238091F9
:10D9C000C5239091C6230E9430D42196EEADFFADC1
:10D9D00021976083718382839383C0922A35D0928A
:10D9E0002B35E0922C35F0922D35B101CE014996C0
:10D9F0000E949C538093B43F8111AAC020E030E084
:10DA000040E85FE36BA97CA98DA99EA90E9430D450
:10DA10006BAB7CAB8DAB9EAB20E030E048EC51E4CF
:10DA20000E94DFD59B01AC0160E070E080E291E4F0
:10DA30000E94E0D82B013C018091CB239091CC2314
:10DA4000A091CD23B091CE238BAF9CAFADAFBEAF35
:10DA5000C090C723D090C823E090C923F090CA2378
:10DA6000A7019601BC01CD010E942FD44B015C019E
:10DA700020E030E040E251E4C301B2010E94DFD572
:10DA80009B01AC01C501B4010E947DD89B01AC0192
:10DA9000C701B6010E9430D46B017C012BA93CA9BF
:10DAA0004DA95EA9CA01B9010E9430D420E030E03E
:10DAB00048EC51E40E94DFD59B01AC016FA978AD21
:10DAC00089AD9AAD0E9430D46FAB78AF89AF9AAF71
:10DAD0009B01AC0125966CAD7DAD8EAD9FAD2597BC
:10DAE0000E94DBD7181634F40150110901151105F5
:10DAF00009F053CF8BAD9CADADADBEAD80932A3553
:10DB000090932B35A0932C35B0932D352B96EEADFD
:10DB1000FFAD2B97E20DF31D8091BF239091C023A1
:10DB2000A091C123B091C223808F918FA28FB38F18
:10DB3000B101CE0149960E949C538093B43F81115C
:10DB400007C08FEB9DE68093CF239093D02382E094
:10DB5000C65BDF4FCDBFDEBFDF91CF911F910F912D
:10DB6000FF90EF90DF90CF90BF90AF909F908F90FD
:10DB70007F906F905F904F903F902F900895CF933C
:10DB8000DF931F92CDB7DEB789830E9481844091D5
:10DB9000D9235091DA236091DB237091DC238981B2
:10DBA0000E943A598091D6230E94DD4F8091D5235F
:10DBB0000E94234F8091D7230E94274F8091D82322
:10DBC0000E9488538091D1239091D223A091D32396
:10DBD000B091D42380932A3590932B35A0932C3584
:10DBE000B0932D3564E08DEE94E30E94F04A0E94DC
:10DBF0007F561092BE3489EA91E20E9473E380E07E
:10DC00000F90DF91CF9108950F931F93CF93C82F5B
:10DC10000BEE14E3F801808191810E94D34A809336
:10DC2000D523F801808191810E94CE4A8093D6232A
:10DC3000F801808191810E94DD4A8093D723F80109
:10DC4000808191810E94E24A8093D823F8018081EB
:10DC500091810E94E94A6093D1237093D2238093EB
:10DC6000D3239093D4238C2F0E942F596093D923D0
:10DC70007093DA238093DB239093DC2381E00E946E
:10DC8000234F80E00E94274F80E00E94DD4F81E01B
:10DC90000E94885340E050E060E271E44093C72363
:10DCA0005093C8236093C9237093CA2385E3C89F08
:10DCB000F0011124ED57FC4C408151816281738148
:10DCC0004093CB235093CC236093CD237093CE23EA
:10DCD0006C2F83EB98E50E94E54B6093C323709310
:10DCE000C4238093C5239093C6230E94035A609354
:10DCF000BF237093C0238093C1239093C223C0930A
:10DD0000BE2383EE9BE68093CF239093D02384E0C1
:10DD10008093BE3480E0CF911F910F910895809140
:10DD2000BE34843059F40E94E74A813049F0E091D2
:10DD3000CF23F091D0238091BE23199483E00895DE
:10DD400082E00895E091DF23F0E0E956FD4C838105
:10DD5000882341F08DEB9EE68093DD239093DE23B4
:10DD600082E008956CE274E284E194E20E949C53A4
:10DD70008093B43F882371F308951F93CF93DF936B
:10DD8000E091DF23F0E0E956FD4C81E09381913092
:10DD900009F080E08093C834C9ECD4E310E0812F0F
:10DDA0000E946F98AB01BC01812F0E947450612FBB
:10DDB0008091EB349091EC340E94E54B6993799318
:10DDC000899399931F5F163051F783EB91E20E947C
:10DDD000797E89E29FE68093DD239093DE2382E0C3
:10DDE000DF91CF911F9108951F93CF93DF930E94EE
:10DDF00081848091E02380939732E091DF23F0E0EB
:10DE00008091E123E956FD4C83870E9424BEC4EE35
:10DE1000D3E210E04991599169917991812F0E9443
:10DE20003A591F5F1630B1F78091E3230E94DD4F0E
:10DE30008091E2230E94274F64E08DEE94E30E94DC
:10DE4000F04A0E947F561092BE34DF91CF911F910D
:10DE500008950E94F46E80E008950F931F93CF936E
:10DE6000DF93CDB7DEB7C058D109CDBFDEBF182FC5
:10DE700087E493E20E9479611E3F29F480EC91E2ED
:10DE80000E94436319C0812F0E9414571F928F93E1
:10DE900085E89BE39F938F938E010F5F1F4F1F9326
:10DEA0000F930E94C9E3C8010E9443630F900F9033
:10DEB0000F900F900F900F9042E062E08AEF0E9467
:10DEC00053630E94F46E8AEFC058DF4FCDBFDEBFB0
:10DED000DF91CF911F910F910895FF920F931F93A0
:10DEE000CF93DF931092C83482E08093BE3404EE67
:10DEF00013E2C3E9D3E3F12C8F2D0E942F59F801CF
:10DF000061937193819391938F01488159816A81C3
:10DF10007B818F2D0E943A596F2D8091EB34909127
:10DF2000EC340E94E54BF801648B758B868B978BE4
:10DF3000F394E596F6E0FF12DFCF64E174E28CEF34
:10DF400093E20E9453C22AE43CE042E85EE30E946E
:10DF5000D8D587FF03C08EEF0E942D6FC8E0D4E2B2
:10DF600013E069917991899199912C893D894E8924
:10DF70005F890E942FD49F772CEA35EC47E257E364
:10DF80000E94DBD718161CF4812F0E942D6F1F5F93
:10DF9000163039F784E08093DF238091A632809396
:10DFA000E12381E08093A632809197328093E02331
:10DFB000109297320E9424BE8091EB349091EC3401
:10DFC0000E94CE4A8093E3238091EB349091EC340D
:10DFD0000E94DD4A8093E22380E00E94274F80E088
:10DFE0000E94DD4F80E00E9456B082EA9EE6809358
:10DFF000DD239093DE2382E0DF91CF911F910F917B
:10E00000FF9008950F931F93CF93DF938C01EB0143
:10E0100080913635882399F080912A3590912B355F
:10E02000A0912C35B0912D35BC01CD019F772CEA04
:10E0300035EC47E257E30E94D8D587FD4FC0888171
:10E040009981AA81BB81BC01CD019F772CEA35EC77
:10E0500047E257E30E94DBD71816F4F48C819D81C8
:10E06000AE81BF81BC01CD019F772CEA35EC47E240
:10E0700057E30E94DBD718167CF488859985AA851A
:10E08000BB85BC01CD019F772CEA35EC47E257E315
:10E090000E94DBD7181624F188E1F801A4E1B4E26C
:10E0A00001900D928A95E1F788E1FE01ACE2B4E2BD
:10E0B00001900D928A95E1F788E1E9ECF4E3DF0144
:10E0C0001D928A95E9F782E08093C8348DE69FE639
:10E0D0008093DD239093DE2380E003C08EE801C0AF
:10E0E00086E8DF91CF911F910F9108958091BE3402
:10E0F000823021F08091C834823049F40E94E74A8E
:10E10000813039F0E091DD23F091DE23199483E032
:10E11000089582E00895ECE2FFE380E2DF011D92C2
:10E120008A95E9F78FEE92E180934A3F90934B3FB7
:10E1300080839183089580914A3F90914B3F8F3E19
:10E14000924111F08CE5089580912C3F90912D3FE4
:10E150008F3E9241B9F780E00895CF93DF93C82FA7
:10E16000CB01BA010E942CD927E0C29FE001112403
:10E17000C45DD04C0E9447D66D837E838F83988781
:10E18000DF91CF91089597E0899FF0011124E45D1C
:10E19000F04C65817681878190850E947AD60895BA
:10E1A0002F923F924F925F926F927F928F929F92A7
:10E1B000AF92BF92CF92DF92EF92FF920F931F9395
:10E1C000CF93DF93CDB7DEB72797CDBFDEBF8C01EE
:10E1D0001B828091BD34823009F440C7D801BC90C5
:10E1E000B11069C780E06E01B3E0CB0ED11C3DC019
:10E1F000F6018081811108C0B72CD7011C926E01F5
:10E20000B3E0CB0ED11C54C7883239F4B72CF701D8
:10E210001082FFEFCF1ADF0A4BC78B33B9F3A82E5A
:10E22000B12CC5010E94C7E1892B39F4B5018AEEF2
:10E2300091E20E9440E2892B51F047018FEF881A4A
:10E24000980AC5010E94EBE1D7018C937401BFEFDE
:10E25000CB1ADB0AF70180818111CACFB72CD80114
:10E260008C916E01B3E0CB0ED11CF8011CC08E3234
:10E27000E1F090E0C0970A97A0F08181803391F49B
:10E28000228130E0205331092A30310558F4DF0172
:10E29000119611968C9111978D938111FACF8081EF
:10E2A00002C0818131968111E2CFF601A080A110D8
:10E2B00007C068C0D6011196AC90BFEFCB1ADB0A3D
:10E2C00076018A2C912CC4010E94DBE1892B91F705
:10E2D000EBE7AE122FC0D60111968C9190E00E9410
:10E2E000E3E18437910531F5F601828190E00E94E7
:10E2F000E3E189369105F1F4D60113968C9190E013
:10E300000E94E3E184369105A9F4BE016F5F7F4F5F
:10E31000C60105960E9443DE0E944CD66093A23C43
:10E320007093A33C8093A43C9093A53CF601A080FD
:10E330008A2C912CC4010E94E3E18D369105A1F451
:10E34000D60111968C9190E00E94E3E1833791050C
:10E3500059F4F601828190E00E94E3E1873691054D
:10E3600019F4F601339602C0FE013396AA2061F03B
:10E370008A2DD701893209F41C9211968C91811152
:10E38000F9CF02C0FE0133968FE2B81609F468C6D1
:10E390008081882319F0CF010E94C55580E1ECE40B
:10E3A000FFE3DF011D928A95E9F78BE5E6E1F6E3ED
:10E3B000DF01982F1D929A95E9F7EBEBF5E3DF016A
:10E3C0001D928A95E9F78DEE94E30E94CB4A8093E3
:10E3D000BC35812C912C80E8A82E8FE3B82E5524D3
:10E3E000539492E0492E24E0322E23C4C701B60193
:10E3F0000E944CD6862F90E08F35910508F034C6E8
:10E40000FC01EC50FF4F0C9423DE1092BC3550926F
:10E41000173680914D3F8F5F80934D3F0AC45092D5
:10E42000BC355092173680914D3F8F5F80934D3FA2
:10E4300000C44092BC355092173680914D3F8F5F9B
:10E4400080934D3FF6C383E08093BC3550921736DE
:10E4500080914D3F8F5F80934D3FEBC38DE0809364
:10E46000BB3550921636E5C388E0B2C01092EB354A
:10E470005092463680914E3F8F5F80934E3FD9C376
:10E480005092EB355092463680914E3F8F5F80938D
:10E490004E3FCFC34092EB355092463680914E3F6F
:10E4A0008F5F80934E3FC5C31092EC355092473634
:10E4B0008091513F8F5F8093513FBBC35092EC35A9
:10E4C000509247368091513F8F5F8093513FB1C347
:10E4D000C701B6010E9497D96C837D838E839F8389
:10E4E00020E030E040E251E4C701B6010E947DD84F
:10E4F0006B017C0120E030E040E251E46C817D81E1
:10E500008E819F810E947DD89B01AC01C701B6011D
:10E510000E942FD40E944CD6623001F128F4662369
:10E5200041F0613089F0A0C56330E9F0643001F159
:10E530009BC5B5E0B093BB355092163680914C3FE9
:10E540008F5F80934C3F75C33092BB356093163616
:10E5500080914C3F8F5F80934C3F6BC35092BB3593
:10E560005092163666C34092BB355092163661C340
:10E5700083E08093BB35509216365BC3C701B6016A
:10E580000E9497D96C837D838E839F8320E030E047
:10E5900040E251E4C701B6010E947DD86B017C01C5
:10E5A00020E030E040E251E46C817D818E819F81EA
:10E5B0000E947DD89B01AC01C701B6010E942FD4F7
:10E5C0000E944CD6662319F0613061F04DC587E09A
:10E5D0008093BB355092163680914C3F8F5F80936D
:10E5E0004C3F27C3E6E0E093BB356093163680913D
:10E5F0004C3F8F5F80934C3F1CC3C701B6010E9404
:10E6000097D96C837D838E839F8320E030E040E246
:10E6100051E4C701B6010E947DD86B017C0120E066
:10E6200030E040E251E46C817D818E819F810E94C7
:10E630007DD89B01AC01C701B6010E942FD40E9476
:10E640004CD6623009F010C58EE08093BB355092F5
:10E650001636EFC25092EE3550924936EAC25092C9
:10E66000ED35509248368091553F8F5F8093553FEE
:10E67000E0C24092ED35509248368091553F8F5F11
:10E680008093553FD6C283E016C03092ED3550924C
:10E6900048368091553F8F5F8093553FCAC2F5E061
:10E6A000F093ED35509248368091553F8F5F8093BF
:10E6B000553FBFC286E08093ED3550924836809139
:10E6C000553F8F5F8093553FB4C2C701B6010E948A
:10E6D00097D96C837D838E839F8320E030E040E276
:10E6E00051E4C701B6010E947DD86B017C0120E096
:10E6F00030E040E251E46C817D818E819F810E94F7
:10E700007DD89B01AC01C701B6010E942FD40E94A5
:10E710004CD6662319F0613059F0A6C41092F0353A
:10E7200050924B368091563F8F5F8093563F81C207
:10E730006093F03560934B368091563F8F5F8093A6
:10E74000563F77C24092F03550924B368091563FFB
:10E750008F5F8093563F6DC23092BC355092173612
:10E7600080914D3F8F5F80934D3F63C2C701B601DB
:10E770000E9497D96C837D838E839F8320E030E055
:10E7800040E251E4C701B6010E947DD86B017C01D3
:10E7900020E030E040E251E46C817D818E819F81F8
:10E7A0000E947DD89B01AC01C701B6010E942FD405
:10E7B0000E944CD6662319F0613059F055C410926E
:10E7C000F13550924C3680914F3F8F5F80934F3F91
:10E7D00030C21092F23560934D3680914F3F8F5F7B
:10E7E00080934F3F26C2C701B6010E9497D96C8320
:10E7F0007D838E839F8320E030E040E251E4C701B7
:10E80000B6010E947DD86B017C0120E030E040E23F
:10E8100051E46C817D818E819F810E947DD89B0116
:10E82000AC01C701B6010E942FD40E944CD66623CA
:10E8300019F0613059F018C45092F13550924C36AD
:10E8400080914F3F8F5F80934F3FF3C16093F235CC
:10E8500060934D3680914F3F8F5F80934F3FE9C16A
:10E86000C701B6010E9497D96C837D838E839F83F5
:10E8700020E030E040E251E4C701B6010E947DD8BB
:10E880006B017C0120E030E040E251E46C817D814D
:10E890008E819F810E947DD89B01AC01C701B6018A
:10E8A0000E942FD40E944CD6613089F028F062304B
:10E8B000A1F06330C1F0D8C399E09093BB3550927A
:10E8C000163680914C3F8F5F80934C3FB2C1AAE0D7
:10E8D000A093BB3560931636ACC1BBE0B093BB359B
:10E8E00050921636A6C1ECE0E093BB355092163636
:10E8F000A0C11092E635509241368091503F8F5F13
:10E900008093503F96C15092E635509241368091A7
:10E91000503F8F5F8093503F8CC1C701B6010E946A
:10E920004CD6862F90E08D33910508F09BC3FC01F7
:10E93000ED5AFE4F0C9423DE1092BD3550921836DE
:10E940008091573F8F5F8093573F73C15092BD3581
:10E95000509218368091573F8F5F8093573F69C11F
:10E960005092F835509253368091593F8F5F809383
:10E97000593F5FC14092F835509253368091593FCC
:10E980008F5F8093593F55C11092F835509253369E
:10E990008091593F8F5F8093593F4BC15092F5351D
:10E9A0005092503646C15092F63550925136809171
:10E9B0005A3F8F5F80935A3F3CC15092F735509237
:10E9C000523680915A3F8F5F80935A3F32C11092E6
:10E9D000F7355092523680915A3F8F5F80935A3F5D
:10E9E00028C15092E9355092443680915B3F8F5F49
:10E9F00080935B3F1EC11092E9355092443680915E
:10EA00005B3F8F5F80935B3F14C15092E73550921C
:10EA1000423680915B3F8F5F80935B3F0AC150928B
:10EA2000013650925C3680915B3F8F5F80935B3FF5
:10EA300000C1C701B6010E9497D90E944CD66093CD
:10EA4000F43550924F36F5C0C092DA35D092DB35AE
:10EA5000E092DC35F092DD35809235369092363694
:10EA6000A0923736B0923836E4C0C0920236D092C7
:10EA70000336E0920436F092053680925D3690922D
:10EA80005E36A0925F36B0926036D3C0C092F93540
:10EA9000D092FA35E092FB35F092FC3580925436F4
:10EAA00090925536A0925636B0925736C2C0C09258
:10EAB000C235D092C335E092C435F092C53580920C
:10EAC0001D3690921E36A0921F36B0922036B1C0ED
:10EAD000C092C635D092C735E092C835F092C9359C
:10EAE0008092213690922236A0922336B09224361C
:10EAF000A0C0C092CA35D092CB35E092CC35F0920E
:10EB0000CD358092253690922636A0922736B09247
:10EB100028368FC0C092CE35D092CF35E092D03516
:10EB2000F092D1358092293690922A36A0922B36D7
:10EB3000B0922C367EC0C092D235D092D335E092BE
:10EB4000D435F092D53580922D3690922E36A09203
:10EB50002F36B09230366DC0C092D635D092D735B0
:10EB6000E092D835F092D935809231369092323693
:10EB7000A0923336B09234365CC0C0920A36D0923E
:10EB80000B36E0920C36F0920D36809265369092FC
:10EB90006636A0926736B09268364BC0C0920E3689
:10EBA000D0920F36E0921036F0921136809269368C
:10EBB00090926A36A0926B36B0926C363AC0C09290
:10EBC0001236D0921336E0921436F09215368092B7
:10EBD0006D3690926E36A0926F36B092703629C024
:10EBE000C0920636D0920736E0920836F092093687
:10EBF0008092613690926236A0926336B09264360B
:10EC000018C0C701B6010E944CD66093BE35709300
:10EC1000BF358093C0359093C13581E090E0A0E08E
:10EC2000B0E08093193690931A36A0931B36B093B8
:10EC30001C36D8012C90222009F424C2822D90E0A9
:10EC40000E94D2E1892B09F42FC23801BFEF6B1A61
:10EC50007B0AF8018181803349F48281883531F45F
:10EC60000E5F1F4FC12CD12C760100C2BE016F5F19
:10EC70007F4FC3010E9443DE6B017C0109811A8131
:10EC80006016710609F0F2C111C28091E6350E944A
:10EC90008853182F01C010E06091353670913636D8
:10ECA00080913736909138360E944CD6662359F0C1
:10ECB0006091DA357091DB358091DC359091DD35EE
:10ECC0000E945753182F6091393670913A368091CF
:10ECD0003B3690913C360E944CD6662371F0609191
:10ECE000DE357091DF358091E0359091E1350E94FD
:10ECF0004CD6862F0E943355182F60913D36709167
:10ED00003E3680913F36909140360E944CD6662325
:10ED100071F06091E2357091E3358091E435909126
:10ED2000E5350E944CD6862F0E947255182F6091AF
:10ED300054367091553680915636909157360E94D0
:10ED40004CD6662359F06091F9357091FA3580916F
:10ED5000FB359091FC350E948AB0182F609158368F
:10ED60007091593680915A3690915B360E944CD6FC
:10ED7000662371F06091FD357091FE358091FF350D
:10ED8000909100360E944CD6862F0E94B155182FC4
:10ED900080914F36882329F08091F4350E94F053FA
:10EDA000182F80915036882329F08091F5350E94E4
:10EDB0002454182F80915336882329F08091F835F8
:10EDC0000E9456B0182F80915136882329F08091E7
:10EDD000F6350E945954182F80915236882329F015
:10EDE0008091F7350E948D54182F809142368823E8
:10EDF00029F08091E7350E940855182F80914336FD
:10EE0000882329F08091E8350E944755182F80917A
:10EE10005C36882329F0809101360E948655182F90
:10EE200080914436882329F08091E9350E9400556D
:10EE3000182F8091BB358D3029F08091463688237C
:10EE4000A9F00FC0609102367091033680910436AC
:10EE5000909105360E9490538093B43F882369F3C4
:10EE60002FC18091EB350E941F4F182F809147369C
:10EE7000882329F08091EC350E94234F182F809130
:10EE80004836882329F08091ED350E94DD4F182FF8
:10EE900080914B36882329F08091F0350E948C5365
:10EEA000182F80914C36882329F08091F1350E94EB
:10EEB000274F182F4091BB3550E04F30510508F0D7
:10EEC000B6C0FA01E057FE4F0C9423DE0E94D952DF
:10EED000182FADC06DE176E382EC95E30E94E45219
:10EEE000182FA5C00E941853182FA1C06DE176E31A
:10EEF00082EC95E30E942353182F99C00E94816BE6
:10EF0000182F95C06DE176E382EC95E30E94A35043
:10EF1000182F8DC00E94CA6B182F89C06DE176E34F
:10EF200082EC95E30E940270182F81C06091023636
:10EF30007091033680910436909105360E944CD62C
:10EF4000862F2DE136E342EC55E36091EA350E94CD
:10EF50002B4F182F6CC06DE176E382EC95E30E9495
:10EF60002051182F64C00E94D351182F60C00E94F6
:10EF70003A52182F5CC00E947152182F58C06091ED
:10EF8000EE358DEE94E30E94664B8091BC35843063
:10EF900038F48230D8F4882349F0813079F047C0C2
:10EFA000843009F044C08093F13441C06DE176E3D0
:10EFB00082EC95E30E94A952182F39C06DE176E3E7
:10EFC00082EC95E30E949C53182F31C0A09012361A
:10EFD000B0901336C0901436D0901536E0900E36AF
:10EFE000F0900F36009110361091113620910A36AC
:10EFF00030910B3640910C3650910D368F938091A5
:10F0000009368F93809108368F93809107368F93BE
:10F01000809106368F936DE176E382EC95E30E9452
:10F020001186182F0F900F900F900F900F9060E0A7
:10F030008DEE94E30E94664B80911836813061F426
:10F040008091BD35811104C00E94B256812F38C015
:10F050000E94E356812F34C0812F32C08BEC30C028
:10F0600083E02EC084E82CC083E82AC0822D90E083
:10F07000FC01E154F109EA31F105B0F7E156FE4F28
:10F080000C9423DE1092B43F6091BE357091BF3571
:10F090008091C0359091C1350E94004B80914136DE
:10F0A000882309F4F8CDF1CD85E60AC086E608C0CC
:10F0B000D8018C91DAC868018B2D78017B2CA4C80B
:10F0C0002796CDBFDEBFDF91CF911F910F91FF90AB
:10F0D000EF90DF90CF90BF90AF909F908F907F90F8
:10F0E0006F905F904F903F902F900895CF93DF9354
:10F0F000EC016AEA7EE30E94B5628093B43F81111D
:10F1000002C095E09F83DF91CF910895FC0187892C
:10F11000908D0C94D07083FF06C0E0918F32F091F7
:10F12000903290E2958382FF06C0E0919132F09197
:10F13000923290E2958381FF06C0E0919332F09184
:10F14000943290E2958380FF06C0E0919532F09171
:10F15000963280E28583089583FF06C0E0918F3266
:10F16000F091903290E2968382FF06C0E091913256
:10F17000F091923290E2968381FF06C0E091933243
:10F18000F091943290E2968380FF06C0E091953230
:10F19000F091963280E2868308958091863C8111B9
:10F1A00007C084E00E948B7881E08093863C0895BC
:10F1B00084E00E94AC781092863C0895CF92DF9252
:10F1C000EF92FF920F931F93CF93DF93C12C26E012
:10F1D000D22EC0927F32D092803230EAE32E36E0D7
:10F1E000F32EE0928132F092823200E816E0009332
:10F1F000833210938432C0E6D6E0C0938532D09338
:10F200008632C0928732D0928832C0938932D093AE
:10F210008A3200938B3210938C32E0928D32F092CE
:10F220008E322DEC3CEC4CED50E40E94DBD7C092CA
:10F230008F32D0929032E0929132F0929232181640
:10F240004CF4C0939332D093943200939532109340
:10F25000963208C00093933210939432C093953243
:10F26000D0939632DF91CF911F910F91FF90EF9045
:10F27000DF90CF9008950E9482D360E070E080E03C
:10F2800091E40E94DE780C94A1D381E080938F3CBE
:10F29000089520E093E088ED08B618BE84BF9093EF
:10F2A00080002091820021FDFCCF08BEFFCF80911D
:10F2B0008F3C81110E94497983E008958091903CB0
:10F2C000882341F0F89461E089E790E00E9484D3BC
:10F2D00082E0089583E00895CF93DF93CDB7DEB742
:10F2E000AD97CDBFDEBF21E2EDEEF1E2DE0111967A
:10F2F00001900D922A95E1F722E02093CA01DE01E8
:10F300009296E8E0F0E024912D933196EE30F105ED
:10F31000D1F72DE228A7E0E1F0E0E491EF7121E0E0
:10F3200030E02C0F3D1F2E0F311DF901208129A740
:10F33000E2E1F0E0E491EF719E012E0F311DF90141
:10F3400021812AA7E4E1F0E0E491EF719E012E0F04
:10F35000311DF90121812BA71CA61092CA0125E0BD
:10F36000FC012783BE016E5D7F4F0E94B5628093D2
:10F37000B43FAD96CDBFDEBFDF91CF91089581E060
:10F380008093903C80E00895CF93DF93EC0120E0E0
:10F3900030E040E051E469857A858B859C850E9448
:10F3A000DBD718166CF0CE010E94645F69857A8500
:10F3B0008B859C850E94DE780E9424BE80E001C07F
:10F3C0008DE6DF91CF91089565E27CE30C9416C23F
:10F3D00067E07CE30C9416C26AEE7BE30C9416C2E1
:10F3E0006CEC7BE30C9416C268EB7BE30C9416C2C6
:10F3F000CF93DF938BE697E49F938F93CCE6DCE586
:10F4000089818F9388818F930E94EEE285E395E452
:10F410009F938F9389818F9388818F930E94EEE2CF
:10F420008DEA94E49F938F9389818F9388818F9342
:10F430000E94EEE283EE93E49F938F9389818F93F2
:10F4400088818F930E94EEE20E94EDA98DB79EB74E
:10F4500040968DBF9EBF80E0DF91CF910895CF93FE
:10F46000DF938EEB93E49F938F93CCE6DCE5898169
:10F470008F9388818F930E94EEE280E592E49F93C0
:10F480008F9389818F9388818F930E94EEE285EC20
:10F4900090E49F938F9389818F9388818F930E94AB
:10F4A000EEE28DEA94E49F938F9389818F93888114
:10F4B0008F930E94EEE283EE93E49F938F93898172
:10F4C0008F9388818F930E94EEE28DB79EB744960A
:10F4D0008DBF9EBF80E0DF91CF910895CF93DF93E2
:10F4E00084EA90E49F938F93CCE6DCE589818F9347
:10F4F00088818F930E94EEE286E29DE39F938F9333
:10F5000089818F9388818F930E94EEE283EE93E44A
:10F510009F938F9389818F9388818F930E94EEE2CE
:10F520008DB79EB70C968DBF9EBF80E0DF91CF91C7
:10F530000895CF93DF938EEF9CE39F938F93CCE658
:10F54000DCE589818F9388818F930E94EEE28DE8BC
:10F550009CE39F938F9389818F9388818F930E94DF
:10F56000EEE283EE93E49F938F9389818F9388815A
:10F570008F930E94EEE28DB79EB70C968DBF9EBF13
:10F5800080E0DF91CF910895CF93DF938AE69CE3EB
:10F590009F938F93CCE6DCE589818F9388818F934D
:10F5A0000E94EEE281E49CE39F938F9389818F9385
:10F5B00088818F930E94EEE283EE93E49F938F9372
:10F5C00089818F9388818F930E94EEE28DB79EB7D9
:10F5D0000C968DBF9EBF80E0DF91CF9108953F9242
:10F5E0004F925F926F927F928F929F92AF92BF9253
:10F5F000CF92DF92EF92FF920F931F93CF93DF93FF
:10F60000CDB7DEB76497CDBFDEBF6C018B015A0169
:10F610008BE79CE2A2E2B0E08F839887A987BA8744
:10F620008AE392E2A0E08E879F87A88B8CE29DE719
:10F63000A0E08B879C87AD8786E0EEE0F2E2DE01FA
:10F64000119601900D928A95E1F7DB01ED91FC9105
:10F650008081811102C083E0AEC1C6010E94696150
:10F66000F5018081D60116968C93F8016080718037
:10F6700023014301F9E08F0E911C72012FEF421A12
:10F68000520AD7016C9170E0CE0107960E9440E2C9
:10F69000892B41F4F801408251823701F2E26F0E6A
:10F6A000711C0DC0D3018C918823A9F24814590410
:10F6B00011F48FE680C1F80140825182DECF420111
:10F6C000FFEF4F1A5F0AD4016C9170E0CE010E96E5
:10F6D0000E9440E2892BE9F0F80140825182D40176
:10F6E0001C9246E050E0B7017601B1E1EB0EF11C4F
:10F6F000C7010E946BE2B70187E493E20E94E65FD4
:10F700008B8B9C8BF60184839583019649F484E668
:10F7100052C146145704D9F3D8014D925C92CFCF11
:10F72000F801608071804301F9E08F0E911C230184
:10F73000D3013D903D01E32CF12CC7010E94C7E1AC
:10F74000892B71F4B701CE0101960E9440E2892B0A
:10F7500039F468147904D9F2F80160827182E7CF34
:10F76000FEE63F1649F022E2321209C0D20111969C
:10F770008C91823209F057C0F6011782E6C0F0E39F
:10F78000EF1AF1082AE0E216F10418F08DE23812BF
:10F7900038C0EB89FC89EE0FFF1FAB89BC89EA0FEB
:10F7A000FB1FEE0FFF1FEE0FFF1FEE0FFF1FEF54AB
:10F7B000FA4EE491E4FF17C0BE016F5E7F4FC201B5
:10F7C0000E9443DEF6016187728783879487D801A0
:10F7D0004D905C9089899A894816590609F4E8C0C9
:10F7E00084E08783B2C0C2010E94C8E0F60161874D
:10F7F00072878387948782E08783D8014D905C90DD
:10F80000A4C0BBE73B126DC088E0F6018783D50139
:10F810008C918F5F8C93F801808191810196808318
:10F82000918382E0C8C0B2016F5F7F4FD8016D93B2
:10F830007C9385E0F60187839B01FB01D9018C91C4
:10F840008C3569F411969C919232E9F49083D80139
:10F850008D919C91119701968D939C9318C0823243
:10F8600091F41082F801A081B181CD0101968083CD
:10F870009183FC0101900020E9F73197E81BF90B17
:10F88000339768F426C08083D8018D919C919C01A8
:10F890002F5F3F4FD8012D933C933196CFCF1196D8
:10F8A0002C9111972033A9F412962C91283789F4C2
:10F8B00040E050E060E070E00E94B4DFF601618754
:10F8C00072878387948783E08783D8014D905C900B
:10F8D0003CC0C6010E94B5628093B43F882391F179
:10F8E0006AC0B4E73B120FC081E0F601878381E074
:10F8F00090E0A0E0B0E081879287A387B487D80129
:10F900004D905C9022C0B6E63B120BC081E0F60140
:10F9100087831186128613861486F80140805180F1
:10F9200014C0FBE53F12C5CE86E0D60117968C9336
:10F93000B201C6010E94B5628093B43F81113BC001
:10F9400087E639C0F80140805180BE01655F7F4F76
:10F95000C2010E9485E2FC01D8018D939C9300971F
:10F9600009F4A7CE208120C0213210F02F3741F4B6
:10F97000CF010196D8018D939C932181FC0114C085
:10F980002D3781F4F501808181508083D8018D91DC
:10F990009C911197FC013196ED93FC93DC0111963B
:10F9A0002C9102C02C3231F02111DECF80E003C057
:10F9B00086E601C082E06496CDBFDEBFDF91CF91C5
:10F9C0001F910F91FF90EF90DF90CF90BF90AF907D
:10F9D0009F908F907F906F905F904F903F90089591
:10F9E0002F923F924F925F926F927F928F929F924F
:10F9F000AF92BF92CF92DF92EF92FF920F931F933D
:10FA0000CF93DF93CDB7DEB72897CDBFDEBF8C0194
:10FA10006E837F8381E08D8319821A821B821C8210
:10FA200080915E3F8F5F80935E3F833008F046C1D8
:10FA30007B01FB0101900020E9F73197E61BF70BF2
:10FA4000E130F24008F03CC1FB0120816B01222330
:10FA500009F448C051E040E0E2E29E2EF701223E68
:10FA600099F48181803881F497012E5F3F4FF7012F
:10FA7000828194E6980F923048F4F6019082C60194
:10FA800001966C01790126C0808101C07901411184
:10FA900018C041E0883209F040E0552321F081325E
:10FAA000C8F08F37B9F05601FFEFAF1ABF0A90E0E8
:10FAB00048870E94E3E1F6018083650150E04885B4
:10FAC00009C041E0893209F440E0F6018083C601B3
:10FAD00001966C01C7010196F7012181222311F0E3
:10FAE0007C01BCCFF60110821092B43F27E6422E73
:10FAF00023E6522E612C32E0732E3324339442E8F5
:10FB0000C42E47E4D42E59E0252E64E8862E67E4FF
:10FB1000962E72E9A72E77E4B72EAE014B5F5F4FAA
:10FB2000BE016A5F7F4FC8010E94EF7A843008F0FF
:10FB3000CAC0833011F480E0C6C0F80187818830E4
:10FB4000C1F5848195810E943E65882381F078010A
:10FB5000F1E1EF0EF11CC7010E94C45F882339F068
:10FB600043E050E0B701CE0101960E946BE2F8013C
:10FB7000E280F380AE014B5F5F4FBE016A5F7F4F53
:10FB8000C7010E94EF7A833009F46EC0898188230F
:10FB900049F043E050E0BE016F5F7F4FC7010D9613
:10FBA0000E946BE2F701E280F380E114F10411F7A7
:10FBB0005BC0F80184819581209102373091033731
:10FBC0008217930711F427E027830E94DB5F8823C5
:10FBD00009F44AC0F801E788F08CF70160816B37BF
:10FBE00029F4B701C8010E94F07C3EC070E088E7AC
:10FBF00091E20E9440E2892B41F180915D3F8111A9
:10FC000007C0BF92AF920E944FE30F900F9006C0C3
:10FC10009F928F920E944FE30F900F907092843CBE
:10FC2000C7010E9427BF3092843CDF92CF920E948E
:10FC30004FE380E090E00E94796120920B37F80159
:10FC4000828193810F900F9035C0F801418A528ACA
:10FC5000638AC7010E94D0706AEA7EE30E948DC069
:10FC6000F8018281938126C0F80187818F3F19F4C2
:10FC7000828193811FC0811104C0C8010E945B5C16
:10FC800010C08091BD34823061F0C8010E94315CA7
:10FC9000C8010E94AE5C05C0F80127812F3F51F0DA
:10FCA0008C01F801828193810097B1F782B193B101
:10FCB00000E010E0892B09F030CF3DCF82E703C090
:10FCC0008BE68093B43F2896CDBFDEBFDF91CF9106
:10FCD0001F910F91FF90EF90DF90CF90BF90AF906A
:10FCE0009F908F907F906F905F904F903F902F905C
:10FCF0000895CF93DF93EC0110925E3F80E090E097
:10FD00000E947961BE010E94F07C42E060E00E94A6
:10FD1000536381E0DF91CF910C944CAC2F923F92D2
:10FD20004F925F926F927F928F929F92AF92BF920B
:10FD3000CF92DF92EF92FF920F931F93CF93DF93B7
:10FD400000D000D0CDB7DEB769837A834B835C8364
:10FD50007A0120E1E21AF108E60EF71E0E947D62A8
:10FD60004C01009731F4A981BA811C9280E090E0A7
:10FD700071C1FC0156808781893021F08FEF850D9C
:10FD8000352D05C082809380F401368181E00981A0
:10FD90001A81FCE26F2EABE77A2EBDE73B2E98E18D
:10FDA000A92E92E2B92E24E1C22E22E2D22E45E003
:10FDB000442E56E0252E8D829E8283173CF4480106
:10FDC000FFEF8F1A9F0AD8017C922FC0831719F07A
:10FDD0003817A4F024C0AD81BE81ED91FC918781DC
:10FDE000883029F4F801708231820E5F1F4F48017C
:10FDF000FFEF8F1A9F0AD8016C9217C0F801AD81EE
:10FE0000BE81CF0101968C01308216962C911697F7
:10FE100023171CF4FC01322FF4CFAD83BE834801BD
:10FE2000BFEF8B1A9B0AF801608280915D3F8111C0
:10FE300008C08D819E8141969F938F93DF92CF92D0
:10FE400007C08D819E8141969F938F93BF92AF9201
:10FE50009F928F920E94A0E38401080F191F0F90B8
:10FE60000F900F900F900F900F90AD81BE8117965D
:10FE70008C9181110BC0EEE1F2E2D801842D01904A
:10FE80000D928A95E1F70C5F1F4FA0C0823069F494
:10FE9000ED81FE8184858F9383858F9382858F93F7
:10FEA00081858F93A3E2B2E215C08330F1F4AD8176
:10FEB000BE811C968C911C978F931B968C911B97DF
:10FEC0008F931A968C911A978F9319968C918F9382
:10FED000A7E2B2E2BF93AF931F930F930E94A0E3F8
:10FEE000080F191FCDBFDEBF71C08530E1F4AD81B1
:10FEF000BE8157968C91579758969C91DC01FD01D5
:10FF000001900020E9F73197EA1BFB0BE00FF11F8E
:10FF1000EE15FF0518F08FEF9FEF9CC09F938F9316
:10FF2000AFE2B2E20DC08630D1F4AD81BE81589609
:10FF30008C9158978F9357968C918F93A4E3B2E24C
:10FF4000BF93AF931F930F930E94A0E3080F191F55
:10FF50000F900F900F900F900F900F9037C084303C
:10FF6000A1F48D819E810E944E65AD81BE8119965E
:10FF70004D915D916D917C911C9718962C91C801C3
:10FF80000E9447C4080F111D21C08130F9F4ED8192
:10FF9000FE8181859285A385B485892B8A2B8B2B45
:10FFA00059F4E9E3F2E2D801822D01900D928A958D
:10FFB000E1F70B5F1F4F0AC0EFE3F2E2D801842D97
:10FFC00001900D928A95E1F70C5F1F4F0E151F05EA
:10FFD00008F0A1CFAD81BE8116968C91169712962E
:10FFE000ED91FC911397ED83FE83309711F03681EC
:10FFF000E4CE22E030E02519310957FC3395280F73
:020000021000EC
:10000000311D87FD3A95200F311F49815A816B813F
:100010007C81460F571F4217530708F47CCF5816B0
:1000200064F4F8019DE79F012F5F3F4F89019083A2
:100030008150581614F4F901F6CF8DE79AE0A0E04C
:10004000F80180839183A283C801029629813A81B5
:10005000821B930B2696CDBFDEBFDF91CF911F9100
:100060000F91FF90EF90DF90CF90BF90AF909F9057
:100070008F907F906F905F904F903F902F9008955A
:1000800040E052E06AEA7CE30E948E7E1816190670
:1000900044F48AEA9CE39F938F930E943DE30F9080
:1000A0000F900895EF92FF920F931F93CF93DF93DA
:1000B000CDB7DEB76297CDBFDEBF182F80915C3F12
:1000C000882309F4F3C080910B37893049F088E028
:1000D00080930B3782E790E0809315379093163723
:1000E0001F36D9F480E090E00E94796188E0809327
:1000F000243782E790E080932E3790932F376AEA77
:100100007EE38091A63C9091A73C0E9427C4BC014D
:100110008CE091E20E9413634FC08091BD3488232C
:1001200009F44AC06DE1E62E67E3F62E0EEFF70103
:1001300087818F3F09F440C0873071F44185528533
:10014000638574854093A23C5093A33C6093A43C88
:100150007093A53C078329C0C7010E944D6082307F
:1001600029F48091633F811120C01DC0843029F49F
:100170008091603F811119C016C0853071F4809163
:10018000623F882381F0F70141855285638574853C
:10019000452B462B472B49F406C0813031F4809122
:1001A000613F811102C0F7010783F701E280F3800C
:1001B000E114F10409F0BBCF4091A23C5091A33C63
:1001C0006091A43C7091A53C4115510561057105F4
:1001D000C9F04093FB395093FC396093FD3970931B
:1001E000FE3944E759E664E670E04093033A5093E1
:1001F000043A6093053A7093063A82E08093F939A5
:100200001092F8398091773281111AC08091A93CFF
:100210008F938091A83C8F931F921F9384E492E266
:100220009F938F938E010F5F1F4F1F930F930E9419
:10023000A0E31092A83C1092A93CCDBFDEBF13C032
:100240000E947CC91F928F931F921F938CE492E2AD
:100250009F938F938E010F5F1F4F1F930F930E94E9
:10026000A0E3CDBFDEBFB8018BE09AE30E94B56288
:100270001092113A86E08093123A86E690E08093DD
:100280001C3A90931D3A40E052E06AEA7CE384E035
:1002900097E30E948E7E1816190644F48AEA9CE3BE
:1002A0009F938F930E943DE30F900F906296CDBF76
:1002B000DEBFDF91CF911F910F91FF90EF900895D6
:1002C000613019F0623029F0089584E097E30C94CE
:1002D00040800C945280FC0181859285A385B48571
:1002E00086309105A105B10580F580935C3F1092A1
:1002F0005F3F1092603F1092613F1092623F1092F8
:10030000633F0097A105B10511F121E020935F3F04
:1003100081309105A105B105D1F02093603F823075
:100320009105A105B10599F02093613F83309105B6
:10033000A105B10561F02093623F0597A105B105C4
:1003400031F42093633F80E008958EE6089580E0C5
:10035000089567E278E40C9416C260ED77E40C949B
:1003600016C26CE977E40C9416C2BF92CF92DF926A
:10037000EF92FF920F931F93CF93DF93CDB7DEB72A
:100380006897CDBFDEBF6B0128E1FC01DE0111964D
:1003900001900D922A95E1F78EE7E82E83E3F82E7F
:1003A0008E010F5F1F4FB12CF7018081823029F43D
:1003B000F80110821182128213828091EE5A8B1101
:1003C00014C02091015B3091025B4091035B50911E
:1003D000045BF80160817181828193810E947DD8E4
:1003E000F601608371838283938380910D5B8B110F
:1003F00014C02091205B3091215B4091225B509191
:10040000235BF80160817181828193810E947DD894
:10041000F601648375838683978380912C5B8B11AF
:1004200014C020913F5B3091405B4091415B509103
:10043000425BF80160817181828193810E947DD845
:10044000F601608771878287938780914B5B8B1160
:1004500014C020915E5B30915F5B4091605B509176
:10046000615BF80160817181828193810E947DD8F6
:10047000F6016487758786879787B394F5E3EF0E57
:10048000F11C0C5F1F4F86E0B8128ECF6896CDBF6F
:10049000DEBFDF91CF911F910F91FF90EF90DF9022
:1004A000CF90BF900895F8940E943B790E94AA8251
:1004B0000E94A1D30E943AC60E94C1B40E948B70D0
:1004C0000E9424BE0E9453A740E060E080E00E94AA
:1004D0004E660E94C2610E9498820E945D840E94C2
:1004E00013500E9499D38091A20084608093A2004F
:1004F0008091A20082608093A2008091A20081601E
:100500008093A20078940E94EDA90E9426BF0E94C9
:10051000A066FDCFE82FF0E0EE0FFF1FED5AF74B7E
:10052000659174914FE450E084E69FE30C9412E2ED
:100530008091833C823041F440E060E081E00E94A1
:100540004E6680E00E94C8670C9475CA682F81E0EF
:100550000C9417C71092B53F1092B63F1092B73F58
:100560001092B83F0895CF93DF93EC018C819D8169
:10057000880F991F880F991F2091B73F3091B83F7E
:10058000820F931F8093B93F9093BA3F44E050E0AD
:100590006FEB7FE30E9499D24091BF3F5091C03FE3
:1005A0006091C13F7091C23F49875A876B877C87B2
:1005B00080E0DF91CF9108950F931F93CF93DF9346
:1005C000EC018091BE34882339F08AE6DF91CF9127
:1005D0001F910F910C9474A949855A856B857C8570
:1005E0004093BB3F5093BC3F6093BD3F7093BE3F71
:1005F000CE010E94B3828093B43F811141C000912B
:10060000BB3F1091BC3F2091BD3F3091BE3F49851B
:100610005A856B857C85401751076207730739F14E
:100620000093BF3F1093C03F2093C13F3093C23F20
:100630008C819D81880F991F880F991F2091B73F4A
:100640003091B83F820F931F8093B93F9093BA3F88
:1006500044E050E06FEB7FE30E942AD33091BB3F30
:100660002091BC3F9091BD3F8091BE3F04C0342F8C
:10067000252F962F872F39872A879B878C8780E0A5
:10068000DF91CF911F910F9108950E943CBA80E0B5
:1006900008958091C33F9091C43F8F3E924111F0E5
:1006A0008EE508958091E93F9091EA3F8F3E924117
:1006B000B9F78091EB3F9091EC3F8F3E924181F7EB
:1006C00080917457909175578F3E924149F7809170
:1006D0007657909177578F3E924111F78091095943
:1006E00090910A598F3E9241D9F680E0089594E0A6
:1006F000899FF0011124ED53F04C428353836483AE
:100700007583089594E0899FF0011124EA58F84A0E
:1007100045AB56AB67AB70AF08955F926F927F9217
:100720008F929F92AF92BF92CF92DF92EF92FF9201
:100730000F931F93CF93DF93CDB7DEB76097CDBFF5
:10074000DEBFBE016F5F7F4F8BEA97E50E94B581E8
:10075000CE0101964C0183E2A82E88E5B82E93E3E2
:10076000C92E98E5D92E23E4E22E28E5F22E03E6E1
:1007700018E535E8632E3BE5732E512CF4014191C9
:100780005191619171914F01F501419351936193A1
:1007900071935F01F60141935193619371936F01DE
:1007A000F70141935193619371937F01852D0E94CD
:1007B000AD70F80111921192119211928F01F30113
:1007C00010821182128213825394F8E16F0E711C11
:1007D00084E05812D3CF6096CDBFDEBFDF91CF91BA
:1007E0001F910F91FF90EF90DF90CF90BF90AF904F
:1007F0009F908F907F906F905F9008958091ED3FD4
:1008000008951F93CF93DF938BE897E1EBEEFFE31F
:10081000DF019C011D9221503040E1F78FEE92E103
:100820008093EB3F9093EC3F809374579093755770
:10083000C4EFDFE3C093EE3FD093EF3FC093F03FB0
:10084000D093F13FC093F23FD093F33F81E090E02B
:1008500068EB76E520E030E01CEB129FA001139FCF
:10086000500D1124FA01E551F04CD90111961A9F4F
:1008700090011B9F300D11242C50304C238734875E
:1008800061877287BA016C50704C9C01019680326E
:10089000910519F78CEB829FF001839FF00D1124D5
:1008A000E551F04CC387D4876187728780E28093DB
:1008B000ED3FDF91CF911F910895CF93DF93E6E74E
:1008C000F7E585E991E0DF01EC011D922197E9F759
:1008D000A3ECBFE388E2ED0119928A95E9F78FEE68
:1008E00092E18D939C938093E93F9093EA3F8083BC
:1008F00091838093095990930A59DF91CF910C9479
:1009000001840E947A8E0E94018480E00C94B54A92
:10091000E091EE3FF091EF3F848581111BC0228171
:100920003381808191814CEBDF011D924A95E9F77B
:10093000228333838083918381E084878091ED3F9C
:1009400081508093ED3F828193818093EE3F90931D
:10095000EF3F05C08CE10E9474A9E0E0F0E0CF0118
:100960000895A0EFBFE3ED91FC911197858781E099
:10097000878782E08487828193818D939C9381E035
:100980000E947EAD0C9482B7EF92FF920F931F935B
:10099000CF93DF9300D01F92CDB7DEB78C014B838E
:1009A0005C8369837A830E948884FC014B815C812B
:1009B00069817A81009761F48EE02496CDBFDEBF15
:1009C000DF91CF911F910F91FF90EF900C94FC4E0F
:1009D00083E0858785E493E8848395830683178382
:1009E0008B017A0126E0D8014D915D916D917D9149
:1009F0008D01CF0185599F4FDC014D935D936D9320
:100A00007C931397D7014D915D916D917D917D01FF
:100A1000418B528B638B748B215034962111E3CF21
:100A200083E02496CDBFDEBFDF91CF911F910F9160
:100A3000FF90EF900C94B184CF92DF92EF92FF92EF
:100A40006B017C010E948884009739F48EE0FF904E
:100A5000EF90DF90CF900C94FC4E2FE935E8FC012D
:100A600024833583E556FF4FC082D182E282F38230
:100A700021E0FC01278782E00E94B18480E0FF90A2
:100A8000EF90DF90CF9008958091F23F9091F33FE7
:100A9000FC0124853EEF320F323018F424E0248725
:100AA0000895243011F080E090E00895E091F23F45
:100AB000F091F33F22813381808191814CEBDF0102
:100AC0001D924A95E9F72283338380839183E091D5
:100AD000F23FF091F33F0280F381E02DE093F23F8B
:100AE000F093F33F8485823011F483E08487809112
:100AF000ED3F8F5F8093ED3F8FEF0E947EAD81E0F1
:100B00004091EE3F5091EF3F2091F23F3091F33F03
:100B10004217530709F080E00895BC016F5E7F4FD4
:100B2000DC011696ED91FC91179785599F4F199509
:100B30000E94568581110E947F5680E00895855657
:100B40009F4F20E034E244E759E4FC016081718169
:100B5000828193810E947DD80E944CD60E9478D6D3
:100B60000E9446BA0E94568581110E947F5680E0FD
:100B700008958091F23F9091F33FFC0124853EEF70
:100B8000320F323018F424E024870895243011F015
:100B900080E090E00895CF93DF93C091F23FD09131
:100BA000F33F8C859EEF980F923018F484E08C8789
:100BB00005C0843019F080E090E010C02097D9F390
:100BC000DE011296ED91FC9113978785882329F019
:100BD000EC17FD0711F0DF01F4CFCD01DF91CF91CC
:100BE0000895CF93DF93EC012A813B81888199811D
:100BF0004CEBFB01DE0101900D924A95E1F72A834F
:100C00003B8388839983DF91CF9108958FEE92E1A2
:100C100080930B5990930C598093C8599093C9595C
:100C200008952F923F924F925F926F927F928F9290
:100C30009F92AF92BF92CF92DF92EF92FF920F936B
:100C40001F93CF93DF93CDB7DEB76A97CDBFDEBFDB
:100C50004C011B0129013A01E986FA860B871C87A2
:100C60001A2D0B2DE8A8B9A8AAA82BA92983809131
:100C70003635882399F080912A3590912B35A091B3
:100C80002C35B0912D35BC01CD019F772CEA35EC88
:100C900047E257E30E94D8D587FD11C7809161369E
:100CA00090916236A0916336B0916436BC01CD015B
:100CB0009F7731E03D832CEA35EC47E257E30E9411
:100CC000DBD7181614F01D8210C02DEC3CEC4CEC58
:100CD0005DE36091063670910736809108369091F9
:100CE00009360E94D8D587FDECC6F101808191813B
:100CF000A281B381BC01CD019F77F1E0FD872CEA91
:100D000035EC47E257E30E94DBD718160CF01D863E
:100D1000F10184819581A681B781BC01CD019F77C6
:100D2000F1E0F98B2CEA35EC47E257E30E94DBD780
:100D300018160CF0198AF10180859185A285B3857A
:100D4000209165363091663640916736509168360D
:100D50002E8B3F8B488F598F2091693630916A36A0
:100D600040916B3650916C362A8B3B8B4C8B5D8B54
:100D700040916D3650916E3660916F36709170363D
:100D8000F0903735F11021C01092535981E08093D3
:100D9000545982E0809355593D81332341F04D856C
:100DA000411195C65989511192C68CE9C1C6CB0132
:100DB000BA019F772CEA35EC47E257E30E94DBD774
:100DC00018160CF089C68BE9B3C6BC01CD019F771C
:100DD000A1E0AA8F2CEA35EC47E257E30E94DBD76B
:100DE00018160CF01A8EB1E0FB1216C0109253596F
:100DF00082E080935459F0925559ED81EE2339F0F9
:100E0000FD85F11164C62A8D222379F260C66A89B4
:100E10007B898C899D89CDCF32E0F31217C081E0A8
:100E200080935359F0925459109255594D8144234F
:100E300041F0598951114BC68A8D882309F4B5CFE9
:100E400046C66E897F89888D998DB3CFB101C40163
:100E50000E94044D9D81992309F451C02091F234E0
:100E60003091F3344091F4345091F534609147352A
:100E7000709148358091493590914A350E942FD420
:100E80009F772CEA35EC47E257E30E94D8D587FFDD
:100E900036C02091F6343091F7344091F8345091B7
:100EA000F93460914B3570914C3580914D3590916E
:100EB0004E350E942FD49F772CEA35EC47E257E35A
:100EC0000E94D8D587FF1BC02091FA343091FB34A3
:100ED0004091FC345091FD3460914F357091503504
:100EE00080915135909152350E942FD49F772CEAF2
:100EF00035EC47E257E30E94D8D587FDE4C58CA9BD
:100F00008093F1348DEE94E30E940C4B86E5EDEE78
:100F1000F4E3A2E7B9E501900D928A95E1F788E143
:100F2000E7E4F5E3AEE0B9E501900D928A95E1F7CB
:100F3000809138358111D5C523E333E34BEC51E47F
:100F40006E2D7B2D8A2D99810E947DD84B015C01ED
:100F500060933E5970933F59809340599093415903
:100F600023E333E34BEC51E4C301B2010E947DD88B
:100F70006093265970932759809328599093295943
:100F800023E333E34BEC51E469857A858B859C85BB
:100F90000E947DD860932A5970932B5980932C59C5
:100FA00090932D5923E333E34BEC51E4612F702FE1
:100FB000C6010E947DD8162F072F412F502FBC014C
:100FC00040932E5950932F59609330597093315953
:100FD0008091023690910336A0910436B091053687
:100FE000BC01CD019F770E94B5D60E944CD660937C
:100FF0004F59709350598093515990935259A091E1
:101000005359A98BB0915459BA8BEB2FF0E0ED8373
:10101000FE837F01EE0CFF1CEE0CFF1CF101EE0DB8
:10102000FF1D80819181A281B381BC01CD019F7799
:101030002CEA35EC47E257E30E94D8D5D82EDD1CC8
:10104000DD24DD1C3989232F30E029833A8389018F
:10105000000F111F000F111FF101E00FF11F808120
:101060009181A281B381BC01CD019F772CEA35EC3F
:1010700047E257E30E94D8D5881F8827881F8D2113
:1010800080934E592CEA35EC47E257E3C501B40191
:101090009F770E94DBD718160CF0F9C0F801EE50CC
:1010A000FB4CD801A95BBA4C2D913D914D915C91BF
:1010B00060817181828193810E942FD46B017C01B8
:1010C000ED81FE81EE0FFF1FEE0FFF1FEE50FB4C78
:1010D000AD81BE81AA0FBB1FAA0FBB1FA95BBA4C73
:1010E0002D913D914D915C916081718182819381BF
:1010F0000E942FD469877A878B879C87A5019401EA
:10110000C501B4010E947DD820E030E040E850E401
:101110000E947DD86D877E878F87988BA701960167
:10112000C701B6010E947DD82B013C0129853A8573
:101130004B855C85CA01B9010E947DD89B01AC0139
:10114000C301B2010E9430D49B01AC016D857E8544
:101150008F8598890E942FD42B013C0120E030E03C
:10116000A9010E94DBD71816C4F4C301B2010E9482
:1011700056D92B013C0129853A854B855C85C701F1
:10118000B6010E94E8D79B01AC01C301B20190589F
:101190000E94DFD52B013C0103C0412C512C3201B0
:1011A0008091F134833021F477FA709477F8709459
:1011B00020E030E0A901C501B4010E94D8D587FF25
:1011C00004C077FA709477F8709409811A81000F3F
:1011D000111F000F111FA801455F564A5A01A301B4
:1011E000920169857A858B859C850E947DD89B01BB
:1011F000AC01C701B6010E942FD420E030E040E0EE
:101200005FE30E947DD8D5015B966D937D938D93AE
:101210009C935E97AD80BE80AA0CBB1CAA0CBB1C25
:10122000F501E55FF64A4F01A3019201C701B6013E
:101230000E947DD89B01AC0169857A858B859C8550
:101240000E9430D420E030E040E05FE30E947DD88F
:10125000D4015B966D937D938D939C935E97E09103
:101260005559F0E0EE0FFF1FEE0FFF1FE55FF64A46
:10127000138E148E158E168EB0913E59B987E0915B
:101280003F59ED87209040593090415925C0570172
:10129000F701E55FF64A838D948DA58DB68D9C018F
:1012A000AD015058F801E55FF64A838D948DA58D08
:1012B000B68DBC01CD0190580E94E8D79B01AB01CF
:1012C000BC0140933E5950933F59609340597093ED
:1012D000415929873D871C01D801A55FB64A5B9615
:1012E000CD90DD90ED90FC905E97E981FA81EE0F54
:1012F000FF1FEE0FFF1FE958F64A13962D913D91FF
:101300004D915C91169760817181828193810E94D9
:101310002FD4A70196010E942FD469837A838B83EF
:101320009C83D501A55FB64A5B964D905D906D900C
:101330007C905E97ED81FE81EE0FFF1FEE0FFF1F89
:10134000E958F64A13962D913D914D915C9116976F
:1013500060817181828193810E942FD4A3019201C7
:101360000E942FD46D837E838F8398879B01AC016D
:1013700069817A818B819C810E94E8D729853D858E
:10138000A1010E942FD44B015C01E894B7F820E042
:1013900030E040E85FE3C501B4010E94DBD71816D6
:1013A0000CF4C3C32AE037ED43EA5BE3C501B401A3
:1013B0000E94D8D587FF12C02AE037ED43E25CE3F4
:1013C00069857D85C1010E947DD89B01AC01C50165
:1013D000B4010E94DBD718160CF4A7C3A301920135
:1013E0005058C701B60190580E94A3D44B015C012C
:1013F000609336597093375980933859909339597F
:1014000080913735813039F4412C512C30E8632EEE
:101410003FEB732E06C0412C512C20E8622E2FE3A7
:10142000722E80914E598823D1F160914F5970915D
:10143000505980915159909152590E9478D66B0120
:101440007C012CEA35EC47E257E30E94D8D587FDB2
:1014500010C01091F1342BED3FE049EC50E4C7018E
:10146000B6010E947DD89B01AC01C12CD12C760124
:10147000B9C081E090E0A0E0B0E080934F59909334
:101480005059A0935159B09352591091F1342BED0A
:101490003FE049EC50E4C12CD12C7601A3C02D8152
:1014A0003E814F81588569817A818B819C810E9420
:1014B000A3D469837A838B839C8360933A59709316
:1014C0003B5980933C5990933D59A50194010E944A
:1014D0002FD46B017C019F772CEA35EC47E257E370
:1014E0000E94D8D587FF18C01091F13460914F59F0
:1014F0007091505980915159909152590E9478D6CB
:101500002BED3FE049EC50E40E947DD89B01AC01FB
:10151000C12CD12C760166C029813A814B815C8136
:10152000C501B4010E94DBD71816F4F42BED3FE09F
:1015300049EC50E4C301B2010E947DD89B01AC018B
:1015400069817A818B819C810E9430D460933A5961
:1015500070933B5980933C5990933D59A501940158
:101560000E942FD46B017C011091F134133099F05B
:1015700060914F59709150598091515990915259A1
:101580000E9478D62BED3FE049EC50E40E947DD8D4
:101590009B01AC0127C02BED3FE049EC50E4C301B7
:1015A000B2010E947DD89B01AC01C701B6010E9427
:1015B0002FD47B018C0160914F59709150598091CB
:1015C0005159909152590E9478D62BED3FE049EC49
:1015D00050E40E947DD89B01AC01C701D8016C0189
:1015E0007D010BC0123049F4C301B2010E947DD8C5
:1015F000A70196010E9430D40AC0C301B2010E9423
:101600007DD89B01AC01C701B6010E942FD47B019C
:10161000AB01BC01409342595093435960934459E4
:10162000709345598C0150905559A52DB0E0FD019E
:10163000EE0FFF1FEE0FFF1FE958F64AAA0FBB1F60
:10164000AA0FBB1FA55FB64A13962D913D914D91F0
:101650005C91169760817181828193810E942FD461
:101660004B015C01609346597093475980934859E8
:10167000909349599701A80169857D85C1010E9410
:101680007DD86B017C0160934A5970934B598093CC
:101690004C5990934D59A50194010E94E8D7698354
:1016A0007A838B839C8360933259709333598093F0
:1016B00034599093355980913635811117C0F09186
:1016C0002A35FD8340902B3520912C352E8B30917F
:1016D0002D353A8F10922A3510922B3510922C35D9
:1016E00010922D3581E08093363512C020912A3535
:1016F00030912B3540912C3550912D3569817A816F
:101700008B819C810E94DFD56D83472E8E8B9A8FB3
:10171000598945E3549FF0011124E158FC4C208184
:10172000318142815381C701B6010E94DFD5662E07
:10173000072F182F792E2D81342D4E895A8D0E9416
:10174000D8D587FF04C06D80042D1E897A8C9A89B4
:1017500085E3989FF0011124E158FC4C20813181F0
:1017600042815381C701B6010E94DFD56B017C0124
:101770009B01AC01662D702F812F972D0E94DBD726
:10178000181624F06C2C0D2D1E2D7F2C862D902FDD
:10179000A12FB72D8093565990935759A09358591C
:1017A000B093595920E030E0A901C501B4019F77F9
:1017B0000E94DBD7181684F5A5E35A9EF001112488
:1017C000E158FC4C2081318142815381C501B40133
:1017D0000E94DFD54B015C01E894B7F8A5019401A4
:1017E000662D702F812F972D0E94DBD7181614F4C9
:1017F000A72C04C0682C092D1A2DAB2C862D902FF8
:10180000A12FBA2D8093565990935759A0935859A8
:10181000B0935959B62C02C0B62CA72CC090C03238
:10182000D090C132E090C232F090C33220E030E07C
:1018300040E850E4C701B6010E947DD82B013C016D
:1018400029853D85A10169857D85C1010E9430D42E
:10185000A70196010E942FD49B01AC01C301B201E4
:101860000E947DD80E9456D92B013C0120EC31EE1C
:1018700044E65CE46B2D702F812F9A2D0E947DD859
:1018800020E030E44CE156E40E94DFD56B017C019E
:101890002091C9323091CA324091CB325091CC3232
:1018A00069817A818B819C810E94DFD54B015C012B
:1018B000A301920169817A818B819C810E94DFD58D
:1018C00087017601A50194010E942FC30E94B5D61D
:1018D0007B018C0120E030E040E85FE30E94DBD731
:1018E00018163CF4B701C8010E9447D64B015C01B1
:1018F00008C0812C912C54018394E12CF12C00E838
:101900001FE3C701D80180935A5990935B59A09364
:101910005C59B0935D599701A80160915659709137
:10192000575980915859909159590E94DFD5609329
:10193000A7597093A8598093A9599093AA59809256
:101940005E5990925F59A0926059B0926159970187
:10195000A8016091425970914359809144599091E6
:1019600045590E94DFD56093625970936359809303
:101970006459909365599701A801609146597091F7
:10198000475980914859909149590E94DFD56093F9
:1019900066597093675980936859909369598090FC
:1019A000365990903759A0903859B0903959C5019F
:1019B000B4010E944CD9C0903E59D0903F59E0905C
:1019C0004059F09041590091535910E0000F111FF8
:1019D000000F111F055F164AA70196010E947DD8CE
:1019E0009B01AC01F80163817481858196810E941D
:1019F0002FD460936A5970936B5980936C5990936C
:101A00006D59C501B4010E94DCD59B01AC01009168
:101A1000545910E0000F111F000F111F055F164AE7
:101A2000C701B6010E947DD89B01AC01D801139675
:101A30006D917D918D919C9116970E942FD460930A
:101A40006E5970936F598093705990937159A0910A
:101A50005559B0E0FD01EE0FFF1FEE0FFF1FE958D3
:101A6000F64AAA0FBB1FAA0FBB1FA55FB64A139663
:101A70008D919D910D90BC91A02D80839183A28327
:101A8000B3831092B43F8091325990913359A09111
:101A90003459B0913559BC01CD019F772CEA35EC12
:101AA00047E257E30E94D8D587FD0FC00E947256C7
:101AB00082E080930D590E94674C80E039C08EE827
:101AC00037C08EE935C08FE933C089EC31C0B10130
:101AD000C4010E94044DC2C9B101C4010E94044D59
:101AE0000ECA8E2D9B2DAA2DB98180933E599093BD
:101AF0003F59A0934059B093415940922659509272
:101B00002759609228597092295929853A854B8521
:101B10005C8520932A5930932B5940932C5950932C
:101B20002D594C015D01C60148CA8BE98093B43F31
:101B30006A96CDBFDEBFDF91CF911F910F91FF90CD
:101B4000EF90DF90CF90BF90AF909F908F907F905D
:101B50006F905F904F903F902F9008958F929F923B
:101B6000AF92BF92CF92DF92EF92FF92CF93DF932B
:101B700080910D59882309F4B1C00E94FE838430FE
:101B800010F482E0ACC020916259309163594091C9
:101B900064595091655960913659709137598091C7
:101BA0003859909139590E9430D46B017C0160936F
:101BB00036597093375980933859909339590E9408
:101BC0004CD980903E5990903F59A0904059B09088
:101BD0004159C0915359D0E0CC0FDD1FCC0FDD1F10
:101BE000C958D64AA50194010E947DD89B01AC0139
:101BF00060916A5970916B5980916C5990916D59AF
:101C00000E9430D4688379838A839B83C701B6019D
